:100000000C94BD2B0C94EE2B0C94EE2B0C94EE2B3D
:100010000C94EE2B0C94EE2B0C94EE2B0C94EE2BFC
:100020000C94EE2B0C94EE2B0C94EE2B0C94EE2BEC
:100030000C94EE2B0C942EDB0C94EE2B0C94EE2BEC
:100040000C94EE2B0C945FB90C94EE2B0C94EE2BCD
:100050000C94EE2B0C94EE2B0C94D1420C94F4D611
:100060000C94EE2B0C942DB60C94EE2B0C94EE2BE2
:100070000C94EE2B0C94EE2B0C94EE2B0C94EE2B9C
:100080000C94EE2B0C94EE2B0C94EE2B0C94EE2B8C
:100090000C94EE2B0C94EE2B0C94EE2B0C9426D49B
:1000A0000C94EE2B0C94EE2B0C94EE2B0C94EE2B6C
:1000B0000C94EE2B0C94EE2B0C94EE2B0C94EE2B5C
:1000C0000C94EE2B0C94EE2B0C94EE2B0C94EE2B4C
:1000D0000C94EE2B0C94EE2B0C94EE2B0C94EE2B3C
:1000E0000C94EE2B1E432C434843564370437E43EF
:1000F00098439C439E43A243AA4378D57DD582D59D
:100100008CD505D696D59ED5A6D5B0D5BAD5C4D5AD
:10011000D3D5DDD505D6E7D5F1D5FBD523D626D663
:1001200019D61DD65DD62AD62ED634D638D63CD68C
:1001300042D646D64AD65DD650D654D658D6084A68
:10014000D73B3BCE016E84BCBFFDC12F3D6C7431EB
:100150009ABD56833DDA3D00C77F11BED9E4BB4C42
:100160003E916BAAAABE000000803F05A84CCDB20C
:10017000D44EB93836A9020C50B9918688083CA6ED
:10018000AAAA2ABE000000803F007C3C3E5E2B3DB8
:100190003F2F5B5D3B2C2A225C004572723A204D5A
:1001A000415854454D50204245440054656D70659A
:1001B000726174757265206865617465642062653A
:1001C00064207377697463686564206F66662E20A7
:1001D0004D415854454D502074726967676572658A
:1001E00064202121004572723A204D494E54454DFC
:1001F00050003A204578747275646572207377698F
:100200007463686564206F66662E204D494E5445C0
:100210004D502074726967676572656420210045DE
:1002200072723A204D415854454D50003A2045785D
:10023000747275646572207377697463686564208D
:100240006F66662E204D415854454D50207472699A
:10025000676765726564202100202D20496E7661F4
:100260006C6964206578747275646572206E756D52
:10027000626572202100504944204175746F747585
:100280006E652066696E69736865642120507574B7
:1002900020746865206C617374204B702C204B694E
:1002A00020616E64204B6420636F6E7374616E74A2
:1002B000732066726F6D2061626F766520696E745F
:1002C0006F20436F6E66696775726174696F6E2E19
:1002D0006800504944204175746F74756E652066DE
:1002E00061696C6564212074696D656F75740020A7
:1002F000403A006F6B20543A006F6B20423A005036
:100300004944204175746F74756E65206661696C2F
:100310006564212054656D70657261747572652025
:10032000746F6F206869676800204B643A20002072
:100330004B693A2000204B703A200020436C6173D7
:100340007369632050494420002054753A200020EE
:100350004B753A2000206D61783A2000206D696E5F
:100360003A200020643A200020626961733A20003C
:100370001000C90210012C01400122017001180176
:10038000B0010E01F00104015002FA00B002F000C9
:100390003003E600D003DC009004D2007005C800F2
:1003A000A006BE000008B400B009AA00D00BA0004F
:1003B000600E960060118C000015820020197800F4
:1003C000C01D6E00A0226400B0275A00902C50007F
:1003D00000314600E0343C0010383200903A2800EA
:1003E000603C1E00A03D1400803E0A00203F00003B
:1003F00070012C0190012701B0012201C0011D01F3
:10040000F00118011002130130020E01600209010F
:1004100090020401C002FF000003FA004003F5004F
:100420008003F000D003EB002004E6007004E1003C
:10043000E004DC004005D700C005D2004006CD0036
:10044000D006C8008007C3003008BE00F008B9001D
:10045000C009B400B00AAF00B00BAA00D00CA500D0
:10046000000EA000500F9B00C0109600501291008B
:1004700000148C00C0158700B0178200B0197D00F1
:10048000D01B7800001E730040206E00902269008F
:10049000F024640040275F0090295A00E02B5500AB
:1004A000102E500020304B0010324600E033410047
:1004B00090353C001037370070383200A0392D00DD
:1004C000B03A2800A03B2300603C1E00103D1900FC
:1004D000903D1400103E0F00703E0A00C03E050023
:1004E000003F0000686F77746F2E70727573613310
:1004F000642E637A00686F77746F2E707275736103
:1005000033642E636F6D00686F77746F2E70727531
:10051000736133642E636F6D00686F77746F2E7034
:100520007275736133642E637A00686F77746F2E0F
:10053000707275736133642E636F6D00666F7275D0
:100540006D2E707275736133642E637A00666F72FC
:10055000756D2E707275736133642E636F6D0066F6
:100560006F72756D2E707275736133642E636F6D6B
:1005700000666F72756D2E707275736133642E63D1
:100580007A00666F72756D2E707275736133642EAA
:10059000636F6D00707275736133642E637A0070DF
:1005A0007275736133642E636F6D00707275736161
:1005B00033642E636F6D00707275736133642E63E4
:1005C0007A00707275736133642E636F6D005779B2
:1005D000626F72206A657A796B612020202020206A
:1005E00020200043616D626961206C61206C656E42
:1005F000677561200053656C657A2E206C61206CF4
:10060000696E677561005679626572206A617A79F0
:100610006B6120202020202020200053656C656322
:1006200074206C616E677561676520202020200052
:10063000506F6C736B6900457370616E6F6C00492D
:1006400074616C69616E6F0043657374696E6100FB
:10065000456E676C697368004572726F7220696ECF
:10066000206D656E752073747275637475726500A4
:100670004572726F7220696E206D656E752073749D
:1006800072756374757265004572726F7220696E5F
:10069000206D656E75207374727563747572650074
:1006A0004572726F7220696E206D656E752073746D
:1006B00072756374757265004572726F7220696E2F
:1006C000206D656E75207374727563747572650044
:1006D000446F737461766F76616E69205A0041646D
:1006E0006A757374696E67205A0041646A75737421
:1006F000696E67205A00446F737461766F76616E1D
:1007000069205A0041646A757374696E67205A00E3
:10071000426162797374657070696E672059004236
:100720006162797374657070696E67205900426107
:1007300062797374657070696E67205900426162F6
:10074000797374657070696E6720590042616279CF
:100750007374657070696E672059004261627973C5
:1007600074657070696E67205800426162797374B5
:10077000657070696E6720580042616279737465B4
:100780007070696E67205800426162797374657099
:1007900070696E6720580042616279737465707089
:1007A000696E6720580020746F6F206C6F6E672031
:1007B000657874727573696F6E2070726576656E98
:1007C0007465640020746F6F206C6F6E67206578AD
:1007D00074727573696F6E2070726576656E74657C
:1007E000640020746F6F206C6F6E67206578747280
:1007F0007573696F6E2070726576656E74656400DE
:1008000020746F6F206C6F6E6720657874727573DB
:10081000696F6E2070726576656E74656400207411
:100820006F6F206C6F6E6720657874727573696F77
:100830006E2070726576656E7465640020636F6CFF
:100840006420657874727573696F6E207072657656
:10085000656E7465640020636F6C642065787472E3
:100860007573696F6E2070726576656E746564006D
:1008700020636F6C6420657874727573696F6E2085
:1008800070726576656E7465640020636F6C6420B9
:10089000657874727573696F6E2070726576656EB7
:1008A0007465640020636F6C64206578747275737E
:1008B000696F6E2070726576656E74656400656E32
:1008C0006473746F7073206869743A2000656E6495
:1008D00073746F7073206869743A2000656E647376
:1008E000746F7073206869743A2000656E64737465
:1008F0006F7073206869743A2000656E6473746F5A
:100900007073206869743A20005374657072617462
:100910006520746F6F20686967683A2000537465BA
:10092000707261746520746F6F20686967683A201F
:1009300000537465707261746520746F6F2068690C
:1009400067683A2000537465707261746520746F33
:100950006F20686967683A2000537465707261742B
:100960006520746F6F20686967683A200043616E84
:100970006E6F7420656E746572207375626469723F
:100980003A200043616E6E6F7420656E746572204C
:100990007375626469723A200043616E6E6F7420F1
:1009A000656E746572207375626469723A200043E3
:1009B000616E6E6F7420656E74657220737562640B
:1009C00069723A200043616E6E6F7420656E7465C3
:1009D00072207375626469723A20006572726F7278
:1009E0002077726974696E6720746F2066696C6520
:1009F000006572726F722077726974696E67207415
:100A00006F2066696C65006572726F72207772691B
:100A100074696E6720746F2066696C650065727218
:100A20006F722077726974696E6720746F206669CF
:100A30006C65006572726F722077726974696E6797
:100A400020746F2066696C65004E6F7420534420DB
:100A50007072696E74696E67004E6F742053442023
:100A60007072696E74696E67004E6F742053442013
:100A70007072696E74696E67004E6F742053442003
:100A80007072696E74696E67004E6F7420534420F3
:100A90007072696E74696E67005344207072696E7B
:100AA00074696E6720627974652000534420707207
:100AB000696E74696E672062797465200053442002
:100AC0007072696E74696E67206279746520005374
:100AD00044207072696E74696E6720627974652053
:100AE000005344207072696E74696E672062797475
:100AF00065200057726974696E6720746F2066699B
:100B00006C653A200057726974696E6720746F20B3
:100B100066696C653A200057726974696E67207463
:100B20006F2066696C653A200057726974696E6758
:100B300020746F2066696C653A2000577269746989
:100B40006E6720746F2066696C653A200046696C98
:100B5000652073656C65637465640046696C652027
:100B600073656C65637465640046696C65207365C4
:100B70006C65637465640046696C652073656C65BB
:100B8000637465640046696C652073656C656374A5
:100B90006564002053697A653A20002053697A65BC
:100BA0003A20002053697A653A20002053697A651B
:100BB0003A20002053697A653A200046696C652026
:100BC0006F70656E65643A200046696C65206F70D1
:100BD000656E65643A200046696C65206F70656ECD
:100BE00065643A200046696C65206F70656E6564C7
:100BF0003A200046696C65206F70656E65643A2026
:100C0000006F70656E206661696C65642C204669B2
:100C10006C653A20006F70656E206661696C656472
:100C20002C2046696C653A20006F70656E20666105
:100C3000696C65642C2046696C653A20006F7065AC
:100C40006E206661696C65642C2046696C653A208B
:100C5000006F70656E206661696C65642C20466962
:100C60006C653A2000776F726B446972206F706513
:100C70006E206661696C656400776F726B4469729F
:100C8000206F70656E206661696C656400776F72B5
:100C90006B446972206F70656E206661696C656473
:100CA00000776F726B446972206F70656E206661A9
:100CB000696C656400776F726B446972206F706550
:100CC0006E206661696C65640053442063617264E0
:100CD000206F6B0053442063617264206F6B00537C
:100CE000442063617264206F6B005344206361721F
:100CF00064206F6B0053442063617264206F6B004B
:100D00006F70656E526F6F74206661696C65640008
:100D10006F70656E526F6F74206661696C656400F8
:100D20006F70656E526F6F74206661696C656400E8
:100D30006F70656E526F6F74206661696C656400D8
:100D40006F70656E526F6F74206661696C656400C8
:100D5000766F6C756D652E696E6974206661696C5D
:100D6000656400766F6C756D652E696E69742066BA
:100D700061696C656400766F6C756D652E696E696E
:100D800074206661696C656400766F6C756D652EA4
:100D9000696E6974206661696C656400766F6C7554
:100DA0006D652E696E6974206661696C65640053B7
:100DB0004420696E6974206661696C00534420693F
:100DC0006E6974206661696C00534420696E6974B1
:100DD000206661696C00534420696E697420666105
:100DE000696C00534420696E6974206661696C0007
:100DF00043616E6E6F74206F70656E2073756264F0
:100E000069720043616E6E6F74206F70656E20733F
:100E100075626469720043616E6E6F74206F7065F5
:100E20006E207375626469720043616E6E6F742028
:100E30006F70656E207375626469720043616E6ED7
:100E40006F74206F70656E207375626469720048FC
:100E50006F74656E64206F6666736574733A0048DC
:100E60006F74656E64206F6666736574733A0048CC
:100E70006F74656E64206F6666736574733A0048BC
:100E80006F74656E64206F6666736574733A0048AC
:100E90006F74656E64206F6666736574733A006F75
:100EA00070656E006F70656E006F70656E006F70BC
:100EB000656E006F70656E00545249474745524554
:100EC000440054524947474552454400545249470B
:100ED000474552454400545249474745524544000E
:100EE000545249474745524544005265706F7274E9
:100EF000696E6720656E6473746F702073746174BB
:100F00007573005265706F7274696E6720656E64E8
:100F100073746F7020737461747573005265706FB1
:100F20007274696E6720656E6473746F7020737479
:100F300061747573005265706F7274696E672065B5
:100F40006E6473746F70207374617475730052658E
:100F5000706F7274696E6720656E6473746F702051
:100F6000737461747573007A5F6D61783A20007AEA
:100F70005F6D61783A20007A5F6D61783A20007A7F
:100F80005F6D61783A20007A5F6D61783A20007A6F
:100F90005F6D696E3A20007A5F6D696E3A20007A63
:100FA0005F6D696E3A20007A5F6D696E3A20007A53
:100FB0005F6D696E3A2000795F6D61783A20007943
:100FC0005F6D61783A2000795F6D61783A20007931
:100FD0005F6D61783A2000795F6D61783A20007921
:100FE0005F6D696E3A2000795F6D696E3A20007915
:100FF0005F6D696E3A2000795F6D696E3A20007905
:101000005F6D696E3A2000785F6D61783A200078F4
:101010005F6D61783A2000785F6D61783A200078E2
:101020005F6D61783A2000785F6D61783A200078D2
:101030005F6D696E3A2000785F6D696E3A200078C6
:101040005F6D696E3A2000785F6D696E3A200078B6
:101050005F6D696E3A2000496E76616C6964206547
:101060007874727564657200496E76616C6964208B
:10107000657874727564657200496E76616C696436
:1010800020657874727564657200496E76616C696A
:101090006420657874727564657200496E76616C5F
:1010A000696420657874727564657200416374695F
:1010B00076652045787472756465723A20004163E4
:1010C000746976652045787472756465723A20009B
:1010D0004163746976652045787472756465723A07
:1010E0002000416374697665204578747275646583
:1010F000723A200041637469766520457874727590
:101100006465723A2000556E6B6E6F776E20636F68
:101110006D6D616E643A202200556E6B6E6F776E56
:1011200020636F6D6D616E643A202200556E6B6EA8
:101130006F776E20636F6D6D616E643A202200558B
:101140006E6B6E6F776E20636F6D6D616E643A20AB
:101150002200556E6B6E6F776E20636F6D6D616EE2
:10116000643A202200526573656E643A200052652D
:1011700073656E643A2000526573656E643A2000B0
:10118000526573656E643A2000526573656E643A09
:1011900020005072696E7465722073746F70706590
:1011A000642064756520746F206572726F72732E8F
:1011B0002046697820746865206572726F722061BC
:1011C0006E6420757365204D39393920746F207233
:1011D0006573746172742E202854656D7065726138
:1011E000747572652069732072657365742E20535F
:1011F0006574206974206166746572207265737409
:10120000617274696E6729005072696E746572202C
:1012100073746F707065642064756520746F2065E9
:1012200072726F72732E204669782074686520652B
:1012300072726F7220616E6420757365204D39394A
:101240003920746F20726573746172742E20285473
:10125000656D706572617475726520697320726561
:101260007365742E205365742069742061667465FB
:10127000722072657374617274696E6729005072AE
:10128000696E7465722073746F7070656420647524
:101290006520746F206572726F72732E20466978B4
:1012A00020746865206572726F7220616E642075AB
:1012B0007365204D39393920746F207265737461FC
:1012C00072742E202854656D706572617475726534
:1012D0002069732072657365742E205365742069CC
:1012E00074206166746572207265737461727469CA
:1012F0006E6729005072696E7465722073746F7026
:101300007065642064756520746F206572726F72F9
:10131000732E2046697820746865206572726F723A
:1013200020616E6420757365204D39393920746FE2
:1013300020726573746172742E202854656D706517
:101340007261747572652069732072657365742E9D
:10135000205365742069742061667465722072651B
:101360007374617274696E6729005072696E746576
:10137000722073746F707065642064756520746F7B
:10138000206572726F72732E2046697820746865CA
:10139000206572726F7220616E6420757365204DD6
:1013A00039393920746F20726573746172742E201C
:1013B0002854656D7065726174757265206973205B
:1013C00072657365742E205365742069742061669C
:1013D0007465722072657374617274696E67290036
:1013E0005072696E7465722068616C7465642E2039
:1013F0006B696C6C28292063616C6C6564210050FA
:1014000072696E7465722068616C7465642E206BFD
:10141000696C6C28292063616C6C656421005072D2
:10142000696E7465722068616C7465642E206B69E6
:101430006C6C28292063616C6C65642100507269B2
:101440006E7465722068616C7465642E206B696CC3
:101450006C28292063616C6C656421005072696E90
:101460007465722068616C7465642E206B696C6CA5
:1014700028292063616C6C6564210020436F756EC0
:101480007420583A200020436F756E7420583A201B
:101490000020436F756E7420583A200020436F750A
:1014A0006E7420583A200020436F756E7420583AAD
:1014B00020004649524D574152455F4E414D453AF5
:1014C0004D61726C696E2056312E302E323B2053A6
:1014D0007072696E7465722F6772626C206D6173D1
:1014E00068757020666F722067656E3620464952B7
:1014F0004D574152455F55524C3A68747470733A77
:101500002F2F6769746875622E636F6D2F70727507
:10151000736133642F50727573612D69332D506C74
:1015200075732F2050524F544F434F4C5F564552C6
:1015300053494F4E3A312E30204D414348494E4594
:101540005F545950453A5072757361206933204594
:10155000585452554445525F434F554E543A3120EA
:10156000555549443A30303030303030302D3030FD
:1015700030302D303030302D303030302D30303074
:101580003030303030303030300A004649524D571C
:101590004152455F4E414D453A4D61726C696E2036
:1015A00056312E302E323B20537072696E74657244
:1015B0002F6772626C206D617368757020666F7240
:1015C0002067656E36204649524D574152455F555A
:1015D000524C3A68747470733A2F2F676974687547
:1015E000622E636F6D2F707275736133642F50724A
:1015F0007573612D69332D506C75732F2050524FC8
:10160000544F434F4C5F56455253494F4E3A312E3B
:1016100030204D414348494E455F545950453A505A
:1016200072757361206933204558545255444552B0
:101630005F434F554E543A3120555549443A303066
:101640003030303030302D303030302D30303030A0
:101650002D303030302D3030303030303030303090
:1016600030300A004649524D574152455F4E414D78
:10167000453A4D61726C696E2056312E302E323BE8
:1016800020537072696E7465722F6772626C206D80
:10169000617368757020666F722067656E362046CC
:1016A00049524D574152455F55524C3A68747470D7
:1016B000733A2F2F6769746875622E636F6D2F7090
:1016C0007275736133642F50727573612D69332D98
:1016D000506C75732F2050524F544F434F4C5F56F0
:1016E000455253494F4E3A312E30204D41434849DF
:1016F0004E455F545950453A5072757361206933B5
:101700002045585452554445525F434F554E543A24
:101710003120555549443A30303030303030302D5A
:10172000303030302D303030302D303030302D30C2
:1017300030303030303030303030300A00464952AE
:101740004D574152455F4E414D453A4D61726C696E
:101750006E2056312E302E323B20537072696E74DB
:1017600065722F6772626C206D6173687570206698
:101770006F722067656E36204649524D574152457B
:101780005F55524C3A68747470733A2F2F676974BE
:101790006875622E636F6D2F707275736133642F7D
:1017A00050727573612D69332D506C75732F2050F5
:1017B000524F544F434F4C5F56455253494F4E3A48
:1017C000312E30204D414348494E455F54595045D4
:1017D0003A5072757361206933204558545255440C
:1017E00045525F434F554E543A3120555549443A7E
:1017F00030303030303030302D303030302D3030EF
:1018000030302D303030302D3030303030303030DE
:10181000303030300A004649524D574152455F4EF4
:10182000414D453A4D61726C696E2056312E302E15
:10183000323B20537072696E7465722F6772626CEE
:10184000206D617368757020666F722067656E36F3
:10185000204649524D574152455F55524C3A6874A3
:101860007470733A2F2F6769746875622E636F6D99
:101870002F707275736133642F50727573612D69A7
:10188000332D506C75732F2050524F544F434F4C93
:101890005F56455253494F4E3A312E30204D414309
:1018A00048494E455F545950453A5072757361200E
:1018B00069332045585452554445525F434F554E65
:1018C000543A3120555549443A3030303030303078
:1018D000302D303030302D303030302D3030303011
:1018E0002D3030303030303030303030300A00532E
:1018F000746F6C696B204F4B2E0042617365206CD6
:101900006973746F2E0050696174746F206661741E
:10191000746F2E00426564204F4B2E004265642098
:10192000646F6E652E0047727A616E69652073740C
:101930006F6C696B612E2E00426173652043616C90
:10194000656E74616E646F0050696174746F2072AB
:10195000697363616C64616D2E005A6168726976A7
:10196000616E69206265642E2E2E004265642048F7
:10197000656174696E672E0047727A616E696520D1
:101980004F4B2E0043616C656E74616E646F206C0A
:101990006973746F2E0052697363616C64616D6565
:1019A0006E746F20666174746F2E005A616872697C
:1019B00076616E69204F4B2E0048656174696E67D1
:1019C00020646F6E652E0047727A616E69652E2EF7
:1019D0002E0043616C656E74616E646F2E2E2E0056
:1019E00052697363616C64616D656E746F2E2E2E27
:1019F000005A6168726976616E692E2E2E00486504
:101A00006174696E672E2E2E004D31303920496E7B
:101A100076616C6964206578747275646572200003
:101A20004D31303920496E76616C69642065787477
:101A3000727564657220004D31303920496E7661CF
:101A40006C696420657874727564657220004D312C
:101A5000303920496E76616C6964206578747275DE
:101A600064657220004D31303920496E76616C69B1
:101A70006420657874727564657220004E6F2074FE
:101A80006865726D6973746F7273202D206E6F209C
:101A900074656D7065726174757265004E6F207447
:101AA0006865726D6973746F7273202D206E6F207C
:101AB00074656D7065726174757265004E6F207427
:101AC0006865726D6973746F7273202D206E6F205C
:101AD00074656D7065726174757265004E6F207407
:101AE0006865726D6973746F7273202D206E6F203C
:101AF00074656D7065726174757265004E6F2074E7
:101B00006865726D6973746F7273202D206E6F201B
:101B100074656D7065726174757265004D32323135
:101B200020496E76616C69642065787472756465AD
:101B30007220004D32323120496E76616C6964202A
:101B4000657874727564657220004D3232312049B7
:101B50006E76616C69642065787472756465722054
:101B6000004D32323120496E76616C6964206578AF
:101B700074727564657220004D32323120496E7680
:101B8000616C696420657874727564657220004DBB
:101B900032313820496E76616C69642065787472E0
:101BA0007564657220004D32313820496E76616C63
:101BB000696420657874727564657220004D3231F5
:101BC0003820496E76616C6964206578747275643A
:101BD000657220004D32313820496E76616C69643F
:101BE00020657874727564657220004D323138203A
:101BF000496E76616C69642065787472756465728B
:101C000020004D32303020496E76616C6964206569
:101C10007874727564657220004D32303020496EE0
:101C200076616C69642065787472756465722000F1
:101C30004D32303020496E76616C6964206578746D
:101C4000727564657220004D32303020496E7661C5
:101C50006C696420657874727564657220004D3219
:101C6000303020496E76616C6964206578747275D5
:101C700064657220004D31303520496E76616C69A3
:101C80006420657874727564657220004D3130355A
:101C900020496E76616C696420657874727564653C
:101CA0007220004D31303520496E76616C696420B8
:101CB000657874727564657220004D313035204945
:101CC0006E76616C696420657874727564657220E3
:101CD000004D31303520496E76616C69642065783D
:101CE00074727564657220004D31303420496E760F
:101CF000616C696420657874727564657220004D4A
:101D000031303420496E76616C6964206578747274
:101D10007564657220004D31303420496E76616CF7
:101D2000696420657874727564657220004D313085
:101D30003420496E76616C696420657874727564CC
:101D4000657220004D31303420496E76616C6964D3
:101D50002065787472756465722000456E64206633
:101D6000696C65206C69737400456E642066696CEB
:101D700065206C69737400456E642066696C65202B
:101D80006C69737400456E642066696C65206C69CB
:101D9000737400456E642066696C65206C697374A9
:101DA00000426567696E2066696C65206C697374B2
:101DB00000426567696E2066696C65206C697374A2
:101DC00000426567696E2066696C65206C69737492
:101DD00000426567696E2066696C65206C69737482
:101DE00000426567696E2066696C65206C69737472
:101DF00000446F6E65207072696E74696E6720664C
:101E0000696C6500446F6E65207072696E74696EEE
:101E1000672066696C6500446F6E65207072696E3C
:101E200074696E672066696C6500446F6E6520702A
:101E300072696E74696E672066696C6500446F6EC6
:101E400065207072696E74696E672066696C6500E2
:101E50004E6F204C696E65204E756D6265722077FD
:101E600069746820636865636B73756D2C204C61C1
:101E70007374204C696E653A20004E6F204C696E79
:101E800065204E756D62657220776974682063689D
:101E900065636B73756D2C204C617374204C696E97
:101EA000653A20004E6F204C696E65204E756D625C
:101EB0006572207769746820636865636B73756DFC
:101EC0002C204C617374204C696E653A20004E6F73
:101ED000204C696E65204E756D626572207769745D
:101EE0006820636865636B73756D2C204C61737437
:101EF000204C696E653A20004E6F204C696E65205B
:101F00004E756D62657220776974682063686563D9
:101F10006B73756D2C204C617374204C696E653A3F
:101F200020004E6F20436865636B73756D20776981
:101F30007468206C696E65206E756D6265722C2008
:101F40004C617374204C696E653A20004E6F2043DB
:101F50006865636B73756D2077697468206C696E52
:101F600065206E756D6265722C204C617374204C17
:101F7000696E653A20004E6F20436865636B737528
:101F80006D2077697468206C696E65206E756D626E
:101F900065722C204C617374204C696E653A200088
:101FA0004E6F20436865636B73756D207769746845
:101FB000206C696E65206E756D6265722C204C61B7
:101FC0007374204C696E653A20004E6F204368653B
:101FD000636B73756D2077697468206C696E65201A
:101FE0006E756D6265722C204C617374204C696E45
:101FF000653A2000636865636B73756D206D697366
:102000006D617463682C204C617374204C696E653B
:102010003A2000636865636B73756D206D69736D3D
:10202000617463682C204C617374204C696E653A4E
:102030002000636865636B73756D206D69736D61F6
:102040007463682C204C617374204C696E653A206F
:1020500000636865636B73756D206D69736D617482
:1020600063682C204C617374204C696E653A2000C3
:10207000636865636B73756D206D69736D617463FF
:10208000682C204C617374204C696E653A20004CBA
:10209000696E65204E756D626572206973206E6F82
:1020A00074204C617374204C696E65204E756D62AE
:1020B00065722B312C204C617374204C696E653A2B
:1020C00020004C696E65204E756D626572206973E3
:1020D000206E6F74204C617374204C696E65204EC5
:1020E000756D6265722B312C204C617374204C69C4
:1020F0006E653A20004C696E65204E756D626572A2
:10210000206973206E6F74204C617374204C696E6B
:1021100065204E756D6265722B312C204C61737495
:10212000204C696E653A20004C696E65204E756DD5
:10213000626572206973206E6F74204C6173742025
:102140004C696E65204E756D6265722B312C204C8A
:10215000617374204C696E653A20004C696E65208D
:102160004E756D626572206973206E6F74204C61CC
:102170007374204C696E65204E756D6265722B31EB
:102180002C204C617374204C696E653A2000446FBA
:102190006E6520736176696E672066696C652E00D6
:1021A000446F6E6520736176696E672066696C6541
:1021B0002E00446F6E6520736176696E67206669D4
:1021C0006C652E00446F6E6520736176696E6720C2
:1021D00066696C652E00446F6E6520736176696E6A
:1021E000672066696C652E006F6B006F6B006F6B0C
:1021F000006F6B006F6B002020506C616E6E65721B
:1022000042756666657242797465733A20002020D3
:10221000506C616E6E657242756666657242797465
:1022200065733A20002020506C616E6E65724275B5
:102230006666657242797465733A20002020506C9E
:10224000616E6E6572427566666572427974657319
:102250003A20002020506C616E6E65724275666691
:10226000657242797465733A200020467265652074
:102270004D656D6F72793A20002046726565204D7C
:10228000656D6F72793A20002046726565204D6554
:102290006D6F72793A20002046726565204D656D3C
:1022A0006F72793A20002046726565204D656D6F2A
:1022B00072793A2000204C61737420557064617407
:1022C00065643A2000204C61737420557064617419
:1022D00065643A2000204C61737420557064617409
:1022E00065643A2000204C617374205570646174F9
:1022F00065643A2000204C617374205570646174E9
:1023000065643A2000207C20417574686F723A2021
:1023100000207C20417574686F723A2000207C2078
:10232000417574686F723A2000207C204175746892
:102330006F723A2000207C20417574686F723A20D9
:102340000020536F667477617265205265736574FF
:102350000020536F667477617265205265736574EF
:102360000020536F667477617265205265736574DF
:102370000020536F667477617265205265736574CF
:102380000020536F667477617265205265736574BF
:1023900000205761746368646F67205265736574C9
:1023A00000205761746368646F67205265736574B9
:1023B00000205761746368646F67205265736574A9
:1023C00000205761746368646F6720526573657499
:1023D00000205761746368646F6720526573657489
:1023E000002042726F776E206F757420526573659E
:1023F00074002042726F776E206F7574205265737F
:102400006574002042726F776E206F75742052657C
:10241000736574002042726F776E206F757420525E
:1024200065736574002042726F776E206F7574203B
:102430005265736574002045787465726E616C2016
:102440005265736574002045787465726E616C2006
:102450005265736574002045787465726E616C20F6
:102460005265736574002045787465726E616C20E6
:102470005265736574002045787465726E616C20D6
:10248000526573657400506F776572557000506FB8
:10249000776572557000506F776572557000506F98
:1024A000776572557000506F776572557000656E74
:1024B000717565696E67202200656E717565696E5C
:1024C00067202200656E717565696E672022006560
:1024D0006E717565696E67202200656E717565693C
:1024E0006E672022007770726F772E207A6D696197
:1024F0006E007061726120746F6D61722065666537
:1025000063746F0020706572206D6F7374726172F6
:102510006520692063616D622E002070726F2070EB
:10252000726F6A6576656E69207A6D656E002066E9
:102530006F722074616B6520656666656374005216
:10254000657374617274206472756B61726B69007B
:102550005265696E6963696172206C6120696D7092
:102560002E005269617676696F206C612073746108
:102570006D702E0052657374617274756A74652093
:102580007469736B61726E75005265626F6F74204F
:10259000746865207072696E746572004D6F642096
:1025A0005B7720777964616A6E6F73635D004D6F4E
:1025B000646F205B6D617320667565727A615D0082
:1025C0004D6F646F205B70697520666F727A615D14
:1025D000004D6F6420205B7679732E2076796B6FC7
:1025E0006E5D004D6F6465205B6869676820706F81
:1025F0007765725D004D6F64202020202020205BD5
:1026000063696368795D004D6F646F20202020202E
:102610005B73696C656E63696F5D004D6F646F20FD
:10262000202020205B73696C656E7A696F736F5D23
:10263000004D6F64202020202020205B7469636897
:10264000795D004D6F646520202020205B73696CEC
:10265000656E745D0057796D69616E612066696CA5
:10266000616D656E74750043616D6269616E646F62
:102670002066696C2E21004D757465766F6C65203F
:1026800066696C2E210056796D656E612066696CF5
:10269000616D656E747521004368616E67696E6770
:1026A0002066696C616D656E7421005770726F777A
:1026B00061647A2066696C616D656E7400496E7341
:1026C000657274612066696C616D656E746F004936
:1026D0006E7365726972652066696C616D656E7492
:1026E0006F00566C6F7A74652066696C616D656EFB
:1026F0007400496E736572742066696C616D656EF5
:1027000074004E616369736E696A2070727A7963CE
:1027100069736B00592070756C736520656C206D52
:10272000616E646F00592070756C736520656C2054
:102730006D616E646F004120737469736B6E6574B4
:102740006520746C616369746B6F00416E64207006
:102750007265737320746865206B6E6F62005779C1
:102760006D69616E61206F6B210043616D6269610B
:1027700072206269656E210043616D6269612E207D
:10278000726975736369746F21005A6D656E61209B
:1027900075737065736E6121004368616E676520B3
:1027A000737563636573732100437A79737A637A0F
:1027B0002E206B6F6C6F72750043617267616E647F
:1027C0006F20636F6C6F720043617267616E646F3C
:1027D00020636F6C6F720043697374656E69206269
:1027E00061727679004C6F6164696E6720636F6C0B
:1027F0006F720050726F737A6520637A656B6163E4
:102800000045737065726100417370657474610096
:1028100050726F73696D2063656B656A74650050F3
:102820006C656173652077616974005770726F77AA
:102830002E2066696C616D656E7475004361726708
:10284000616E646F2066696C2E0043617267616E11
:10285000646F2066696C2E005A61766164656E69EA
:102860002066696C616D656E7475004C6F6164699A
:102870006E672066696C616D656E74004B6F6C6F7E
:1028800072207A616E6965637A79737A2E00436F7C
:102890006C6F72206E6F20636C61726F00436F6C9F
:1028A0006F72206E6F20636C61726F00426172768E
:1028B00061206E656E6920636973746100436F6C9B
:1028C0006F72206E6F7420636C656172004272617A
:1028D0006B2066696C616D656E74750046696C2E5F
:1028E000206E6F206361726761646F0046696C2EB1
:1028F000206E6F206361726761646F0046696C616E
:102900006D656E74206E657A61766564656E0046ED
:10291000696C616D656E74206E6F74206C6F61649C
:102920006564004E6965004E6F004E6F004E650095
:102930004E6F0054616B00536900536900416E6F24
:10294000005965730057796D69616E61206F6B3F47
:102950000043616D626961646F20636F72726563C9
:102960002E3F0043616D626961746F20636F727204
:102970002E3F0056796D656E61206F6B3F00436896
:10298000616E67656420636F72726563746C793F12
:1029900000506F6D6F6300537570706F72740053E9
:1029A0007570706F727400506F64706F7261005355
:1029B0007570706F7274004E6167727A656A206418
:1029C00079737A65210050726563616C2E20657899
:1029D000747275736F7221005072657269732E2064
:1029E0007567656C6C6F210050726564656872650F
:1029F0006A746520747279736B7521005072656812
:102A000065617420746865206E6F7A7A6C65210048
:102A1000424C41443A004552524F523A00455252BC
:102A20004F523A0043485942413A004552524F52A0
:102A30003A00526563747261637400526563747224
:102A400061637400526563747261637400526563FC
:102A500074726163740052656374726163740057C9
:102A600070726F7761647A2066696C616D656E74EF
:102A700000496E74726F64756369722066696C6177
:102A80006D656E746F004361726963617265206683
:102A9000696C616D656E746F005A61766573742040
:102AA00066696C616D656E74004C6F616420666967
:102AB0006C616D656E740057796A61632066696C3C
:102AC000616D656E740053616361722066696C614B
:102AD0006D656E746F005363617269636172652026
:102AE00066696C2E0056796A6D6F75742066696C24
:102AF000616D656E7400556E6C6F61642066696C03
:102B0000616D656E740047727A616E69650050721E
:102B10006563616C656E7461720050726572697391
:102B200063616C646100507265646568726576000B
:102B30005072656865617400557374617769656E7C
:102B4000696100416A7573746500496D706F7374D3
:102B5000617A696F6E69004E6173746176656E6942
:102B60000053657474696E6773004B616C696272BF
:102B70006F776163205A0047726164756172205AF1
:102B80000043616C696272617465205A004B616C2C
:102B90006962726F766174205A0043616C69627277
:102BA000617465205A004175746F646F7374726F3D
:102BB0006963205A3F004175746F204D6963726FDD
:102BC0007061736F205A3F004175746F20726567A2
:102BD0006F6C617265205A203F004175746F2064EC
:102BE0006F6C61646974205A203F004175746F20D6
:102BF00061646A757374205A203F00456E64737473
:102C00006F702061626F727400456E6473746F70D0
:102C10002061626F727400456E6473746F7020611E
:102C2000626F727400456E6473746F702061626FBE
:102C3000727400456E6473746F702061626F727499
:102C400000446F7374726F6A656E6965206F737983
:102C5000205A004D6963726F7061736F205A004291
:102C600061627973746570205A00446F6C616465A9
:102C70006E69206F7379205A004C69766520616413
:102C80006A757374205A00426162797374657020AA
:102C90005900426162797374657020590042616223
:102CA000797374657020590042616279737465703C
:102CB0002059004261627973746570205900426145
:102CC000627973746570205800426162797374652B
:102CD0007020580042616279737465702058004218
:102CE000616279737465702058004261627973740F
:102CF00065702058005A204F6666736574005A202C
:102D00004F6666736574005A204F6666736574007B
:102D10005A204F6666736574005A204F6666736565
:102D20007400486F6D6520582F59206265666F7278
:102D300065205A00486F6D6520582F5920626566DE
:102D40006F7265205A00486F6D6520582F592062B8
:102D500065666F7265205A00486F6D6520582F595F
:102D6000206265666F7265205A00486F6D65205855
:102D70002F59206265666F7265205A005A20707262
:102D80006F6265206F75742E20626564005A207032
:102D9000726F6265206F75742E20626564005A2020
:102DA00070726F6265206F75742E20626564005AC0
:102DB0002070726F6265206F75742E2062656400EA
:102DC0005A2070726F6265206F75742E2062656480
:102DD0000056796D656E6974205344004368616ED6
:102DE00067652053442063617264004368616E67C5
:102DF0006520534420636172640056796D656E6985
:102E000074205344004368616E6765205344206317
:102E100061726400496E69632E20534400496E69F3
:102E2000742E205344206361726400496E69742ECD
:102E3000205344206361726400496E69632E2053FD
:102E40004400496E69742E2053442063617264000B
:102E500057796D69656E69632066696C616D656E31
:102E6000740043616D626961722066696C616D65B1
:102E70006E746F0043616D62696172652066696C92
:102E8000616D656E746F0056796D656E697420664C
:102E9000696C616D656E74004368616E676520667C
:102EA000696C616D656E74004175746F5265747202
:102EB0002E004175746F526574722E004175746FE7
:102EC000526574722E004175746F526574722E00D3
:102ED0004175746F526574722E00556E5265742080
:102EE000205600556E52657420205600556E52656E
:102EF0007420205600556E52657420205600556E81
:102F0000526574202056005320556E5265742B6D07
:102F10006D005320556E5265742B6D6D0053205516
:102F20006E5265742B6D6D005320556E5265742B77
:102F30006D6D005320556E5265742B6D6D00556E8E
:102F4000526574202B6D6D00556E526574202B6D8B
:102F50006D00556E526574202B6D6D00556E526577
:102F600074202B6D6D00556E526574202B6D6D00B5
:102F7000486F70206D6D00486F70206D6D00486F58
:102F800070206D6D00486F70206D6D00486F70206F
:102F90006D6D005265747261637420205600526535
:102FA0007472616374202056005265747261637498
:102FB00020205600526574726163742020560052BE
:102FC00065747261637420205600537761702052DB
:102FD000652E6D6D00537761702052652E6D6D000A
:102FE000537761702052652E6D6D005377617020AC
:102FF00052652E6D6D00537761702052652E6D6D98
:103000000052657472616374206D6D005265747254
:10301000616374206D6D0052657472616374206D1C
:103020006D0052657472616374206D6D0052657439
:1030300072616374206D6D0053544F505045442E9F
:1030400020005041524144410041525245535441A5
:10305000544F200053544F505045442E2000535499
:103060004F505045442E20004B494C4C45442E2097
:103070000050415241444120444520454D4552476E
:103080002E0055434349534F20004B494C4C454477
:103090002E20004B494C4C45442E20004E6F206D95
:1030A0006F76652E0053696E206D6F76696D696568
:1030B0006E746F004E657373756E204D6F76696D1B
:1030C000656E746F004E6F206D6F76652E004E6FCB
:1030D000206D6F76652E004472756B2070727A6574
:1030E0007277616E79005072696E742061626F72DE
:1030F000746564005374616D70612061626F7274F5
:10310000697461005469736B2070726572757365C0
:103110006E005072696E742061626F727465640033
:10312000577A6E6F7769656E6965206472756B7525
:1031300000526573756D69656E646F20696D70729C
:10314000652E0052697072656E6469205374616DFA
:103150007061004F626E6F76656E69207469736B83
:103160007500526573756D696E67207072696E7453
:10317000005761697420666F7220757365722E2E18
:103180002E004573706572616E646F206F726465A6
:103190006E657300417474656E6469205574656E64
:1031A00074652E2E2E005761697420666F7220752B
:1031B0007365722E2E2E005761697420666F72201F
:1031C000757365722E2E2E00536C6565702E2E2E33
:1031D000005265706F736F2E2E2E00536F737065E3
:1031E0006E73696F6E652E2E2E00536C6565702EA2
:1031F0002E2E00536C6565702E2E2E004272616B70
:10320000206B61727479205344004E6F206861799D
:10321000207461726A657461205344004E6F2053BC
:1032200044204361727461005A61646E61205344AA
:10323000206B61727461004E6F2053442063617291
:1032400064004472756B207A205344004D656E759E
:10325000206465205344004D656E7520534420431F
:1032600061727461005469736B207A20534400507A
:1032700072696E742066726F6D205344005A6174D7
:10328000727A796D6163206472756B004465746550
:103290006E657220696D70726573696F6E00417240
:1032A0007265737461207374616D7061005A61732B
:1032B0007461766974207469736B0053746F702045
:1032C0007072696E74004B6F6E74796E756F776192
:1032D00063005265616E7564617220696D7072651C
:1032E000732E0052697072656E6469207374616D2B
:1032F000706100506F6B7261636F7661740052652C
:1033000073756D65207072696E740050727A6572A3
:10331000776163206472756B005061757361722010
:10332000696D70726573696F6E00506175736100CD
:10333000506F7A61737461766974207469736B007D
:103340005061757365207072696E74004E6173749C
:10335000726F696300416A757374617200416461E0
:10336000747461004C616469740054756E6500503A
:103370007269707261766100507265706172650089
:103380005072657061726500507269707261766129
:10339000005072657061726500496E666F726D6192
:1033A000636A65004D6F6E69746F72697A6172004D
:1033B00047756172646100496E666F726D61636525
:1033C00000496E666F2073637265656E004F626EB2
:1033D0006F7669740052656672657368005265663F
:1033E00072657368004F626E6F766974005265662D
:1033F00072657368004F626E6F76697420767963C8
:10340000686F7A6900526573746F726520666169CE
:103410006C7361666500526573746F7265206661D6
:10342000696C73616665004F626E6F7669742076B1
:103430007963686F7A6900526573746F726520668C
:1034400061696C7361666500556C6F7A6974207090
:10345000616D6574004C6F6164206D656D6F72798C
:10346000004C6F6164206D656D6F727900556C6FF3
:103470007A69742070616D6574004C6F6164206DB1
:10348000656D6F72790053746F7265206D656D6F35
:1034900072790053746F7265206D656D6F7279007B
:1034A00053746F7265206D656D6F72790053746F20
:1034B0007265206D656D6F72790053746F7265204F
:1034C0006D656D6F7279004C434420636F6E74724A
:1034D000617374004C434420636F6E747261737443
:1034E000004C434420636F6E7472617374004C43EC
:1034F0004420636F6E7472617374004C43442063A4
:103500006F6E74726173740046696C2E2044696139
:103510002E20330046696C2E204469612E20330032
:1035200046696C2E204469612E20330046696C2E5A
:10353000204469612E20330046696C2E2044696165
:103540002E20330046696C2E204469612E20320003
:1035500046696C2E204469612E20320046696C2E2B
:10356000204469612E20320046696C2E2044696136
:103570002E20320046696C2E204469612E203200D4
:1035800046696C2E204469612E20310046696C2EFC
:10359000204469612E20310046696C2E2044696107
:1035A0002E20310046696C2E204469612E203100A6
:1035B00046696C2E204469612E2031004520696ED9
:1035C000206D6D33004520696E206D6D3300452000
:1035D000696E206D6D33004520696E206D6D33007E
:1035E0004520696E206D6D330046696C616D656EB6
:1035F000740046696C616D656E740046696C616D3E
:10360000656E740046696C616D656E740046696C28
:10361000616D656E7400506F687962004D6F7469FA
:103620006F6E004D6F74696F6E00506F6879620045
:103630004D6F74696F6E0054656D7065726174755D
:1036400072610054656D70657261747572610054C9
:10365000656D7065726174757261005465706C6F30
:1036600074610054656D70657261747572650045B2
:1036700073746570732F6D6D004573746570732F6F
:103680006D6D004573746570732F6D6D00457374B7
:103690006570732F6D6D004573746570732F6D6D5C
:1036A000005A73746570732F6D6D005A7374657072
:1036B000732F6D6D005A73746570732F6D6D005AA2
:1036C00073746570732F6D6D005A73746570732F0A
:1036D0006D6D005973746570732F6D6D005973743F
:1036E0006570732F6D6D005973746570732F6D6DF8
:1036F000005973746570732F6D6D00597374657024
:10370000732F6D6D005873746570732F6D6D005855
:1037100073746570732F6D6D005873746570732FBB
:103720006D6D005873746570732F6D6D00587374F0
:103730006570732F6D6D00412D72657472616374D5
:1037400000412D7265747261637400412D7265745D
:103750007261637400412D7265747261637400411B
:103760002D7265747261637400416D61782000414F
:103770006D61782000416D61782000416D61782095
:1037800000416D617820005654726176206D696E3B
:10379000005654726176206D696E005654726176DF
:1037A000206D696E005654726176206D696E005608
:1037B00054726176206D696E00566D696E00566DAB
:1037C000696E00566D696E00566D696E00566D69C2
:1037D0006E00650065006500650065007A007A008E
:1037E0007A007A007A00790079007900790079000E
:1037F00078007800780078007800566D61782000B5
:10380000566D61782000566D61782000566D6178A4
:103810002000566D6178200056652D6A65726B0038
:1038200056652D6A65726B0056652D6A65726B0070
:1038300056652D6A65726B0056652D6A65726B0060
:10384000567A2D6A65726B00567A2D6A65726B0026
:10385000567A2D6A65726B00567A2D6A65726B0016
:10386000567A2D6A65726B005678792D6A65726B8F
:10387000005678792D6A65726B005678792D6A65E5
:10388000726B005678792D6A65726B005678792DC7
:103890006A65726B00416363656C00416363656CCC
:1038A00000416363656C00416363656C0041636361
:1038B000656C005049442D43005049442D4300504D
:1038C00049442D43005049442D43005049442D4361
:1038D000005049442D44005049442D44005049446F
:1038E0002D44005049442D44005049442D4400507B
:1038F00049442D49005049442D49005049442D491F
:10390000005049442D49005049442D490050494434
:103910002D50005049442D50005049442D50005026
:1039200049442D50005049442D50004F6666004FC9
:103930006666004F6666004F6666004F6666004F1B
:103940006E20004F6E20004F6E20004F6E20004F03
:103950006E20004175746F74656D70004175746FF1
:1039600074656D70004175746F74656D700041759C
:10397000746F74656D70004175746F74656D70005F
:1039800020022046616374002002204661637400B7
:1039900020022046616374002002204661637400A7
:1039A00020022046616374002002204D61780020CF
:1039B00002204D6178002002204D61780020022015
:1039C0004D6178002002204D6178002002204D6971
:1039D0006E002002204D696E002002204D696E00AD
:1039E0002002204D696E002002204D696E004B6F51
:1039F0006E74726F6C6100436F6E74726F6C004313
:103A00006F6E74726F6C004B6F6E74726F6C6100CE
:103A1000436F6E74726F6C00507275746F6B2032EE
:103A200000466C6F77203200466C6F772032005072
:103A30007275746F6B203200466C6F7720320050C5
:103A40007275746F6B203100466C6F7720310046C1
:103A50006C6F77203100507275746F6B20310046A7
:103A60006C6F77203100507275746F6B2030004698
:103A70006C6F77203000466C6F7720300050727585
:103A8000746F6B203000466C6F7720300050727A74
:103A900065706C797700466C756A6F00466C75735B
:103AA000736F00507275746F6B00466C6F770050C7
:103AB0007265646B6F73632077656E742E00566554
:103AC0006E74696C61646F720056656E746F6C61C0
:103AD00000527963686C6F73742076656E742E0083
:103AE00046616E2073706565640053746F6C696B1A
:103AF00000426173650050696174746F00426564CF
:103B00000042656400547279736B6133004E6F7AC2
:103B10007A6C6533004E6F7A7A6C65330054727933
:103B2000736B6133004E6F7A7A6C6533005472792F
:103B3000736B6132004E6F7A7A6C6532004E6F7A29
:103B40007A6C653200547279736B6132004E6F7A11
:103B50007A6C6532004479737A61004675736F72CE
:103B6000005567656C6C6F00547279736B61004E21
:103B70006F7A7A6C6500507265646B6F7363005680
:103B8000656C6F63696461640056656C636974C3D6
:103B9000A000527963686C6F73740053706565643C
:103BA00000506F73756E6F7574206F2031306D6DBE
:103BB000004D6F76652031306D6D004D6F7665205C
:103BC00031306D6D00506F73756E6F7574206F209E
:103BD00031306D6D004D6F76652031306D6D005068
:103BE0006F73756E6F7574206F20316D6D004D6F42
:103BF000766520316D6D004D6F766520316D6D00FD
:103C0000506F73756E6F7574206F20316D6D004D40
:103C10006F766520316D6D00506F73756E6F7574C2
:103C2000206F20302E316D6D004D6F766520302E67
:103C3000316D6D004D6F766520302E316D6D005009
:103C40006F73756E6F7574206F20302E316D6D003F
:103C50004D6F766520302E316D6D0045787472752C
:103C6000646572330045787472756465723300451B
:103C70007874727564657233004578747275646522
:103C800072330045787472756465723300457874D8
:103C9000727564657232004578747275646572324B
:103CA0000045787472756465723200457874727577
:103CB00064657232004578747275646572320045CD
:103CC00078747275646572004578747275736F727A
:103CD000004573747275736F726500457874727500
:103CE0006465720045787472756465720050727A0A
:103CF0006573756E6163205A004D6F766572205A48
:103D0000004D756F7669205A00506F73756E6F7530
:103D100074205A004D6F7665205A0050727A657390
:103D2000756E61632059004D6F7665722059004DA4
:103D3000756F7669205900506F73756E6F757420BA
:103D400059004D6F766520590050727A6573756E13
:103D500061632058004D6F7665722058004D756F75
:103D60007669205800506F73756E6F757420580017
:103D70004D6F76652058004D6F76657220656A65D7
:103D800073004D756F7669204173736500506F73D2
:103D9000756E6F7574206F7375004D6F7665206159
:103DA000786973005265747261637400526574724D
:103DB0006163740052657472616374005265747259
:103DC0006163740052657472616374004578747243
:103DD00075646F766174004578747275646500452A
:103DE000787472756465004578747275646F766175
:103DF000740045787472756465005A61706E6F75F1
:103E000074207A64726F6A005377697463682070F3
:103E10006F776572206F66660053776974636820F8
:103E2000706F776572206F6666005A61706E6F758D
:103E300074207A64726F6A005377697463682070C3
:103E40006F776572206F6666005679706E6F757455
:103E5000207A64726F6A0053776974636820706FA8
:103E6000776572206F6E0053776974636820706F96
:103E7000776572206F6E005679706E6F7574207A58
:103E800064726F6A0053776974636820706F776536
:103E900072206F6E00577963686C6F647A69630093
:103EA000456E66726961720052616666726564642D
:103EB00061005A63686C6164697400436F6F6C647D
:103EC0006F776E0050726564656872657620414256
:103ED0005320636F6E66005072656865617420419F
:103EE000425320636F6E660050726568656174208E
:103EF00041425320636F6E6600507265646568725C
:103F000065762041425320636F6E6600507265688B
:103F10006561742041425320636F6E660050726584
:103F200064656872657620414253204265640050A2
:103F30007265686561742041425320426564005097
:103F40007265686561742041425320426564005087
:103F500072656465687265762041425320426564EB
:103F60000050726568656174204142532042656467
:103F70000050726564656872657620414253204145
:103F80006C6C005072656865617420414253204139
:103F90006C6C005072656865617420414253204129
:103FA0006C6C00507265646568726576204142539E
:103FB00020416C6C00507265686561742041425309
:103FC00020416C6C005072656465687265762041B2
:103FD000425320330050726568656174204142533A
:103FE000203300507265686561742041425320336C
:103FF00000507265646568726576204142532033D3
:10400000005072656865617420414253203300504E
:1040100072656465687265762041425320320050B3
:1040200072656865617420414253203200507265A8
:1040300068656174204142532032005072656465A6
:10404000687265762041425320320050726568657F
:104050006174204142532032005072656465687279
:104060006576204142532031005072656865617465
:1040700020414253203100507265686561742041CF
:104080004253203100507265646568726576204144
:10409000425320310050726568656174204142537B
:1040A0002031005072656465687265762041425324
:1040B000005072656865617420414253005072651A
:1040C000686561742041425300507265646568728E
:1040D00065762041425300507265686561742041E5
:1040E00042530050726564656872657620504C4199
:1040F00020636F6E66005072656865617420504C75
:104100004120636F6E66005072656865617420506F
:104110004C4120636F6E660050726564656872651D
:104120007620504C4120636F6E6600507265686562
:10413000617420504C4120636F6E6600507265645C
:10414000656872657620504C41204265640050726B
:10415000656865617420504C41204265640050726E
:10416000656865617420504C41204265640050725E
:104170006564656872657620504C41204265640034
:104180005072656865617420504C4120426564003E
:1041900050726564656872657620504C4120416CB0
:1041A0006C005072656865617420504C4120416C10
:1041B0006C005072656865617420504C4120416C00
:1041C0006C0050726564656872657620504C4120C1
:1041D000416C6C005072656865617420504C4120E0
:1041E000416C6C0050726564656872657620504C55
:1041F000412033005072656865617420504C412045
:1042000033005072656865617420504C4120330062
:1042100050726564656872657620504C41203300A9
:104220005072656865617420504C412033005072B3
:104230006564656872657620504C4120320050728A
:10424000656865617420504C412032005072656889
:1042500065617420504C412032005072656465687D
:1042600072657620504C412032005072656865615D
:104270007420504C4120320050726564656872654C
:104280007620504C41203100507265686561742081
:10429000504C412031005072656865617420504C6B
:1042A0004120310050726564656872657620504C1B
:1042B000412031005072656865617420504C412086
:1042C000310050726564656872657620504C41001B
:1042D0005072656865617420504C41005072656889
:1042E00065617420504C4100507265646568726568
:1042F0007620504C41005072656865617420504CC6
:1043000041004E617374617620706F636174656BF8
:1043100000536574206F726967696E00536574207D
:104320006F726967696E004E617374617620706F99
:10433000636174656B00536574206F726967696EA1
:10434000004E617374617620706F636174656B20D9
:10435000686F6D650053657420686F6D65206F66CA
:1043600066736574730053657420686F6D65206FA4
:10437000666673657473004E617374617620706F46
:10438000636174656B20686F6D65005365742068A8
:104390006F6D65206F666673657473004175746F29
:1043A00020686F6D65004C6C6576617220616C20D1
:1043B0006F726967656E004175746F20486F6D6537
:1043C000004175746F20686F6D65004175746F20D2
:1043D000686F6D650057796C61637A7963207369E2
:1043E0006C6E696B6900417061676172206D6F74FA
:1043F0006F726573004469736162696C69746120EE
:104400004D6F746F7269005679706E6F7574206DA0
:104410006F746F72790044697361626C65207374A4
:10442000657070657273004175746F737461727436
:10443000004175746F7374617274004175746F73A9
:1044400074617274004175746F73746172740041A9
:1044500075746F7374617274004D656E7520676C4E
:104460006F776E65004D656E75207072696E636959
:1044700070616C004D656E75207072696E63697055
:10448000616C6500486C61766E69206E616269647A
:104490006B61004D61696E004B61727461207779C8
:1044A0006A657461005461726A6574612072657432
:1044B00069726164610053442043617264207269CF
:1044C0006D6F737361004B617274612076796A6DF0
:1044D00075746100436172642072656D6F76656406
:1044E000004B6172746120776C6F7A6F6E6100545B
:1044F00061726A65746120636F6C6F6361646100EF
:104500005344204361726420696E736572697461FB
:10451000004B6172746120766C6F7A656E61004346
:1045200061726420696E736572746564005072759F
:10453000736120693320676F746F77610050727503
:104540007361206933206C697374610050727573F4
:10455000612069332070726F6E746F2E0050727517
:1045600073612069332070726970726176656E6163
:104570000050727573612069332072656164792E11
:10458000004D383420582059205A2045004D3234EF
:10459000004D3233202573006175746F25692E67D5
:1045A000000A002F000A002E0044656C6574696FD4
:1045B0006E206661696C65642C2046696C653A20E2
:1045C0000046696C652064656C657465643A002E0C
:1045D000002E002E002E004E6F77206672657368E5
:1045E0002066696C653A20004E6F7720646F696EB3
:1045F000672066696C653A20002220706F73002284
:1046000020706172656E743A2200535542524F55C4
:1046100054494E452043414C4C2074617267657487
:104620003A2200747279696E6720746F2063616C3E
:104630006C207375622D67636F64652066696C65B5
:1046400073207769746820746F6F206D616E7920B4
:104650006C6576656C732E204D4158206C657665CF
:104660006C2069733A0000002110422063308440BE
:10467000A550C660E770088129914AA16BB18CC131
:10468000ADD1CEE1EFF13112100273325222B552A8
:104690009442F772D662399318837BB35AA3BDD381
:1046A0009CC3FFF3DEE36224433420040114E66478
:1046B000C774A44485546AA54BB528850995EEE5D1
:1046C000CFF5ACC58DD55336722611163006D77688
:1046D000F6669556B4465BB77AA719973887DFF721
:1046E000FEE79DD7BCC7C448E5588668A778400850
:1046F000611802282338CCC9EDD98EE9AFF9488971
:1047000069990AA92BB9F55AD44AB77A966A711AE7
:10471000500A333A122AFDDBDCCBBFFB9EEB799BC0
:10472000588B3BBB1AABA66C877CE44CC55C222C37
:10473000033C600C411CAEED8FFDECCDCDDD2AAD10
:104740000BBD688D499D977EB66ED55EF44E133EC7
:10475000322E511E700E9FFFBEEFDDDFFCCF1BBF60
:104760003AAF599F788F8891A981CAB1EBA10CD13A
:104770002DC14EF16FE18010A100C230E320045042
:10478000254046706760B9839893FBA3DAB33DC3B5
:104790001CD37FE35EF3B1029012F322D232354292
:1047A000145277625672EAB5CBA5A89589856EF545
:1047B0004FE52CD50DC5E234C324A01481046674E2
:1047C000476424540544DBA7FAB79987B8975FE795
:1047D0007EF71DC73CD7D326F2369106B016576632
:1047E0007676154634564CD96DC90EF92FE9C8991D
:1047F000E9898AB9ABA94458654806782768C01882
:10480000E1088238A3287DCB5CDB3FEB1EFBF98BF4
:10481000D89BBBAB9ABB754A545A376A167AF10AD1
:10482000D01AB32A923A2EFD0FED6CDD4DCDAABD04
:104830008BADE89DC98D267C076C645C454CA23C21
:10484000832CE01CC10C1FEF3EFF5DCF7CDF9BAFD4
:10485000BABFD98FF89F176E367E554E745E932E71
:10486000B23ED10EF01E22004D3232302053256967
:1048700000203A2000004C414E472053454C204632
:104880004F52434544002200205A3A0020593A0032
:1048900020453A00205A3A0020593A00583A002060
:1048A000002E0020423A0020453A00543A0020579A
:1048B0003A0020453A00543A002042403A00204055
:1048C0003A00202F003A00205400202F0020423AC6
:1048D00000202F006F6B20543A002569206D696E0F
:1048E0002C2025692073656300256920686F757227
:1048F00073202569206D696E75746573004D3131C3
:1049000030004D3239004D61722020382032303174
:104910003600436F6D70696C65643A2000286E6FD5
:104920006E652C2064656661756C7420636F6E66BD
:10493000696729004D6172202038203230313620DD
:1049400032303A35323A3531007374617274002274
:10495000002200FFFFFF0000A0400000A040000078
:10496000004000005643000046431FC54843000076
:104970000000000000001F856B3E00005643000051
:1049800046430000494300000000000000001F856E
:104990006B3E6563686F3A004572726F723A00470A
:1049A0003120453430204631303000473120453702
:1049B000302046343030004D383300473120452D0B
:1049C00038302046343030004D3833002D2D3A2D0C
:1049D0002D002D2D2D005344000120000120004DFD
:1049E00036303000464C4558202D20203233302FB1
:1049F00035300050502020202D20203235342F31EA
:104A000030300048495053202D20203232302F3191
:104A100030300050455420202D20203234302F39A2
:104A20003000504C4120202D20203231302F3530A5
:104A30000041425320202D20203235352F31303097
:104A4000004D3834004D383420582059205A204524
:104A5000004D3234004D3233202573005800590088
:104A60005A00457874727564657200473238004D9B
:104A7000383400473238205A0045334476366C6962
:104A800074650052414D426F31306100315F3735FE
:104A90006D6D002D2D2D2D2D2D2D2D2D2D2D2D0020
:104AA0004669726D77617265202D20322E322E3468
:104AB0000048617264636F64656420446566617573
:104AC0006C742053657474696E6773204C6F6164F5
:104AD00065640046696C616D656E742073657474FD
:104AE000696E67733A2044697361626C6564002083
:104AF00020204D32303020440046696C616D656E77
:104B0000742073657474696E67733A002020204DB9
:104B10003230392053004175746F2D5265747261C3
:104B200063743A20533D3020746F2064697361626E
:104B30006C652C203120746F20696E746572707200
:104B4000657420657874727564652D6F6E6C79205C
:104B50006D6F766573206173207265747261637422
:104B600073206F72207265636F766572696573007A
:104B70002046002020204D323038205300526563FB
:104B80006F7665723A20533D4578747261206C658A
:104B90006E67746820286D6D2920463A53706565EC
:104BA0006420286D6D2F6D2900205A0020460020BA
:104BB00020204D3230372053005265747261637487
:104BC0003A20533D4C656E67746820286D6D29202E
:104BD000463A537065656420286D6D2F6D29205A03
:104BE0003A205A4C69667420286D6D2900204400D3
:104BF0002049002020204D333031205000504944BE
:104C00002073657474696E67733A00205A002059E6
:104C10000020204D323036205800486F6D65206FDF
:104C2000666673657420286D6D293A002045002062
:104C30005A0020580020420020540020204D3230DD
:104C400035205300416476616E636564207661723D
:104C50006961626C65733A20533D4D696E206665EB
:104C600065647261746520286D6D2F73292C205442
:104C70003D4D696E2074726176656C206665656471
:104C80007261746520286D6D2F73292C20423D6D53
:104C9000696E696D756D207365676D656E742074DE
:104CA000696D6520286D73292C20583D6D617869E8
:104CB0006D756D205859206A65726B20286D6D2FB7
:104CC00073292C20205A3D6D6178696D756D205ACD
:104CD000206A65726B20286D6D2F73292C2020456A
:104CE0003D6D6178696D756D2045206A65726B2038
:104CF000286D6D2F73290020540020204D32303450
:104D0000205300416363656C65726174696F6E3A2C
:104D100020533D616363656C65726174696F6E2CCD
:104D200020543D7265747261637420616363656CC5
:104D300065726174696F6E00204500205A00205929
:104D40000020204D3230312058004D6178696D755A
:104D50006D20416363656C65726174696F6E2028B4
:104D60006D6D2F7332293A00204500205A002059DA
:104D70000020204D3230332058004D6178696D7528
:104D80006D2066656564726174657320286D6D2F92
:104D900073293A00204500205A0020590020204D58
:104DA0003932205800537465707320706572207515
:104DB0006E69743A0045303A20005A3A2000593A58
:104DC0002000583A20004D53312C4D533220506969
:104DD0006E730A005A00205A3A00590020593A00CE
:104DE000580020583A0024F4D43050C38E20C2A278
:104DF0004017828B7011127A910D816CD90AA861CB
:104E0000E108C7586607615143061E4B5D05C14561
:104E1000A7041A411104093D980371393103403642
:104E2000DB0265339102D4305402802E1D02632CC4
:104E3000EE01752AC501B028A001102781018F2538
:104E400064012B244B01E0223401AC211F018D2091
:104E50000D01801FFC00841EED00971DDF00B81CB3
:104E6000D200E61BC600201BBC00641AB200B219B7
:104E7000A8000A19A0006A189900D11791004017DC
:104E80008B00B516840031167E00B31579003A15F3
:104E90007300C7146F0058146A00EE13660088137D
:104EA000630025135E00C7125B006C1257001512D9
:104EB0005400C111510070114F0021114B00D61048
:104EC00049008D1047004610440002104200C00FF8
:104ED0004000800F3E00420F3C00060F3B00CB0E0F
:104EE0003800930E37005C0E3500270E3400F30DAA
:104EF0003200C10D3100900D3000600D2E00320DDA
:104F00002D00050D2C00D90C2B00AE0C2900850CB2
:104F100029005C0C2700350C27000E0C2600E80B3E
:104F20002400C40B2400A00B23007D0B23005A0B8C
:104F30002100390B2100180B2000F80A1F00D90AA4
:104F40001E00BB0A1E009D0A1D00800A1D00630A88
:104F50001C00470A1B002C0A1B00110A1A00F70943
:104F60001A00DD091900C4091900AB0919009209DA
:104F700017007B091800630917004C091600360951
:104F80001600200916000A091500F5081500E008AA
:104F90001400CC081400B8081400A40814009008E9
:104FA00013007D0812006B08130058081200460811
:104FB0001200340811002308110012081100010822
:104FC0001100F0071000E0071000D0071000C00724
:104FD0001000B0070F00A107100091070E00830713
:104FE0000F0074070F0065070E0057070E004907F2
:104FF0000E003B070D002E070E0020070D001307C3
:105000000D0006070D00F9060C00ED060D00E00688
:105010000C00D4060C00C8060C00BC060C00B00640
:105020000C00A4060B0099060C008D060B008206EE
:105030000B0077060B006C060B0061060A00570692
:105040000B004C060A0042060A0038060A002E062B
:105050000A0024060A001A060A00100609000706BC
:105060000A00FD050900F4050900EB050900E20549
:105070000900D9050900D0050900C7050900BE05CA
:105080000900B5050800AD050800A50509009C0547
:105090000800940508008C050800840508007C05BC
:1050A0000800740508006C050700650508005D052B
:1050B0000700560508004E05070047050700400594
:1050C000080038050700310507002A0507002305F9
:1050D00007001C050600160507000F050700080558
:1050E000060002050700FB040600F5040700EE04B5
:1050F0000600E8040600E2040700DB040600D5040D
:105100000600CF040600C9040600C3040600BD045F
:105110000600B7040600B1040500AC040600A604AE
:105120000600A00405009B040600950405009004F9
:1051300006008A04050085040500800406007A0440
:10514000050075040500700405006B040500660485
:105150000500610405005C040500570405005204C5
:1051600005004D04050048040500430405003E0405
:1051700004003A04050035040500300404002C0442
:10518000050027040400230405001E0404001A047B
:10519000040016040500110404000D0404000904B1
:1051A00005000404040000040400FC030400F803E8
:1051B0000400F4030400F0030400EC030400E8031B
:1051C0000400E4030400E0030400DC030400D8034B
:1051D0000400D4030400D0030400CC030400C8037B
:1051E0000300C503030024F404D9201BC40C5C0E87
:1051F0009804C4095F0265077101F405F900FB0416
:10520000B30048048700C103690058035500030335
:105210004500BE023A008402310053022A002902EE
:10522000250004022000E4011C00C8011900AF01A0
:10523000170098011400840113007101100061012E
:10524000100051010E0043010D0036010B002B012F
:105250000B0020010B00150109000C0109000301DE
:105260000800FB000800F3000800EB000700E40062
:105270000600DE000600D8000600D2000600CC00C2
:105280000500C7000500C2000500BD000400B9000C
:105290000400B5000400B1000400AD000400A90042
:1052A0000400A5000300A20003009F0004009B006F
:1052B0000300980003009500020093000300900093
:1052C00003008D0002008B000300880002008600AE
:1052D000020084000300810002007F0002007D00C4
:1052E00002007B00020079000200770001007600D6
:1052F00002007400020072000100710002006F00E1
:1053000002006D0001006C0002006A0001006900EB
:1053100002006700010066000100650001006400F2
:1053200002006200010061000100600001005F00F6
:1053300002005D0001005C0001005B0001005A00FA
:1053400001005900010058000100570001005600FB
:1053500001005500010054000100530000005300FB
:1053600001005200010051000100500001004F00F7
:1053700001004E0000004E0001004D0001004C00F5
:1053800001004B0000004B0001004A0001004900F1
:1053900001004800000048000100470001004600ED
:1053A00000004600010045000000450001004400E7
:1053B00001004300000043000100420000004200E1
:1053C00001004100000041000100400001003F00D9
:1053D00000003F0001003E0000003E0001003D00D3
:1053E00000003D0001003C0000003C0000003C00CB
:1053F00001003B0000003B0001003A0000003A00C1
:1054000001003900000039000100380000003800B8
:1054100000003800010037000000370001003600AE
:1054200000003600000036000100350000003500A5
:10543000000035000100340000003400000034009A
:10544000010033000000330000003300010032008F
:105450000000320000003200010031000000310085
:10546000000031000100300000003000000030007A
:1054700001002F0000002F0000002F0000002F006F
:1054800001002E0000002E0000002E0001002D0063
:1054900000002D0000002D0000002D0001002C0058
:1054A00000002C0000002C0000002C0001002B004C
:1054B00000002B0000002B0000002B0001002A0040
:1054C00000002A0000002A0000002A000100290034
:1054D0000000290000002900000029000000290028
:1054E000010028000000280000002800000028001B
:1054F000000028000100270000002700000027000E
:105500000000270000002700010026000000260000
:1055100000002600000026000000260001002500F3
:1055200000002500000025000000250000002500E7
:1055300000002500010024000000240000002400D9
:1055400000002400000024000100230000002300CC
:1055500000002300000023000000230000002300BF
:1055600000002300010022000000220000002200B1
:1055700000002200000022000000220001002100A3
:105580000000210000002100000021000000210097
:105590000000210000002100010020000000200088
:1055A000000020000000200000002000000020007B
:1055B000000020000000200001001F0000001F006C
:1055C00000001F0000001F0000001F0000001F005F
:1055D00000001F0001001E0000001E0000001E0051
:1055E00000001E0000000000090A02080B0C0D0755
:1055F000060304010000000000000000000000009D
:10560000000000000000000000000000000000009A
:10561000000011100F00000000000000000000005A
:10562000000000000000000000000000000000007A
:105630000000000000000000000000000102102037
:1056400020080810204010204080020102010804B8
:10565000020101020408102040808040201008044C
:1056600002018004020180402010080402010804A5
:1056700002010102040810204080010204081020E9
:105680004080100804088010204004408010204012
:10569000048005050505070508080808020202023E
:1056A0000A0A0808040404040101010101010101BE
:1056B0000303030303030303040707070C0C0C0C89
:1056C0000C0C0C0C02020202060606060606060672
:1056D0000B0B0B0B0B0B0B0B07070A0A0A0A0A0A28
:1056E0000505050404040808000020002300260026
:1056F00029002C002F0032000001000003010601E8
:10570000090100002200250028002B002E00310096
:10571000340002010000050108010B010000210016
:10572000240027002A002D00300033000101000072
:10573000040107010A01024E414E494E495459499C
:105740004E46CDCCCC3D0AD7233C17B7D13877CCC9
:105750002B329595E6241FB14F0A0000204100002E
:10576000C84200401C4620BCBE4CCA1B0E5AAEC5E7
:105770009D744C86BFA0FAD3508611241FBECFEF74
:10578000D1E2DEBFCDBF00E00CBF1DE0A0E0B2E083
:10579000EAEBFEEC01E00BBF02C007900D92A833CC
:1057A000B107D9F72CE1A8E3BDE001C01D92AD34EB
:1057B000B207E1F717E5C8E7D7E500E006C0229792
:1057C0000109FE010BBF0E94E5E0C237D10780E06E
:1057D0000807A9F70E94FED70C944CE70C94000030
:1057E000CF93DF93EC019C012C5F3F4F41E050E0F1
:1057F00060E070E0898D9A8D0E949236882399F03E
:105800004D895E896F89788D452B462B472B59F43E
:105810004C815D816E817F814D8B5E8B6F8B788F2C
:10582000998190689983DF91CF910895CF92DF920B
:10583000EF92FF920F931F93CF93DF93EC0189892F
:105840009A89AB89BC89803E9F4FAF41B10510F06A
:1058500080E06BC0CE01C4DF8823D1F30E94A63460
:10586000182F8823A9F3E98DFA8DCC80DD80EE8096
:10587000FF8032E0C31AD108E108F108058404C0B2
:10588000CC0CDD1CEE1CFF1C0A94D2F78685978594
:10589000A089B189C80ED91EEA1EFB1E81E0809343
:1058A0003E0DC092410FD092420FE092430FF09212
:1058B000440F80E092E0E1E4FDE0DF019C011D92F5
:1058C00021503040E1F701E0E98DFA8D848108171D
:1058D00090F421E43DE0B701A601400F511D611D88
:1058E000711D80913F0D9091400D0E94615A882357
:1058F000E1F00F5FE9CFC12C82E0D82EE12CF12C32
:10590000058404C0CC0CDD1CEE1CFF1C0A94D2F7ED
:1059100049895A896B897C894C0D5D1D6E1D7F1DDF
:10592000498B5A8B6B8B7C8B812FDF91CF911F9191
:105930000F91FF90EF90DF90CF900895CF93DF937A
:10594000EC0141E0611101C040E06C857D858E85F0
:105950009F850E94E634882341F0888920E2829F57
:10596000C00111248F5B924F02C080E090E0DF9174
:10597000CF91089530E020E04EE2DC015C9150329E
:1059800071F0383029F4FB01E20FF11D40832F5FE5
:10599000FB01E20FF11DDC015C9150832F5F3F5F43
:1059A00001963B3051F7FB01E20FF11D1082089583
:1059B000CF93DF93EB01FC012381211102C080E032
:1059C0000EC02250223020F48FE28883198206C054
:1059D00060E0B4DF009799F3BE01CCDF81E0DF9196
:1059E000CF910895FB012BE030E231932150E9F78C
:1059F000DC0190E027E03A2FEB2F8D9181110AC056
:105A0000DA013C931196EC9381E0FB019081903296
:105A100039F525C08F32A1F38E3219F0EAE8F1E0B2
:105A200008C02A30E1F098E02AE0E5CF3196381737
:105A3000B1F034913111FACF291788F03FED380FCA
:105A40003E3568F431E0390FFB01E90FF11D9FE9A4
:105A5000980F9A3108F480528083932FCCCF80E046
:105A600008950F931F93CF93DF93EC018B018B81EC
:105A7000882311F080E042C0FB018789803139F131
:105A80008032C1F783E08B83F801428D538D648DA2
:105A9000758D4D8B5E8B6F8B788F9E012F5E3F4F88
:105AA000C8010E949D35882329F31A8F098F81E050
:105AB00089831C821D821E821F82188619861A867F
:105AC0001B861C861D861E861F86188A17C082E0CC
:105AD0008B831D8A1E8A1F8A188EFB01408D518D73
:105AE00060E070E095E0440F551F661F771F9A95A0
:105AF000D1F7498B5A8B6B8B7C8BD7CFDF91CF91B2
:105B00001F910F9108952F923F924F925F926F9243
:105B10007F928F929F92AF92BF92CF92DF92EF923D
:105B2000FF920F931F93CF93DF93EC015B016A0108
:105B30008B81811103C08FEF9FEFC7C0898180FFE8
:105B4000FACF49895A896B897C8988859985AA8584
:105B5000BB852601612C712C8A019B01081B190B46
:105B60002A0B3B0B401651066206730618F06A01B9
:105B7000C81AD90A76013E0124E0620E711CE114B4
:105B8000F10409F476C0488559856A857B854A0108
:105B900081E098222B811A012B01E9E05694479469
:105BA00037942794EA95D1F7898D9A8DFC0122309C
:105BB00049F4628D738D848D958D620D731D841DE6
:105BC000951D3CC014811150122181149104C1F41F
:105BD000111116C0452B462B472B49F48D899E8900
:105BE000AF89B88D8C839D83AE83BF8309C04C8100
:105BF0005D816E817F81930121D7882309F49BCF3A
:105C0000E98DFA8D6C817D818E819F816250710951
:105C100081099109058404C0660F771F881F991FA9
:105C20000A94D2F72685378540895189620F731F00
:105C3000841F951F610F711D811D911D20E032E0B1
:105C40002819390987012E153F0508F48901011526
:105C5000F2E01F0769F52091410F3091420F40910A
:105C6000430F5091440F621773078407950719F487
:105C70001FC0C6012AC09501AB01BC0180913F0D38
:105C80009091400D0E94EC59882309F454CFA00E46
:105C9000B11E88859985AA85BB85800F911FA11D9E
:105CA000B11D88879987AA87BB87E01AF10A67CF59
:105CB00040E08CD6882309F43ECFB4016F5B724F6D
:105CC000A801C5010E940BE4E2CFDF91CF911F91A3
:105CD0000F91FF90EF90DF90CF90BF90AF909F908B
:105CE0008F907F906F905F904F903F902F9008958E
:105CF000CF93DF931F92CDB7DEB741E050E0BE01F6
:105D00006F5F7F4F00DF019719F4898190E002C037
:105D10008FEF9FEF0F90DF91CF910895CF92DF9299
:105D2000EF92FF920F931F93CF93DF936C01EB01E0
:105D30007A01FC018381823060F000851185228523
:105D400033850F71112722273327012B022B032BB9
:105D500011F08FEF5CC04115510511F0F701108271
:105D60001DE040E250E0BE01C601CDDE803291056B
:105D700039F021E0892B09F420E0822F819547C07A
:105D800028812223C1F0253E61F32E3251F33B8559
:105D90003F733F3061F4E114F10449F04A8D5B8DAB
:105DA000452B29F42F713FEF320F343030F02B8523
:105DB00023FDD7CF2CC080E02AC030E0215031092C
:105DC000129FC001139F900D1124F701E80FF91FD6
:105DD000298120832B8121832D8122832F8123837D
:105DE000298524832E852583288926832A8927834C
:105DF0002C8920872E892187288D22872C8D238727
:105E00002E8D2487288126FFD2CF1586D0CFDF9113
:105E1000CF911F910F91FF90EF90DF90CF90089559
:105E20001F93CF93DF93EC018B81823018F480E0D5
:105E300090E023C0488559856A857B85A5E07695E5
:105E4000679557954795AA95D1F7142F1F70CE01E6
:105E50004FDF97FDECCF488559856A857B85415E8C
:105E60005F4F6F4F7F4F488759876A877B8720E254
:105E7000129FC00111248F5B924FDF91CF911F9130
:105E800008954F925F926F927F92AF92BF92CF929E
:105E9000DF92EF92FF920F931F93CF93DF93EC016A
:105EA0006A017B012B81222349F089899A89AB8978
:105EB000BC8984179507A607B70710F480E06BC06C
:105EC000223009F463C0C114D104E104F10449F49F
:105ED0001C821D821E821F82188619861A861B86C6
:105EE00059C088859985AA85BB85E98DFA8DE58598
:105EF000F0E03996AC01BD014150510961097109C9
:105F00000E2E04C076956795579547950A94D2F75B
:105F100097018601015011092109310904C0369504
:105F2000279517950795EA95D2F7041715072607C1
:105F3000370720F0892B8A2B8B2B49F48D899E897A
:105F4000AF89B88D8C839D83AE83BF8304C0041B4F
:105F5000150B260B370B280139015E0184E0A80ED2
:105F6000B11C411451046104710481F04C815D81C4
:105F70006E817F819501898D9A8D60D591E0491A56
:105F80005108610871088111ECCF05C0C886D98617
:105F9000EA86FB8681E0DF91CF911F910F91FF9000
:105FA000EF90DF90CF90BF90AF907F906F905F9019
:105FB0004F9008950F931F93CF93DF93EC018B8144
:105FC0008823D1F1898187FF32C061E0CE01B6DC40
:105FD0008C01009789F1FC018081853E69F18B81FC
:105FE000823040F449895A896B897C89448F558F66
:105FF000668F778F4D895E896F89788DF801538F11
:10600000428F758B648BE091380DF091390D30978C
:1060100059F0B8016A5E7F4FC80148961995F8019A
:10602000808D918D938B828B89818F778983DF918E
:10603000CF911F910F918AC481E0888380E0DF9126
:10604000CF911F910F910895CF93DF93EC01B2DFB1
:106050001B82DF91CF910895FC0123812111F4CFA0
:1060600008954F925F926F927F92AF92BF92CF92BC
:10607000DF92EF92FF920F931F93CF93DF9300D0A5
:106080001F92CDB7DEB75C016A017B01FC01838101
:106090008130E9F4818181FF1AC0F50181899289FB
:1060A000A389B48984179507A607B70780F0892BC1
:1060B0008A2B8B2B09F472C0F501408451846284D1
:1060C0007384B701A601C501DCDE811102C080E046
:1060D00066C0F501818D928DC114D104E104F104F3
:1060E00069F4458956896789708D25D7882379F3A6
:1060F000F501158A168A178A108E37C0F50144817A
:106100005581668177819E012F5F3F4F97D4882309
:10611000F1F249815A816B817C81F501818D928DEB
:10612000FC012789203139F4483FFFEF5F07610503
:106130007105D8F407C0483F2FEF520762072FE0E0
:10614000720798F4F8D6882309F4C1CFF501448189
:106150005581668177810FEF1FEF2FEF3FE0818D33
:10616000928D51D5882309F4B2CFF501C18AD28A24
:10617000E38AF48A818180688183C5011BDF8823DB
:1061800009F4A5CFB701A6014C145D046E047F0489
:1061900010F4B301A201C50174DE01C081E00F90CB
:1061A0000F900F900F90DF91CF911F910F91FF9063
:1061B000EF90DF90CF90BF90AF907F906F905F9007
:1061C0004F900895FF920F931F93CF93DF93EC01AD
:1061D000F42E80E2689FF0011124EF5BF24F83857B
:1061E000817121F0842F827109F04EC08091410F9E
:1061F0009091420FA091430FB091440F8C879D87DF
:10620000AE87BF87688B4489558960E070E0BA012A
:1062100055274427028D138D20E030E0402B512B71
:10622000622B732B4D8B5E8B6F8B788F8385887180
:1062300051F4048D158D268D378D098B1A8B2B8B80
:106240003C8B81E00BC08031F9F49E012F5E3F4F03
:10625000898D9A8D72D48823B9F084E08B838F2D39
:106260008F7089831C821D821E821F821886198668
:106270001A861B86F4FE0BC040E050E0BA01CE0146
:10628000F0DE811104C011C01B8280E00EC0F5FE5B
:106290000BC049895A896B897C89CE01DF91CF91E6
:1062A0001F910F91FF90EDCD81E0DF91CF911F9174
:1062B0000F91FF900895AF92BF92CF92DF92EF922D
:1062C000FF920F931F93CF93DF937C01EB016A0141
:1062D000B22E898D9A8DF701928F818F40E050E028
:1062E000BA01CE01CEDDA12C088519852A853B8512
:1062F00089899A89AB89BC89081719072A073B073E
:10630000A0F585E036952795179507958A95D1F7DD
:106310000F70CE0185DD009709F481C0FC0120815A
:10632000222311F0253EB9F4A1100EC04091410F77
:106330005091420F6091430F7091440FF7014487D1
:10634000558766877787008BFC018081AA24A394F8
:106350008111CACF0AC04BE050E0BC01C6010E94C7
:10636000FEE3892B09F0C0CF58C08B2D8274823494
:1063700009F055C0AA2049F0F701008961E0C70182
:10638000DDDAEC01009769F44AC08B81823009F4B0
:1063900046C0CE014BDA882309F441C0C1E4DDE0F8
:1063A00000E080E2FE0111928A95E9F78BE0F601A8
:1063B000DE0101900D928A95E1F7E091380DF091A0
:1063C000390D309739F0BE01625F7F4FCE014096A4
:1063D000199508C081E298E2998B888B80E098E05B
:1063E0009F878E87888999899B8B8A8B998F888FC5
:1063F0008E859F859F8B8E8BA9D2882381F04B2D14
:10640000602FC701DF91CF911F910F91FF90EF9007
:10641000DF90CF90BF90AF90D5CEB7FEF0CF80E0A9
:10642000DF91CF911F910F91FF90EF90DF90CF9070
:10643000BF90AF9008953F924F925F926F927F927C
:106440008F929F92AF92BF92CF92DF92EF92FF9284
:106450000F931F93CF93DF93CDB7DEB7C354D1090A
:106460000FB6F894DEBF0FBECDBF5C016B01249662
:106470005FAF4EAF2497522E1C8E1F8E19821C8246
:106480006115710511F410E073C0FC018381811165
:10649000FACF2496EEADFFAD249780818F3211F0B4
:1064A00076011DC02496EEADFFAD249780818F321A
:1064B00031F431962496FFAFEEAF2497F3CFF60177
:1064C00083818250823060F3F601618D728DCE013E
:1064D0000196C7DA8823B9F2CE0101967C018E01BC
:1064E000045E1F4F3801FE0131964F01402E312EC0
:1064F00019C08823A9F121E0AE01495C5F4FB701C3
:10650000C801D9DE882309F4BECFEC14FD0411F0D4
:10651000C7019ADD0615170501F1942D832D780129
:10652000092F182FAE014E5B5F4FBE01695C7F4F94
:1065300024968EAD9FAD249755DA882309F4A3CF16
:106540002496EEADFFAD249780818F3291F631967F
:106550002496FFAFEEAF2497F3CF982D892DDFCF90
:10656000252DAE01495C5F4FB701C501A4DE182F90
:10657000CE01019671DDCE014C966EDD812FCD5B93
:10658000DF4F0FB6F894DEBF0FBECDBFDF91CF91C6
:106590001F910F91FF90EF90DF90CF90BF90AF9041
:1065A0009F908F907F906F905F904F903F90089555
:1065B000CF93DF93EC0140E050E0BA0152DD882335
:1065C00061F061E0CE01BAD9009739F025EEFC0107
:1065D00020831B82DF91CF91B9C180E0DF91CF9101
:1065E00008951F93CF93DF93CDB7DEB76B970FB6A8
:1065F000F894DEBF0FBECDBFAB0119821C8222E032
:10660000BC01CE01019617DF182F882321F0CE019F
:106610000196CEDF182FCE0101961EDD812F6B96DD
:106620000FB6F894DEBF0FBECDBFDF91CF911F91A3
:1066300008952F923F924F925F926F927F928F9226
:106640009F92AF92BF92CF92DF92EF92FF920F9301
:106650001F93CF93DF9300D01F921F92CDB7DEB769
:106660008C015B013A01DC0113968C911397813008
:10667000C1F411968C9181FF14C082FF18C0F801FB
:10668000418952896389748980859185A285B38502
:1066900084179507A607B70751F0C801F2DB8111EF
:1066A00006C081E0F80180838FEF9FEF37C163015F
:1066B00083C0D80159968D919C915A97FC01F48121
:1066C000F1501A012B0169E05694479437942794AE
:1066D0006A95D1F7F221FD834A0121E09222FF233E
:1066E00009F476C080E092E08819990976018C154A
:1066F0009D0508F47C01D8015996ED91FC915A97BB
:1067000014962D903D904D905C901797B2E02B1A07
:10671000310841085108058404C0220C331C441C74
:10672000551C0A94D2F786859785A089B189280ED1
:10673000391E4A1E5B1EED812E0E311C411C511C60
:10674000E114F2E0FF0609F089C08091410F9091B9
:10675000420FA091430FB091440F82159305A405F9
:10676000B50569F410923E0D8FEF9FEFDC01809329
:10677000410F9093420FA093430FB093440F9501A4
:10678000B201A10180913F0D9091400D0E94615A8C
:10679000882309F486CFF80180859185A285B38589
:1067A0008E0D9F1DA11DB11D80879187A287B38784
:1067B000AE0CBF1CCE18DF08D80118964D915D9124
:1067C0006D917C911B97C114D10409F072CF7AC0EE
:1067D0008114910409F086CF14964D915D916D91CD
:1067E0007C911797411551056105710559F455962E
:1067F0008D919D910D90BC91A02D0097A105B105A3
:1068000039F520C09E012F5F3F4F18D1882309F42E
:1068100048CF89819A81AB81BC81F801218D328D6D
:10682000F9012789203139F4883FFFEF9F07A1053F
:10683000B10540F40DC0883F2FEF9207A2072FE06B
:10684000B20730F0C8010E94F02B81114BCF29CF45
:10685000F80184839583A683B78344CF8114910480
:1068600011F5D80118964D915D916D917C911B9712
:1068700051968D919D910D90BC91A02D481759076F
:106880006A077B0780F062D0882309F40ACF81E091
:1068900080933E0D2092410F3092420F4092430F61
:1068A0005092440F07C041E0C201B1018FD088234C
:1068B00009F4F7CEA701B501C4018F5B924F0E9486
:1068C0000BE469CF51968D919D910D90BC91A02DB7
:1068D000F801218184179507A607B70738F4418B83
:1068E000528B638B748B206821830CC08091380D90
:1068F0009091390D892B31F06114710419F02068E1
:10690000F8012183D80111968C9183FD02C0C30147
:1069100005C0C8014FDB8111FACFC3CE0F900F9095
:106920000F900F900F90DF91CF911F910F91FF90DB
:10693000EF90DF90CF90BF90AF909F908F907F901F
:106940006F905F904F903F902F900895CF938091DC
:106950003E0D8823B9F14091410F5091420F609153
:10696000430F7091440F21E43DE080913F0D9091E1
:10697000400D0E94615AC82F811102C0C0E023C09F
:1069800040913A0D50913B0D60913C0D70913D0D41
:10699000411551056105710591F021E43DE08091BB
:1069A0003F0D9091400D0E94615A882339F3109257
:1069B0003A0D10923B0D10923C0D10923D0D10922D
:1069C0003E0D01C0C1E08C2FCF910895CF92DF9290
:1069D000EF92FF92CF936B017C01C42F8091410F06
:1069E0009091420FA091430FB091440F8C159D05DB
:1069F000AE05BF05C9F0AADF811102C080E018C052
:106A000021E43DE0B701A60180913F0D9091400D3A
:106A10000E94EC59882391F3C092410FD092420F0B
:106A2000E092430FF092440F81E0C11180933E0D3C
:106A3000CF91FF90EF90DF90CF9008958F929F922B
:106A4000AF92BF92CF92DF92EF92FF920F931F937C
:106A5000CF93DF93EC016A017B01890189859A85D7
:106A6000AB85BC850196A11DB11D84179507A607AE
:106A7000B70710F480E054C08F89803129F499273A
:106A8000872F762F652F0BC08032A1F7CB01BA017B
:106A900027E096958795779567952A95D1F78B8806
:106AA0009C88AD88BE88680D791D8A1D9B1D8090CD
:106AB000410F9090420FA090430FB090440F681583
:106AC00079058A059B0581F48F89803191F4DD2455
:106AD000EE24FF24F601EE0FFF1FEF5BF24F8081E3
:106AE0009181A0E0B0E016C040E070DF8111ECCFF2
:106AF000C1CFE894C7F8DD24EE24FF24F601EE0FA1
:106B0000FF1FEE0FFF1FEF5BF24F80819181A2818B
:106B1000B381BF70F80180839183A283B38381E046
:106B2000DF91CF911F910F91FF90EF90DF90CF9069
:106B3000BF90AF909F908F9008954F925F926F9209
:106B40007F92AF92BF92CF92DF92EF92FF920F931C
:106B50001F93CF93DF9300D01F92CDB7DEB78C0188
:106B600049835A836B837C835901C12CD12C7601D4
:106B7000412C42E0542E612C712C49815A816B8149
:106B80007C819E012F5F3F4FC80158DF882341F170
:106B9000D301C201F801058404C0880F991FAA1F00
:106BA000BB1F0A94D2F7C80ED91EEA1EFB1E4981EC
:106BB0005A816B817C818789803139F481E0483F3B
:106BC0005F4F6105710538F4D8CF81E0483F5F4FD2
:106BD0006F4F7F4090F2F501C082D182E282F38252
:106BE0000F900F900F900F90DF91CF911F910F9109
:106BF000FF90EF90DF90CF90BF90AF907F906F901D
:106C00005F904F9008954F925F926F927F928F9214
:106C10009F92AF92BF92CF92DF92EF92FF920F932B
:106C20001F93CF93DF93EC014A015B0128013901E7
:106C3000423051056105710508F462C049855A85E5
:106C40006B857C854F5F5F4F6F4F7F4F48155905B0
:106C50006A057B0508F454C08F89803129F4FF242C
:106C6000EB2CDA2CC92C0CC0803209F049C075011C
:106C7000640177E0F694E794D794C7947A95D1F7B6
:106C80004B895C896D897E89C40ED51EE61EF71E70
:106C900041E0C701B6019ADE882391F19F899031C6
:106CA00059F49924AA24BB24F401EE0FFF1FEF5BD3
:106CB000F24F5182408210C0E89487F89924AA24A8
:106CC000BB24F401EE0FFF1FEE0FFF1FEF5BF24F2F
:106CD00040825182628273829A89923090F04D8113
:106CE0005E816F8178854C0D5D1D6E1D7F1D40930B
:106CF0003A0D50933B0D60933C0D70933D0D01C0D8
:106D000080E0DF91CF911F910F91FF90EF90DF9086
:106D1000CF90BF90AF909F908F907F906F905F903B
:106D20004F9008952F923F924F925F926F927F9271
:106D30008F929F92AF92BF92CF92DF92EF92FF928B
:106D40000F931F93CF93DF93CDB7DEB72F970FB677
:106D5000F894DEBF0FBECDBF1C014C875D876E87E8
:106D60007F873B872A87DC0119960D911D912D9114
:106D70003C911C970F5F1F4F2F4F3F4F0D831E837A
:106D80002F833887EA85FB8580809180A280B3803D
:106D900081149104A104B10431F0FFEF8F1A9F0A0E
:106DA000AF0ABF0A10C0DC018D909D90AD90BC90E1
:106DB000B1E0B9870C851D852E853F850130110511
:106DC0002105310509F0198675016401412C512C0A
:106DD0003201F10181859285A385B4854816590653
:106DE0006A067B0608F04EC00D811E812F81388512
:106DF0000C151D052E053F0550F4F2E0CF2ED12CC9
:106E0000E12CF12CA2E08A2E912CA12CB12C9E0118
:106E10002F5F3F4FB701A601C10110DE882391F11A
:106E200049815A816B817C81D701C6010196A11DE0
:106E3000B11D452B462B472B19F04C015D010FC0AE
:106E4000AC01BD01481959096A097B090C851D85EA
:106E50002E853F85401751076207730741F01FEFEA
:106E6000411A510A610A710A6C017D01B2CF0FEF1C
:106E70001FEF2FEF3FE0B701A601C101C4DE8D83F4
:106E8000811113C01D823DC02601370121E0421A45
:106E900051086108710897018601B301A201C1017F
:106EA000B2DE882379F3730162018C149D04AE0471
:106EB000BF0450F3AA85BB854D915D916D917C9186
:106EC0004115510561057105A9F4EA85FB858082AC
:106ED0009182A282B382F985FF2399F00FEF801A85
:106EE000900AA00AB00AD1018D929D92AD92BC92F7
:106EF000139707C095018401C10185DE8111E5CF9B
:106F0000C1CF8D812F960FB6F894DEBF0FBECDBFD7
:106F1000DF91CF911F910F91FF90EF90DF90CF9075
:106F2000BF90AF909F908F907F906F905F904F90A9
:106F30003F902F900895AF92BF92CF92DF92EF9241
:106F4000FF920F931F93CF93DF9300D01F92CDB783
:106F5000DEB75C016A017B0182E090E0A0E0B0E076
:106F6000F50180839183A283B3839E012F5F3F4FFE
:106F7000B701A601C50162DD811102C080E023C016
:106F800000E010E09801B701A601C5013CDE8823AE
:106F9000A9F3C980DA80EB80FC80F5018789803114
:106FA00049F481E0F8EFCF16FFEFDF06E104F104CA
:106FB00050F4DBCF81E098EFC9169FEFD906E906C0
:106FC0009FE0F90690F20F900F900F900F90DF91D5
:106FD000CF911F910F91FF90EF90DF90CF90BF90D6
:106FE000AF9008957F928F929F92AF92BF92CF926F
:106FF000DF92EF92FF920F931F93CF93DF93EC01F9
:10700000142F7093400D60933F0D1F8A82E090E033
:10701000A0E0B0E088839983AA83BB8310923E0DE1
:1070200010923A0D10923B0D10923C0D10923D0DB6
:107030008FEF9FEFDC018093410F9093420FA0935D
:10704000430FB093440F442349F1453008F0DEC0AC
:1070500040E060E070E0CB01B9DC882309F4D6C0E1
:1070600020E1129FF0011124E151F14F80818F77CF
:1070700009F0CCC084859585A685B78584369105B1
:10708000A105B10508F4C2C0C084D184E284F384B0
:10709000C114D104E104F10421F4B8C0C12CD12CF5
:1070A000760140E0C701B60191DC782E882309F40F
:1070B000ADC080914C0D90914D0D8115924009F01D
:1070C000A5C03091510D332309F4A0C080914F0D1C
:1070D0009091500D892B09F499C020914E0D2223D7
:1070E00009F494C03A8B2C831D8630E041E050E0D7
:1070F0006D85062FCA01062E02C0880F991F0A94BB
:10710000E2F72817390731F081E0860F8D87683064
:1071100078F37CC02091570D3091580D2115310521
:1071200019F040E050E008C02091650D3091660DE7
:107130004091670D5091680D2D833E834F83588792
:1071400080914F0D9091500D46015701880E991E68
:10715000A11CB11C8B8A9C8AAD8ABE8AE091520D1B
:10716000F091530DF98FE88FA091510DB0E00E947E
:10717000D5E0680D791D8A1D9B1D6A8F7B8F8C8FD2
:107180009D8FB5E0EE0FFF1FBA95E1F7E150FE4F7E
:10719000EF2FFF27E695DC01CB018E0F9F1FA11D6E
:1071A000B11D8E879F87A88BB98B8090540D9090CE
:1071B000550D8114910419F0A12CB12C08C08090B8
:1071C000610D9090620DA090630DB090640DA701C9
:1071D0009601281B390B4A0B5B0BDA01C901880D9C
:1071E000991DAA1DBB1D04C0B695A79597958795B7
:1071F0000A95D2F789879A87AB87BC87853F3FE09E
:107200009307A105B10520F48CE08F8B712C15C07C
:10721000853F9F4FA105B10510F480E10DC080911D
:107220006D0D90916E0DA0916F0DB091700D8A8FC4
:107230009B8FAC8FBD8F80E28F8B872DDF91CF919D
:107240001F910F91FF90EF90DF90CF90BF90AF9084
:107250009F908F907F9008954F925F926F927F9250
:107260008F929F92AF92BF92CF92DF92EF92FF9256
:107270000F931F93CF93DF932C0124EF33E081E032
:1072800090E0F90145915491441655060CF062C006
:10729000AC0141505109DA01AA0FBB1FAA0FBB1F55
:1072A000AE50BC4FFD0165917491440F551F440FC2
:1072B000551F40515C4FFA0165907490FC01EE0F30
:1072C000FF1FEE0FFF1FEE50FC4FA590B490FD0185
:1072D00005911491F901C591D491FA01859094908A
:1072E000882777FD8095982F0E944FDD6B017C01E8
:1072F000B20166197709882777FD8095982F0E943B
:107300004FDD2B013C01B501601B710B882777FD18
:107310008095982F0E944FDD9B01AC01C301B20103
:107320000E9482DF2B013C01BE0168197909882780
:1073300077FD8095982F0E944FDD9B01AC01C30122
:10734000B2010E94B4DC9B01AC01C701B6010E94EE
:10735000D4DB11C001962C5F3F4F8D33910509F0AE
:1073600090CFE2EEF4E065917491882777FD8095E7
:10737000982F0E944FDDDF91CF911F910F91FF90C9
:10738000EF90DF90CF90BF90AF909F908F907F90C5
:107390006F905F904F9008954F925F926F927F929F
:1073A0008F929F92AF92BF92CF92DF92EF92FF9215
:1073B0000F931F93CF93DF932C01662371F1E8E9BC
:1073C000F9E48491882341F09091C00095FFFCCFAF
:1073D0008093C6003196F5CF70E04AE050E08BE232
:1073E00095E10E9482B7E9E5F2E08491882341F0BB
:1073F0009091C00095FFFCCF8093C6003196F5CFE9
:107400008091C00085FFFCCF8AE08093C6000E9477
:10741000536460E070E0CB017EC024E733E081E09C
:1074200090E0F90145915491441655060CF062C064
:10743000AC0141505109DA01AA0FBB1FAA0FBB1FB3
:10744000AE58BC4FFD0165917491440F551F440F18
:10745000551F40595C4FFA0165907490FC01EE0F86
:10746000FF1FEE0FFF1FEE58FC4FA590B490FD01DB
:1074700005911491F901C591D491FA0185909490E8
:10748000882777FD8095982F0E944FDD6B017C0146
:10749000B20166197709882777FD8095982F0E9499
:1074A0004FDD2B013C01B501601B710B882777FD77
:1074B0008095982F0E944FDD9B01AC01C301B20162
:1074C0000E9482DF2B013C01BE01681979098827DF
:1074D00077FD8095982F0E944FDD9B01AC01C30181
:1074E000B2010E94B4DC9B01AC01C701B6010E944D
:1074F000D4DB11C001962C5F3F4F8032910509F01B
:1075000090CFEEEEF3E065917491882777FD80953A
:10751000982F0E944FDDDF91CF911F910F91FF9027
:10752000EF90DF90CF90BF90AF909F908F907F9023
:107530006F905F904F90089560E080919A0F9091C6
:107540009B0F2ADF6093960F7093970F8093980F8D
:107550009093990F8091940F9091950F7DDE609399
:10756000900F7093910F8093920F9093930F8FB71A
:10757000F8941092880F8FBF0895209114023091D3
:107580001502409116025091170260E070E08FE7FB
:1075900093E40E94B4DC6093680F7093690F80934A
:1075A0006A0F90936B0F089597FF03C080918F0F20
:1075B00004C0FC01EE59F04F808190E00895CF9314
:1075C000DF93D82FC62FC19561E00E945ED66C2F45
:1075D0008D2F0E9497D66C2F70E08D2FDF91CF9169
:1075E0000C9454D5CF93C1E020E030E048E452E45D
:1075F0006091960F7091970F8091980F9091990FCD
:107600000E94B0DE18160CF0C0E06C2F88E090E00D
:10761000CF91D5CF2F923F924F925F926F927F92F0
:107620008F929F92AF92BF92CF92DF92EF92FF9292
:107630000F931F93CF93DF93CDB7DEB728970FB685
:10764000F894DEBF0FBECDBF8091880F882309F468
:10765000F8C172DF8090960F9090970FA090980FCE
:10766000B090990F00919E0F10919F0FB80188273D
:1076700077FD8095982F0E944FDDA50194010E940F
:10768000D3DB6B017C016093700F7093710F80935B
:10769000720F9093730F20E030E040E251E40E94BB
:1076A000B0DE181624F481E08093670FF7C020E065
:1076B00030E040E251ECC701B6010E94ADDC87FD2D
:1076C00002C0012B21F481E08093670F0CC18091EF
:1076D000670F882351F01092840F1092850F10923B
:1076E000860F1092870F1092670F20911802309129
:1076F000190240911A0250911B02C701B6010E9463
:1077000082DF69837A838B839C8360937C0F709381
:107710007D0F80937E0F90937F0F2091840F309187
:10772000850F4091860F5091870FC701B6010E94C7
:10773000D4DB2B013C0120906C0F30906D0F109129
:107740006E0F00916F0F9101412F502F0E94ADDC01
:1077500087FD14C02090680F3090690F10916A0F58
:1077600000916B0F9101412F502FB201C3010E9474
:10777000B0DE18161CF01201162D072DC101A12F25
:10778000B02F8093840F9093850FA093860FB093B2
:10779000870F2091140230911502409116025091EA
:1077A0001702B101812F902F0E9482DF6D837E83AB
:1077B0008F8398876093780F7093790F80937A0FF7
:1077C00090937B0F2091800F3091810F4091820F19
:1077D0005091830FC501B4010E94D3DB20911002A8
:1077E0003091110240911202509113020E9482DFE7
:1077F00020ED3CEC4CE45DE30E9482DF2B013C0178
:1078000023E333E343E75FE36091740F7091750FF7
:107810008091760F9091770F0E9482DF9B01AC01DF
:10782000C301B2010E94D4DB2B013C016093740FB1
:107830007093750F8093760F9093770F2D813E8113
:107840004F81588569817A818B819C810E94D4DB2C
:10785000A30192010E94D3DB2B013C0120E030E028
:107860004FE753E40E94B0DE20E030E0A901181693
:10787000E4F4C701B6010E94B0DE18167CF4A7013B
:107880009601B101812F902F0E94D3DB6093840F6A
:107890007093850F8093860F9093870F412C512C06
:1078A0009FE7692E93E4792E21C0C301B2010E94A3
:1078B000ADDC87FF1BC020E030E0A901C701B601A5
:1078C0000E94ADDC87FF0FC0A7019601B101812F97
:1078D000902F0E94D3DB6093840F7093850F809369
:1078E000860F9093870F412C512C32018092800F8C
:1078F0009092810FA092820FB092830F60915A0FE5
:1079000070915B0F882777FD8095982F0E944FDD3F
:107910009B01AC01C501B4010E94B0DE1816DCF475
:107920006091080270910902882777FD8095982F51
:107930000E944FDD9B01AC01C501B4010E94ADDC8A
:1079400087FF09C0C301B2010E941CDD75956795D0
:107950006093620F02C01092620F0E943ED70091A6
:107960005E0F10915F0F2091600F3091610F601BCF
:10797000710B820B930B653C79408105910558F0A2
:1079800031DE0E943ED760935E0F70935F0F80934D
:10799000600F9093610F0E943ED70091630F10918A
:1079A000640F2091650F3091660F601B710B820B85
:1079B000930B683873418105910508F442C00E9419
:1079C0003ED76093630F7093640F8093650F90931D
:1079D000660FC090900FD090910FE090920FF090B2
:1079E000930F20E030E040E751E4C701B6010E9468
:1079F000B0DE18161CF520E030E046E153E4C70184
:107A0000B6010E94ADDC87FF19C060919C0F709198
:107A10009D0F882777FD8095982F0E944FDD9B0151
:107A2000AC01C701B6010E94B0DE87FD03C0109211
:107A30008F0F07C08FE780938F0F03C010928F0FB7
:107A4000A59828960FB6F894DEBF0FBECDBFDF9184
:107A5000CF911F910F91FF90EF90DF90CF90BF904B
:107A6000AF909F908F907F906F905F904F903F90DE
:107A70002F900895CF93DF9310926C0F10926D0F9B
:107A800010926E0F10926F0F209114023091150218
:107A9000409116025091170260E070E08FE793E486
:107AA0000E94B4DC6093680F7093690F80936A0F33
:107AB00090936B0F6D9A8091010180618093010119
:107AC0009D9A8091010188608093010187ED8093E8
:107AD0007A0010927E0010927D0080917E0081607D
:107AE00080937E0080917E00826080937E008091F2
:107AF0007E00846080937E0080E888BD80916E0067
:107B0000846080936E006AEF70E080E090E00E94F5
:107B10006DD78FE090E090935B0F80935A0F60E0F9
:107B200080910A0290910B0237DC20E030E040E7C0
:107B300051E40E94ADDC87FF0AC080910A02909157
:107B40000B02409790930B0280930A02E8CF89E0E2
:107B500091E0909309028093080260E080915C0FAD
:107B600090915D0F19DC20E030E844E853E40E9476
:107B7000B0DE181654F480915C0F90915D0F409622
:107B800090935D0F80935C0FE8CFC091580FD09118
:107B9000590FCE0161DB20E030E046E153E40E9462
:107BA000B0DE181634F46096D093590FC093580F76
:107BB000ECCFDF91CF910895089510929F0F10920E
:107BC0009E0F10929D0F10929C0F1092620F75984D
:107BD00010929D0F10929C0F10928F0FA5980895F0
:107BE0002F923F924F925F926F927F928F929F92CD
:107BF000AF92BF92CF92DF92EF92FF920F931F93BB
:107C0000CF93DF93CDB7DEB7AE970FB6F894DEBF54
:107C10000FBECDBF6B8F7C8F8D8F292E5A874987E2
:107C20003CA72BA70E943ED76F8F78A389A39AA366
:107C30000E943ED76FA378A789A79AA729853A857E
:107C4000121613061CF0E4EEFBE017C0E7EFFBE0B2
:107C50008191882339F09091C00095FFFCCF8093EB
:107C6000C600F6CF8091C00085FFFCCF1BC290916B
:107C7000C00095FFFCCF8093C60081918111F7CFA2
:107C80008091C00085FFFCCF8AE08093C60095DF1D
:107C900049855A858FE7452B99F180938F0F8F8DFA
:107CA00098A1A9A1BAA1898B9A8BAB8BBC8B8D872C
:107CB0009E87AF87B88B1D8290E4988FACE1A98F27
:107CC000B6E4BA8F1DA61D8A1E8A1F8A2FE730E0F0
:107CD00040E050E029833A834B835C83EFE74E2EEC
:107CE000512C612C712C1BA21CA21DA21EA231E0E2
:107CF0003E8F1C861B86312C00E010E01EA605C0BE
:107D00008093620FCCCF0E9455988091880F882372
:107D100009F4F6C011DC49855A85452B51F03090A5
:107D2000900F0091910F1091920F5091930F5EA7B9
:107D300009C03090960F0091970F1091980F809185
:107D4000990F8EA7232D302F412F5EA56DA57D891C
:107D50008E899F890E94B0DE18162CF03DA60D8BEF
:107D60001E8B9EA59F8B232D302F412F5EA56D81ED
:107D7000788D898D9A8D0E94ADDC87FD05C03D828E
:107D8000088F198FAEA5AA8F0E943ED72FA138A5C4
:107D900049A55AA5621B730B840B950B653C794072
:107DA0008105910538F01EDC0E943ED76FA378A7AD
:107DB00089A79AA74E8D442309F44FC02B8D3C8D83
:107DC0004D8D522D632D702F812F9EA50E94B0DE08
:107DD00018160CF095C00E943ED729893A894B8924
:107DE0005C89621B730B840B950B693873418105A9
:107DF000910508F485C0D301C20129813A814B81E4
:107E00005C81821B930BA40BB50B49855A85B595F4
:107E1000A79597958795452B19F080938F0F02C0F2
:107E20008093620F0E943ED76D877E878F87988BE5
:107E3000DC01CB0129893A894B895C89821B930B30
:107E4000A40BB50B8BA39CA3ADA3BEA33B8D3DA7F9
:107E50004C8D4D8B5D8D5E8B2F8A2B8D3C8D4D8D8A
:107E6000522D632D702F812F9EA50E94ADDC87FFC0
:107E7000EEC20E943ED72D853E854F855889621BF4
:107E8000730B840B950B693873418105910508F4D8
:107E9000DEC20E943ED7698B7A8B8B8B9C8BDC0178
:107EA000CB012D853E854F855889821B930BA40BF2
:107EB000B50B4B855C85452B09F010C189819A81F2
:107EC000AB81BC81840D951DA61DB71D29853A8502
:107ED000B595A79597958795232B09F4B5C28093FF
:107EE0008F0F4B855C854F5F5F4F5C874B875B8D4A
:107EF0005D838C8D888F9D8D998F2A8EA1E0AE8FAA
:107F000020E030E040EA51E46B8D7C8D8D8D922D28
:107F10000E94D4DB9B01AC01632D702F812F9EA5A5
:107F20000E94B0DE181694F4EFEFF2E084918823FB
:107F300041F09091C00095FFFCCF8093C600319630
:107F4000F5CF8091C00085FFFCCFACC00E943ED72A
:107F50002F8D38A149A15AA1621B730B840B950B7D
:107F6000613D77408105910508F44FC049855A85E8
:107F7000452B81F0E0908F0FF12CE9EFF2E0849136
:107F80008823C1F09091C00095FFFCCF8093C6007C
:107F90003196F5CFE090620FF12CE3EFF2E084919F
:107FA000882341F09091C00095FFFCCF8093C600DC
:107FB0003196F5CF22E030E0432D502F612F7EA582
:107FC0008BE295E10E9458B8EFEEF2E084918823AD
:107FD00041F09091C00095FFFCCF8093C600319690
:107FE000F5CF4AE050E0B7018BE295E10E9482B7FD
:107FF0008091C00085FFFCCF8AE08093C6000E947C
:108000003ED76F8F78A389A39AA30E943ED76B01B6
:108010007C010E943ED789889A88AB88BC882D85D0
:108020003E854F855889820E931EA41EB51EC81822
:10803000D908EA08FB08C60ED71EE81EF91E31E86B
:10804000C3163FE4D30632E1E306F10490F0E2ED1B
:10805000F2E08491882341F09091C00095FFFCCF1D
:108060008093C6003196F5CF8091C00085FFFCCF8C
:1080700019C04B855C858BA59CA5841795070CF0D2
:1080800042CEE6E7F2E08491882341F09091C0006F
:1080900095FFFCCF8093C6003196F5CF8091C0004C
:1080A00085FFFCCF8AE08093C600AE960FB6F894A9
:1080B000DEBF0FBECDBFDF91CF911F910F91FF901B
:1080C000EF90DF90CF90BF90AF909F908F907F9078
:1080D0006F905F904F903F902F9008958BA09CA041
:1080E000ADA0BEA0880E991EAA1EBB1E2BA13CA14E
:1080F0004DA15EA1281B390B4A0B5B0BCA01B901CC
:1081000029813A814B815C810E9448E0A50194015C
:108110000E94ADE0240D351D461D571D243131054B
:108120004105510504F129013A013CEE4316510481
:10813000610471042CF06BEE462E512C612C712CD5
:1081400040E84416510461047104DCF08EEF90E0C5
:10815000A0E0B0E084199509A609B70989839A833C
:10816000AB83BC8312C054E1452E512C612C712C81
:1081700024E130E040E050E029833A834B835C8384
:1081800004C049825A826B827C82E8E6F3E08491E3
:10819000882341F09091C00095FFFCCF8093C600EA
:1081A0003196F5CF2AE030E0B301A2018BE295E1F0
:1081B0000E9457B7E3E6F3E08491882341F0909161
:1081C000C00095FFFCCF8093C6003196F5CF2AE022
:1081D00030E049815A816B817C818BE295E10E947C
:1081E00057B7ECE5F3E08491882341F09091C0000B
:1081F00095FFFCCF8093C6003196F5CF22E030E0AA
:108200004D81588D698D7A8D8BE295E10E9458B829
:10821000E5E5F3E08491882341F09091C00095FF5B
:10822000FCCF8093C6003196F5CF22E030E04DA51B
:108230005D896E897F898BE295E10E9458B88091B3
:10824000C00085FFFCCF8AE08093C6002B853C856B
:10825000233031050CF432CE69817A818B819C8187
:108260000E944FDD20E030E040E850E40E9482DFD1
:108270006B017C012D81388D498D5A8D6DA57D89CD
:108280008E899F890E94D3DB20ED3FE049E450E4D2
:108290000E9482DF20E030E040E05FE30E9482DF66
:1082A0009B01AC01C701B6010E94B4DC6B017C01EB
:1082B000C501B4010E944FDD20E030E04AE754E4FC
:1082C0000E94B4DC4B015C01EFE4F3E0849188236D
:1082D00041F09091C00095FFFCCF8093C60031968D
:1082E000F5CF22E030E0B701A6018BE295E10E94D4
:1082F00058B8E9E4F3E08491882341F09091C000FC
:1083000095FFFCCF8093C6003196F5CF22E030E098
:10831000B501A4018BE295E10E9458B88091C0009C
:1083200085FFFCCF8AE08093C6002AE939E949E15C
:108330005FE3C701B6010E9482DF6B017C019B01F4
:10834000AC010E94D4DBA50194010E94B4DC6D83D2
:108350007E838F839887A5019401C701B6010E948F
:1083600082DF20E030E040E05EE30E9482DF4B01EC
:108370005C01EBE3F3E08491882341F09091C0002D
:1083800095FFFCCF8093C6003196F5CF8091C00059
:1083900085FFFCCF8AE08093C600E5E3F3E084919B
:1083A000882341F09091C00095FFFCCF8093C600D8
:1083B0003196F5CF22E030E0B701A6018BE295E1DE
:1083C0000E9458B88091C00085FFFCCF8AE080935E
:1083D000C600EFE2F3E08491882341F09091C00061
:1083E00095FFFCCF8093C6003196F5CF22E030E0B8
:1083F0004D815E816F8178858BE295E10E9458B84E
:108400008091C00085FFFCCF8AE08093C600E9E23E
:10841000F3E08491882341F09091C00095FFFCCF58
:108420008093C6003196F5CF22E030E0B501A4017B
:108430008BE295E10E9458B88091C00085FFFCCF87
:108440008AE08093C6003ACD8093620F4ACD1E8E9B
:1084500057CDCF93C82FB1DB0E94A269811134C0E0
:10846000E8E9F9E49491992341F08091C00085FFF7
:10847000FCCF9093C6003196F5CF6C2F70E04AE0A8
:1084800050E08BE295E10E9482B78091C00085FFA9
:10849000FCCF8AE08093C600ECE2F2E0849188236E
:1084A00041F09091C00095FFFCCF8093C6003196BB
:1084B000F5CF8091C00085FFFCCF8AE08093C60095
:1084C0008FE192E00E94C697CF910C944A69CF93B6
:1084D000C82F73DB0E94A269811134C0E8E9F9E476
:1084E0009491992341F08091C00085FFFCCF909337
:1084F000C6003196F5CF6C2F70E04AE050E08BE279
:1085000095E10E9482B78091C00085FFFCCF8AE090
:108510008093C600E2EFF1E08491882341F09091CE
:10852000C00095FFFCCF8093C6003196F5CF8091B7
:10853000C00085FFFCCF8AE08093C60085EE91E005
:108540000E94C697CF910C944A69A5980E94A2698F
:10855000811125C0E8E9F9E48491882341F09091E4
:10856000C00095FFFCCF8093C6003196F5CFEBEAB3
:10857000F1E08491882341F09091C00095FFFCCFF9
:108580008093C6003196F5CF8091C00085FFFCCF67
:108590008AE08093C6008AE991E00E94C6970C9415
:1085A0004A691F920F920FB60F9211240BB60F92C9
:1085B0000F931F932F933F934F935F936F937F93EB
:1085C0008F939F93AF93BF93CF93DF93EF93FF93DB
:1085D00080910702811112C08091620F8093570F22
:1085E000882311F0759A01C0759880918F0F809340
:1085F000560F882311F0A59A01C0A5989091570FA6
:1086000080910702981708F475989091560F809101
:108610000702981708F4A598809107028F5F8F775B
:10862000809307028091060290E08B30910508F05C
:1086300093C0FC01EE58FF4F0C94C9E010927B00F0
:1086400080E480937C0080917A00806480937A003B
:108650000E94CF9781E019C0209178003091790075
:108660008091520F9091530FA091540FB091550FDC
:10867000820F931FA11DB11D8093520F9093530F32
:10868000A093540FB093550F82E08093060264C00C
:1086900010927B0082E480937C0080917A00806459
:1086A00080937A000E94CF9783E0EFCF20917800EB
:1086B0003091790080914E0F90914F0FA091500F03
:1086C000B091510F820F931FA11DB11D80934E0FCA
:1086D00090934F0FA093500FB093510F84E0D5CFDC
:1086E00010927B0081E480937C0080917A0080640A
:1086F00080937A000E94CF9785E0C7CF20917800C1
:108700003091790080914A0F90914B0FA0914C0FBE
:10871000B0914D0F820F931FA11DB11D80934A0F81
:1087200090934B0FA0934C0FB0934D0F86E0ADCFBD
:108730000E94CF9787E0A9CF88E0A7CF0E94CF976C
:1087400089E0A3CF109206028091490F8F5F80933A
:10875000490F02C0109206028091490F803108F43F
:1087600063C08091880F811110C08091520F909149
:10877000530F90939B0F80939A0F80914E0F90917F
:108780004F0F9093950F8093940F81E08093880F03
:108790001092490F1092520F1092530F1092540FD3
:1087A0001092550F10924A0F10924B0F10924C0FCF
:1087B00010924D0F1092450F1092460F1092470FD6
:1087C0001092480F10924E0F10924F0F1092500FB0
:1087D0001092510F20919A0F30919B0F80915C0F56
:1087E00090915D0F8217930714F080E032DE2091A4
:1087F0009A0F30919B0F80910A0290910B022817DB
:10880000390714F080E063DE2091940F3091950FCA
:108810008091580F9091590F821793072CF0109266
:108820009D0F10929C0F91DE00E010E0E801CC0F4C
:10883000DD1FC757D04F888199811816190644F457
:1088400061E0802F0E946EC188819981019709C0E3
:10885000892B49F060E0802F0E946EC18881998148
:108860000196998388830F5F1F4F03301105F1F63E
:10887000FF91EF91DF91CF91BF91AF919F918F9138
:108880007F916F915F914F913F912F911F910F9128
:108890000F900BBE0F900FBE0F901F9018952CEAF3
:1088A00035EC47E25EE30C9482DF2CEA35EC47E2DC
:1088B0005EE30C94B4DC2CEA35EC47E25EE30C9406
:1088C000B4DC2CEA35EC47E25EE30C9482DFCF9314
:1088D000DF93EC0160E08E810E9497D681E090E00A
:1088E0000E9491D761E08E810E9497D681E090E04E
:1088F0000E9491D760E08E810E9497D684E690E036
:10890000DF91CF910C9491D7CF92DF92EF92FF92AB
:108910000F931F93CF93DF937C01C0E0D0E0C62E6E
:10892000D12C87010C0F1D1F61E0F80187810E9487
:108930005ED6B6010C2E02C0759567950A94E2F7D3
:108940006170F80187810E9497D62196C430D105C5
:1089500041F7C701DF91CF911F910F91FF90EF90E9
:10896000DF90CF90B4CFCF92DF92EF92FF920F9330
:108970001F93CF93DF937C01C0E0D0E0C62ED12CB3
:1089800087010C0F1D1F61E0F80187810E945ED6F0
:10899000B6010C2E02C0759567950A94E2F76170D6
:1089A000F80187810E9497D62196C830D10541F7FA
:1089B000C701DF91CF911F910F91FF90EF90DF9052
:1089C000CF9085CF1F93CF93DF93EC01162F642FA9
:1089D0008C810E9497D68D818F3F19F060E00E94B4
:1089E00097D68F85612F84FF05C0CE01DF91CF918F
:1089F0001F91B9CF70E084E0759567958A95E1F78E
:108A0000CE0182DF612FCE01DF91CF911F917CCF0C
:108A100040E0D8CF61E0FCDF80E496E00C9491D791
:108A200062E0F6DF80E496E00C9491D7CF93DF9379
:108A3000CDB7DEB728970FB6F894DEBF0FBECDBF17
:108A400028E0EFE5FBE0DE01119601900D922A95FA
:108A5000E1F7FC012389421710F04FEF420FFE01AE
:108A60003196E40FF11DE40FF11D2081260F2068DF
:108A7000622F28960FB6F894DEBF0FBECDBFDF91F0
:108A8000CF91C6CFFC016089262F2460208B6C60BB
:108A9000BFCFCF93DF93EC01423018F08F85886011
:108AA0008F874B8B1C8A222329F0413019F48F8544
:108AB00084608F8780E593EC0E9491D760E08C8181
:108AC0000E9497D660E08E810E9497D68D818F3F5D
:108AD00019F060E00E9497D66F8564FD19C063E0CD
:108AE000CE0112DF84E991E10E9491D763E0CE01CB
:108AF0000BDF84E991E10E9491D763E0CE0104DFAE
:108B000086E990E00E9491D762E0CE01FDDE13C0BD
:108B10006062CE017DDF84E991E10E9491D76F858B
:108B20006062CE0175DF86E990E00E9491D76F8583
:108B30006062CE016DDF6F856062CE0169DF8CE31C
:108B400090E00E9491D784E0888BCE019BDF8CE37C
:108B500090E00E9491D7CE015DDF88EB9BE00E9400
:108B600091D782E0898B66E0CE0152DF8CE390E002
:108B7000DF91CF910C9491D76F927F928F92AF92A9
:108B8000CF92EF920F931F93CF93DF93CDB7DEB7C2
:108B90003C01162F842F5E854F8538899989F30112
:108BA000848325830683E782C086A18682865387D5
:108BB00044873587968761E00E945ED6F301858100
:108BC0008F3F19F061E00E945ED661E0F30186817B
:108BD0000E945ED6112319F0F301178603C080E1CD
:108BE000F301878720E041E060E1C301DF91CF918D
:108BF0001F910F91EF90CF90AF908F907F906F90DB
:108C000048CF8F92AF92CF92EF920F93DC011396E1
:108C10001C921E921297E5E2FCE0ED93FC931F92EA
:108C20001F921F921F928C2CAE2CC02EE22E042F6E
:108C30002FEF462F61E0A0DF0F900F900F900F9065
:108C40000F91EF90CF90AF908F900895CF93DF93D7
:108C5000EC01423018F08F8588608F874B8B1C8A1F
:108C6000222329F0413019F48F8584608F8780E5B5
:108C700093EC0E9491D760E08C810E9497D660E0CF
:108C80008E810E9497D68D818F3F19F060E00E94FF
:108C900097D66F8564FD19C063E0CE0135DE84E9A7
:108CA00091E10E9491D763E0CE012EDE84E991E14B
:108CB0000E9491D763E0CE0127DE86E990E00E9412
:108CC00091D762E0CE0120DE13C06062CE01A0DE4B
:108CD00084E991E10E9491D76F856062CE0198DEB0
:108CE00086E990E00E9491D76F856062CE0190DEA8
:108CF0006F856062CE018CDE8CE390E00E9491D79C
:108D000084E0888BCE01BEDE8CE390E00E9491D798
:108D1000CE0186DE80E496E00E9491D782E0898BC6
:108D200066E0CE0175DE8CE390E00E9491D740E0D2
:108D300068E0CE017BDE62E07DE0CE010E94CBDB0D
:108D400041E068E0CE0172DE62E07DE0CE010E948B
:108D5000CBDB42E066E0CE0169DE60E07DE0CE0183
:108D6000DF91CF910C94CBDBCF92DF92EF92FF9209
:108D70000F931F93CF93DF931F921F92CDB7DEB750
:108D80008C01677088E0689FB00111246064C8019D
:108D900049835A833DDE4981C42E5A81D52EE12C68
:108DA000F12CD6016D916D01D801ED91FC910190EE
:108DB000F081E02DC8011995BFEFEB1AFB0AE8E03E
:108DC000EE16F10471F70F900F90DF91CF911F9184
:108DD0000F91FF90EF90DF90CF90089541E0F2DD8A
:108DE00081E090E008950F931F93CF93DF93EC0100
:108DF0008B0144E150E0BC0180EA9FE00E94D5E392
:108E0000CE010E94B4E3992744E150E0481B590B7E
:108E1000B8018056904F0E94D5E380EA9FE0DF9131
:108E2000CF911F910F910895AF92BF92CF92DF9291
:108E3000EF92FF920F931F93CF93DF93EC015B01AF
:108E40007A01690144E150E0BC0180EA9FE00E94A0
:108E5000D5E3CE010E94B4E3EC01DD2704E110E08C
:108E6000A8014C1B5D0BB501CE018056904F0E94AE
:108E7000D5E3C5010E94B4E3C80FD91FDD27A801BF
:108E80004C1B5D0BB701CE018056904F0E94D5E37D
:108E9000C7010E94B4E38C0F9D1F9927A801481BAE
:108EA000590BB6018056904F0E94D5E380EA9FE0AF
:108EB000DF91CF911F910F91FF90EF90DF90CF90B6
:108EC000BF90AF9008952F923F924F925F926F9212
:108ED0007F928F929F92AF92BF92CF92DF92EF924A
:108EE000FF920F931F93CF93DF93CDB7DEB7CF548D
:108EF000D1090FB6F894DEBF0FBECDBF1C017E8F27
:108F00006D8F4A012FAB09AF2896EFAE28972C96AC
:108F1000ACAEBDAECEAEDFAE2C9734E0239F500199
:108F20001124FC01EA0DFB1D80819181A281B38196
:108F3000898F9A8FAB8FBC8FDA01AA0DBB1DBCAF96
:108F4000ABAF4D905D906D907C90A3019201698DC7
:108F50007A8D8B8D9C8D0E94D4DB21966CAF7DAF7A
:108F60008EAF9FAF2197B4E00B9F80011124F101D8
:108F7000E00FF11F20813181428153812F8F38A36F
:108F800049A35AA3A401400F511F23965FAF4EAFD0
:108F90002397DA01CD90DD90ED90FC90A70196012A
:108FA0006F8D78A189A19AA10E94D4DB27966CAF1E
:108FB0007DAF8EAF9FAF27972896EFAD2897B4E08F
:108FC000EB9FC0011124F101E80FF91F20813181CD
:108FD000428153812BA33CA34DA35EA3ED8DFE8D57
:108FE000E80FF91F60817181828193810E94D3DB38
:108FF0006FA378A789A79AA7AD8DBE8D1C968D917A
:109000009D910D90BC91A02D60968CAF9DAFAEAFA1
:10901000BFAF6097D1011C962D913D914D915C9110
:109020001F972BA73CA74DA75EA7A30192015058FD
:109030002D8B3E8B4F8B588FD701C601B058898B33
:109040009A8BAB8BBC8BED8DFE8DEA0DFB1D2081C9
:109050003181428153812FA738AB49AB5AAB21965E
:109060002CAD3DAD4EAD5FAD21976FA578A989A917
:109070009AA90E94D3DB6B017C01ED8DFE8DE00F80
:10908000F11F80819181A281B3818BAB9CABADAB91
:10909000BEAB27962CAD3DAD4EAD5FAD2797BC0165
:1090A000CD010E94D3DB4B015C01A70196016D89C4
:1090B0007E898F89988D0E9482DF2B013C01A5015A
:1090C000940169897A898B899C890E9482DF9B013E
:1090D000AC01C301B2010E94D4DB2B013C01A5010C
:1090E00094016D897E898F89988D0E9482DF4B0162
:1090F0005C01A701960169897A898B899C890E9404
:1091000082DF9B01AC01C501B4010E94D3DBA30146
:1091100092010E9447DC6B017C0120E030E0A90154
:109120000E94ADDC87FF0AC02BED3FE049EC50E424
:10913000C701B6010E94D4DB6B017C01AA968FADFA
:10914000AA97882351F02BED3FE049EC50E4C7018A
:10915000B6010E94D3DB6B017C012FA538A949A978
:109160005AA9698D7A8D8B8D9C8D0E94ADDC811101
:109170001FC02BA93CA94DA95EA96F8D78A189A11B
:109180009AA10E94ADDC811113C020E030E0A9015A
:10919000C701B6010E94ADDC81110AC02BED3FE092
:1091A00049EC50E4C701B6010E94D4DB6B017C019D
:1091B000A9962CAD3DAD4EAD5FADA997C701B601E7
:1091C0000E9482DF2FA138A549A55AA55F770E948A
:1091D000BDDE4B015C012FE632E143E85AE30E9419
:1091E000ADDC87FDC8C1C501B4010E948ADD0E94C3
:1091F00021DD7A8F698FDB01AB2B21F4E1E0F0E018
:10920000FA8FE98F298D3A8DB90180E090E00E94B4
:109210004DDD4B015C019B01AC01C701B6010E9411
:10922000B4DC2B013C01A50194016FA178A589A5AF
:109230009AA50E94B4DC6FA778AB89AB9AAB2BA53B
:109240003CA54DA55EA560966CAD7DAD8EAD9FAD88
:1092500060970E94D3DBA50194010E94B4DC6BAB44
:109260007CAB8DAB9EAB20E030E040E05FE3C30120
:10927000B2010E9482DFA30192010E9482DF9B0162
:10928000AC0160E070E080E89FE30E94D3DB6FA355
:1092900078A789A79AA7CE010196FC0128964FAD21
:1092A000289734E0439FE00DF11D11242BA13CA130
:1092B0004DA15EA120833183428353832BA53CA51E
:1092C0004DA55EA52D873E874F87588BB12C41E079
:1092D00050E058A34F8F1C01BFA9A4E0BA9F800D96
:1092E000911D112498AF8FAB910159AD44E0549F6B
:1092F000200D311D11243AAF29AFFCA7EBA74F8DEC
:1093000058A1898D9A8D4817590708F01AC188E12C
:109310008B150CF444C02FA138A549A55AA569891D
:109320007A898B899C890E9482DF6B017C01A30171
:1093300092016D897E898F89988D0E9482DFA701B5
:1093400096010E94D4DBA62E172F982E892E2FA1CE
:1093500038A549A55AA56D897E898F89988D0E9467
:1093600082DF6B017C01A301920169897A898B8973
:109370009C890E9482DF9B01AC01C701B6010E945B
:10938000D3DB6D8B7E8B8F8B988FB3948A2D912F2F
:10939000A92DB82D898B9A8BAB8BBC8B6CC0AF8DF4
:1093A000B8A1BD0180E090E00E944DDDA3019201D3
:1093B0000E9482DF6B017C010E94B1DC698B7A8B99
:1093C0008B8B9C8BC701B6010E94E5DF4B015C01D2
:1093D000EBADFCADC080D180E280F380F7FAF09471
:1093E000F7F8F0942396AEADBFAD23972D913D9144
:1093F0004D915C912BA33CA34DA35EA329893A898F
:109400004B895C89C701B6010E9482DF6D8B7E8B20
:109410008F8B988FA50194016BA17CA18DA19EA13A
:109420000E9482DF9B01AC016D897E898F89988DB6
:109430000E94D4DB6D8B7E8B8F8B988FA50194015E
:10944000C701B6010E9482DF6B017C0129893A893C
:109450004B895C896BA17CA18DA19EA10E9482DFBA
:109460009B01AC01C701B6010E94D3DB698B7A8BEB
:109470008B8B9C8BB12C2D893E894F89588D2196E1
:109480006CAD7DAD8EAD9FAD21970E94D4DBEFA971
:10949000F8AD608371838283938329893A894B89EC
:1094A0005C8927966CAD7DAD8EAD9FAD27970E94F0
:1094B000D4DBA9ADBAAD6D937D938D939C93139737
:1094C0002FA538A949A95AA9EBA5FCA560817181EE
:1094D000828193810E94D4DBABA5BCA56D937D9363
:1094E0008D939C9313972BA93CA94DA95EA96D85DB
:1094F0007E858F8598890E94D4DB6D877E878F87D4
:10950000988BC1010E949B60FE01E659FF4F6F01DD
:109510002C96ECACFDAC0EAD1FAD2C979E01235FDD
:109520003F4FAE01475F5F4FBE016B5F7F4FC10191
:109530000E9469C82F8D38A12F5F3F4F38A32F8F0E
:10954000DECE2D8D3E8D245F3F4F4D8D5E8D485F6D
:109550005F4F6D8D7E8D6C5F7F4FDE01A659BF4FD3
:109560006D012C96ECACFDAC0EAD1FAD2C978D8D26
:109570009E8D0E9469C8C15BDF4F0FB6F894DEBFB5
:109580000FBECDBFDF91CF911F910F91FF90EF9054
:10959000DF90CF90BF90AF909F908F907F906F9013
:1095A0005F904F903F902F900895FC011482178296
:1095B0001382128283E29DE091838083089523E2E7
:1095C0003DE0FC01318320832781222319F004969A
:1095D0000C9424300895CF92DF92EF92FF920F9374
:1095E0001F93CF93DF93EC01875B9F4FDEDFCE01AC
:1095F00086599F4FDADF7E0129E8E20EF11C8701D0
:109600006E0131E4C31A3EEFD30AC801CEDF015E1A
:109610001F4F0C151D05C9F7FE01EF53FE4F89E1E1
:10962000818314823596178ACE018C519E4FBDDFFF
:10963000FE01EB56FD4F1082118212821382389682
:1096400010821182128213821A821B82188219825E
:109650006E0187E6C81A8DEFD80AF60110821182D2
:1096600012821382F80111821082FE01ED5FFD4F1C
:10967000108286E391E0F7019C0111922150304065
:10968000E1F7FE01EF55FD4F81E08083C95BDF4FBD
:10969000198218820E943ED768577C4E8F4F9F4F89
:1096A000F6016083718382839383DF91CF911F9151
:1096B0000F91FF90EF90DF90CF900895FC0120E094
:1096C0003EE2DB014C91403241F0283011F430830E
:1096D0003196DB014C91408331962F5F6F5F7F4F56
:1096E0002B3079F7108208952F923F924F925F921C
:1096F0006F927F928F929F92AF92BF92CF92DF92A2
:10970000EF92FF920F931F93CF93DF93CDB7DEB706
:10971000CA58D1090FB6F894DEBF0FBECDBF8C0179
:109720006B017A014901CA57DF4F1882C658D040F1
:1097300084E0E80EF11C180191E1290E311CF801BA
:10974000EA5BFF4FC957DF4FF983E883C758D04022
:109750003801FEE56F1AFDEF7F0A58018CE5A81A63
:109760008DEFB80A90E4492E512C4C0E5D1E94E00A
:10977000490E511CA101BE016F5F7F4FC7010E94BE
:109780008E2E18160CF04AC12C85322F38713031CC
:1097900009F0ACC0F301808191810197029708F430
:1097A000A5C0BE016F5F7F4FCE0187589F4F86DFF8
:1097B000A0961FAEA097F6018081811107C069E2D3
:1097C0007CE0CE01815A9F4F0E942EE4B601CE016B
:1097D000815A9F4F0E942EE4BE0167587F4FCE01F1
:1097E000815A9F4F0E942EE469E27CE0CE01815AAB
:1097F0009F4F0E942EE4CE01805C9F4FD6DE21E079
:10980000AE0147585F4FB701C2010E941B32811160
:1098100047C0F30180819181892B09F041C0E2E9C1
:10982000F9E48491882341F09091C00095FFFCCF2A
:109830008093C6003196F5CFE091C011F0E0EE0FB5
:10984000FF1FE45EFD4F0190F081E02DEA57FE4FCF
:109850000190F081E02D8191882339F09091C00032
:1098600095FFFCCF8093C600F6CF8091C00085FFA6
:10987000FCCF8AE08093C600FE01E758FF4F81913C
:10988000882339F09091C00095FFFCCF8093C600EB
:10989000F6CF8091C00085FFFCCF8AE08093C600A0
:1098A0008BE1FE01EC5BFF4FDE01959601900D927E
:1098B0008A95E1F724968EAD9FAD24979CA38BA348
:1098C00083E29DE09AA389A320E030E0AE014F5DE2
:1098D0005F4FBE01615A7F4FC80106DFCE018196FE
:1098E0006EDECE01805C9F4F6ADE44CF8981882383
:1098F00009F494C08E3209F43DCF8F3509F43ACF84
:10990000F80181898E3209F435CF8F3509F432CFD1
:1099100023FD30CF81E0303109F080E0C957DF4FBF
:10992000E881F981C758D0408083811108C08985BA
:10993000873409F01FCF8A858E3709F41BCF980131
:109940002C5F3F4FBE016F5F7F4FC901C757DF4F8D
:109950002883C958D040C657DF4F3883CA58D040F3
:10996000ADDEF30180819181C757DF4F2881C9584F
:10997000D040C657DF4F3881CA58D0400097F1F425
:10998000F6018191882339F09091C00095FFFCCFBA
:109990008093C600F6CFF9018191882339F0909128
:1099A000C00095FFFCCF8093C600F6CF8091C00029
:1099B00085FFFCCF8AE08093C600DCCE8130910524
:1099C00039F4F50180819181019691838083D2CE13
:1099D000029709F0CFCE8114910439F0B901C40186
:1099E0000E941BE4892B71F419C0CA57DF4FF8811C
:1099F000C658D0402F2F30E0F50180819181281783
:109A0000390761F0CA57DF4FF881C658D040FF5F71
:109A1000CA57DF4FF883C658D040ACCEC657DF4F89
:109A20000FB6F894DEBF0FBECDBFDF91CF911F916F
:109A30000F91FF90EF90DF90CF90BF90AF909F90ED
:109A40008F907F906F905F904F903F902F900895F0
:109A50000F931F93CF93DF93CDB7DEB76F970FB6FA
:109A6000F894DEBF0FBECDBF8C01FC01EE55FD4F5B
:109A70001182108240E050E0BA01835B9F4F0E9448
:109A8000412FC801875B9F4F2BE1FC013496DE011B
:109A9000159601900D922A95E1F7FC018281938140
:109AA0009C838B8383E29DE09A83898320E030E06E
:109AB000AE014F5F5F4F68E07DE0C80115DECE016B
:109AC00001967DDD6F960FB6F894DEBF0FBECDBF59
:109AD000DF91CF911F910F9108952BE1FB013496F7
:109AE000DC01149601900D922A95E1F7FB01228189
:109AF0003381FC01338322830895EF92FF920F9309
:109B00001F93CF93DF93EC011B82FC01E05BFF4FBF
:109B10008081882329F0CE01835B9F4F0E942430EF
:109B20007E018FE3E81A8EEFF80A45E360E0C70193
:109B30000E94395981112CC0E2E9F9E4849188230B
:109B400041F09091C00095FFFCCF8093C600319604
:109B5000F5CFE091C011F0E0EE0FFF1FE45EFD4F86
:109B60000190F081E02DE857FE4F0190F081E02D4B
:109B70008491882341F09091C00095FFFCCF8093A1
:109B8000C6003196F5CF8091C00085FFFCCF9EC006
:109B90008E010A531E4F41E0B701C8010E94F237FF
:109BA000811133C040E0B701C8010E94F237811132
:109BB0002CC0E8E9F9E48491882341F09091C00039
:109BC00095FFFCCF8093C6003196F5CFE091C01190
:109BD000F0E0EE0FFF1FE45EFD4F0190F081E02DFD
:109BE000E657FE4F0190F081E02D8491882341F0EB
:109BF0009091C00095FFFCCF8093C6003196F5CFC1
:109C00008091C00085FFFCCF61C0B801CE01835BAD
:109C10009F4F0E94312D81112CC0E8E9F9E4849115
:109C2000882341F09091C00095FFFCCF8093C6003F
:109C30003196F5CFE091C011F0E0EE0FFF1FE45E2A
:109C4000FD4F0190F081E02DE457FE4F0190F0812F
:109C5000E02D8491882341F09091C00095FFFCCFC6
:109C60008093C6003196F5CF8091C00085FFFCCF70
:109C70002DC081E08B83E2E9F9E48491882341F0EF
:109C80009091C00095FFFCCF8093C6003196F5CF30
:109C9000E091C011F0E0EE0FFF1FE45EFD4F019078
:109CA000F081E02DE257FE4F0190F081E02D84918C
:109CB000882341F09091C00095FFFCCF8093C600AF
:109CC0003196F5CF8091C00085FFFCCF8AE080936C
:109CD000C6008E01075B1F4FB801CE0186599F4F0A
:109CE000FCDEC859DF4F19830883DF91CF911F91A4
:109CF0000F91FF90EF900895FC0112821382089556
:109D0000FC012381222311F021E022830895FC012C
:109D10002281211112820895AF92BF92CF92DF92D9
:109D2000EF92FF920F931F93CF93DF931F92CDB7C4
:109D3000DEB78C018FE2FB0181935F01D12C41E002
:109D40007801F1E4EF1AFEEFFF0A6FE1C62E2D2D28
:109D500030E0F7018081918128173907D8F4C29E3D
:109D6000C001C39E900D112483579F4FB501800FF2
:109D7000911F49830E94D82CC50149815C0101963D
:109D8000F5012081222321F04D3810F44F5FF6CFEA
:109D9000D394DDCF47FD11C0B501C80188519E4F56
:109DA0000F90DF91CF911F910F91FF90EF90DF9077
:109DB000CF90BF90AF900C94D82CF50110820F90EB
:109DC000DF91CF911F910F91FF90EF90DF90CF9097
:109DD000BF90AF9008953F924F925F926F927F92A3
:109DE0008F929F92AF92BF92CF92DF92EF92FF92AB
:109DF0000F931F93CF93DF93CDB7DEB7AC970FB61A
:109E0000F894DEBF0FBECDBF7C015B01FC018381F6
:109E1000882309F408C1C70188519E4F0E9424304D
:109E2000F7011282CE0101966C01BFDB270198E693
:109E3000490E511CC701875B9F4FF20191838083BC
:109E4000F50180818F3209F084C06FE270E0C501B6
:109E50000E9439E48C010F5F1F4F7AE0372E011505
:109E6000110509F47CC06FE270E0C8010E9439E47A
:109E70004C01009709F474C00817190708F070C066
:109E80003C01601A710AA301B801CE0180960E94BC
:109E900062E4E0E2F0E0EC0FFD1FE60DF71D10823A
:109EA000FE01B0968191882339F09091C00095FF12
:109EB000FCCF8093C600F6CF8091C00085FFFCCF19
:109EC0003092C600F201608171816115710519F04F
:109ED0006C5F7F4F02C060E070E021E0AE01405E49
:109EE0005F4FCE0105960E941B3281112BC0EBE221
:109EF000FCE08491882341F09091C00095FFFCCF55
:109F00008093C6003196F5CFFE01B09681918823EB
:109F100039F09091C00095FFFCCF8093C600F6CF3A
:109F2000EFECF5E48491882341F09091C00095FF17
:109F3000FCCF8093C6003196F5CF8091C00085FF9D
:109F4000FCCF6CC0F201D182C08284010F5F1F4F31
:109F500086CFC70186599F4FF20191838083850187
:109F6000F20180819181009711F0049602C080E097
:109F700090E0B8010E94F132882339F1E1ECF5E478
:109F80008491882341F09091C00095FFFCCF80938D
:109F9000C6003196F5CFF8018191882339F0909170
:109FA000C00095FFFCCF8093C600F6CF8091C00023
:109FB00085FFFCCF8AE08093C600F701E356FD4F92
:109FC00010821182128213822CC0E9EAF5E4849196
:109FD000882341F09091C00095FFFCCF8093C6008C
:109FE0003196F5CFF8018191882339F09091C00026
:109FF00095FFFCCF8093C600F6CFE7EAF5E48491A5
:10A00000882341F09091C00095FFFCCF8093C6005B
:10A010003196F5CF8091C00085FFFCCF8AE0809318
:10A02000C600C601CCDAAC960FB6F894DEBF0FBE00
:10A03000CDBFDF91CF911F910F91FF90EF90DF90F7
:10A04000CF90BF90AF909F908F907F906F905F90D8
:10A050004F903F9008958F929F92AF92BF92CF9270
:10A06000DF92EF92FF92CF93DF931F92CDB7DEB7CF
:10A070007C01FC018281882309F4BCC07196819126
:10A08000882339F09091C00095FFFCCF8093C600E3
:10A09000F6CFE5EAF5E48491882341F09091C00081
:10A0A00095FFFCCF8093C6003196F5CFE091C011AB
:10A0B000F0E0EE0FFF1FE45EFD4F0190F081E02D18
:10A0C000E456FE4F0190F081E02D8491882341F009
:10A0D0009091C00095FFFCCF8093C6003196F5CFDC
:10A0E000F701E356FD4F40815181628173812AE07F
:10A0F00030E08BE295E10E94AEB7E3EAF5E48491AB
:10A10000882341F09091C00095FFFCCF8093C6005A
:10A110003196F5CFF701EB56FD4F408151816281B9
:10A1200073812AE030E08BE295E10E94AEB7809126
:10A13000C00085FFFCCF8AE08093C6000E943ED716
:10A14000E0E6CE2EEAEEDE2EE12CF12CA701960100
:10A150000E948BE049015A016091BD0F7091BE0FC2
:10A160008091BF0F9091C00FA70196010E948BE0D4
:10A17000821A930AC4016CE370E00E9464E0698370
:10A18000CE0101960E944399FC012191CF01222327
:10A1900039F03091C00035FFFCCF2093C600F4CFDA
:10A1A00040E050E06AE38BE295E10E9466B7C401AB
:10A1B0006CE370E00E9464E08983CE0101960E9406
:10A1C0004399FC012191CF01222339F03091C00045
:10A1D00035FFFCCF2093C600F4CFE1EAF5E484918B
:10A1E0008823E1F09091C00095FFFCCF8093C600DA
:10A1F0003196F5CFEFE3FCE08491882341F0909114
:10A20000C00095FFFCCF8093C6003196F5CF8091BA
:10A21000C00085FFFCCF8AE08093C6000F90DF91DD
:10A22000CF91FF90EF90DF90CF90BF90AF909F9035
:10A230008F900895AF92BF92CF92DF92EF92FF92EC
:10A240000F931F93CF93DF935C01EB01FB01019010
:10A250000020E9F78F0101501109061B170B6C0153
:10A26000F8E1CF1AFEEFDF0AF60110826EE470E02B
:10A27000CE010E9439E47C01009729F4F80131975E
:10A28000EC0FFD1F0DC060E270E00E9439E4EC01AC
:10A2900021966AE270E0C7010E9439E4FC0131971F
:10A2A0008DE081838AE082831382BE01C5018C51D7
:10A2B0009E4F0E946BB8F6018081882371F1E8E916
:10A2C000F9E48491882341F09091C00095FFFCCF80
:10A2D0008093C6003196F5CFE091C011F0E0EE0F0B
:10A2E000FF1FE45EFD4F0190F081E02DE056FE4F30
:10A2F0000190F081E02D8491882341F09091C0007D
:10A3000095FFFCCF8093C6003196F5CF8091C000B9
:10A3100085FFFCCF8AE08093C600DF91CF911F912B
:10A320000F91FF90EF90DF90CF90BF90AF90089586
:10A330002F923F924F925F926F927F928F929F9255
:10A34000AF92BF92CF92DF92EF92FF920F931F9343
:10A35000CF93DF93CDB7DEB7CC55D1090FB6F894C4
:10A36000DEBF0FBECDBF4C018C010F551D4F6623C4
:10A3700039F0F8011082F401838181111DC015C0EC
:10A38000F8018081882309F4AFC0F401E756FD4F3E
:10A39000C080D180E280F3800E943ED7C616D706E7
:10A3A000E806F90608F4A0C0E4CFC401A6DBF40176
:10A3B0008381882309F498C07401F7E4EF0EF11C3F
:10A3C000F70181818F9380818F9388E995E49F9332
:10A3D0008F938E01015C1F4F1F930F930E9471E4B6
:10A3E0000F900F900F900F900F900F90B12CF801DD
:10A3F00001900020E9F73197E01BF10BBE1684F4C1
:10A400006801CB0CD11CB7FCDA94F6018081992746
:10A4100087FD90950E94A5E3F6018083B394E7CF72
:10A42000FDE48F0E911C40E050E0BA01C4010E948F
:10A43000412F512CCE0101966C0181E9682E85E4F3
:10A44000782E5E0191E2A90EB11C40E050E0B60109
:10A45000C4010E948E2E1816DCF5412CF6010190E5
:10A460000020E9F73197EC19FD094E1674F4160136
:10A47000240C311C47FC3A94F101808190E00E9449
:10A48000A5E3F10180834394E9CF8A858E37E9F211
:10A4900045E050E0B801C6010E9454E4892BA9F6BA
:10A4A0001F930F937F926F92BF92AF920E9471E4BD
:10A4B000C5010E943A5C8DE895E40E94BA5C0F9059
:10A4C0000F900F900F900F900F9055245394BDCF85
:10A4D000511004C08FEF9FEFF70104C0F701808196
:10A4E0009181019691838083C45ADF4F0FB6F8940F
:10A4F000DEBF0FBECDBFDF91CF911F910F91FF90B7
:10A50000EF90DF90CF90BF90AF909F908F907F9013
:10A510006F905F904F903F902F9008950F931F93EF
:10A52000CF93DF93EC018C0108511E4FC8010E94AC
:10A53000DA2FC8010E94243018821982DF91CF914E
:10A540001F910F910895CF92DF92EF92FF920F9398
:10A550001F93CF93DF93CDB7DEB76F970FB6F89405
:10A56000DEBF0FBECDBF8C016A017C0188E6E80E1C
:10A57000F11CC80186599F4FF70191838083E65CE7
:10A58000FD4F22E030E03183208332967183608377
:10A5900040E050E0BA0104960E94412FF70180810B
:10A5A00091812BE1FC013496DE01159601900D920C
:10A5B0002A95E1F7FC01828193819C838B8383E25E
:10A5C0009DE09A8389839601AE014F5F5F4F68E0FB
:10A5D0007DE0C80189D8CE0101960E94DF4A6F96BE
:10A5E0000FB6F894DEBF0FBECDBFDF91CF911F91A4
:10A5F0000F91FF90EF90DF90CF9008952F923F92B0
:10A600004F925F926F927F928F929F92AF92BF9282
:10A61000CF92DF92EF92FF920F931F93CF93DF932E
:10A62000CDB7DEB7AC970FB6F894DEBF0FBECDBF87
:10A630008C016B01342EDC0113968C91882309F474
:10A6400049C3F801E551FE4F8081882309F4F5C024
:10A650002111C1C07801BDEFEB1AFB0AF70180811F
:10A66000882361F1E8E9F9E48491882341F090912D
:10A67000C00095FFFCCF8093C6003196F5CFE3E292
:10A68000F6E48491882341F09091C00095FFFCCFBF
:10A690008093C6003196F5CF4AE050E061E070E06B
:10A6A0008BE295E10E9482B78091C00085FFFCCFCC
:10A6B0008AE08093C6000E9453640CC3E2E9F9E487
:10A6C0008491882341F09091C00095FFFCCF809346
:10A6D000C6003196F5CFEAE0F6E48491882341F094
:10A6E0009091C00095FFFCCF8093C6003196F5CFC6
:10A6F000F6018191882339F09091C00095FFFCCF3D
:10A700008093C600F6CFEFEFF5E48491882341F003
:10A710009091C00095FFFCCF8093C6003196F5CF95
:10A72000D7018C91FDE8BF2EB801B89E600D711D58
:10A730001124685F7D4FC801EFDAF7018081F801CD
:10A74000B89EE00DF11D1124E85FFD4F8191882333
:10A7500039F09091C00095FFFCCF8093C600F6CFF2
:10A76000E9EFF5E48491882341F09091C00095FFD2
:10A77000FCCF8093C6003196F5CF5801F3E6AF1AAF
:10A78000FDEFBF0AD5014D915D916D917C912AE05D
:10A7900030E08BE295E10E94AEB78091C00085FF6A
:10A7A000FCCF8AE08093C600F7012081F80184E0A5
:10A7B000289FE00DF11D1124EC5FFD4FD5014D9157
:10A7C0005D916D917C9140835183628373832F5F90
:10A7D000F70120832CC0E2E9F9E48491882341F059
:10A7E0009091C00095FFFCCF8093C6003196F5CFC5
:10A7F000E8EEF5E48491882341F09091C00095FF44
:10A80000FCCF8093C6003196F5CFF6018191882365
:10A8100039F09091C00095FFFCCF8093C600F6CF31
:10A820008091C00085FFFCCF8AE08093C600C801FC
:10A8300088519E4F0E94243030C0F801ED5FFD4FDB
:10A840001082E2E9F9E48491882341F09091C000FC
:10A8500095FFFCCF8093C6003196F5CFE7EDF5E488
:10A860008491882341F09091C00095FFFCCF8093A4
:10A87000C6003196F5CFF6018191882339F0909189
:10A88000C00095FFFCCF8093C600F6CF8091C0003A
:10A8900085FFFCCF8AE08093C600D80112961C92F7
:10A8A000FE0131965F01CF010E94D54A2801F8E6EA
:10A8B0004F0E511CC801875B9F4FD2018D939C9313
:10A8C000F60180818F3209F091C06FE270E0C6011D
:10A8D0000E9439E401967C01EAE02E2EE114F10495
:10A8E00009F48AC06FE270E0C7010E9439E44C01AC
:10A8F000009709F482C0E816F90608F07EC03C0112
:10A900006E187F08A301B701CE0180960E9462E411
:10A91000E0E2F0E0EC0FFD1FE60DF71D1082FE01F6
:10A92000B0968191882339F09091C00095FFFCCFBB
:10A930008093C600F6CF8091C00085FFFCCF2092A7
:10A94000C600D2016D917C916115710519F06C5FA3
:10A950007F4F02C060E070E021E0AE01405E5F4FDB
:10A96000CE0105960E941B32811138C0E091C011C2
:10A97000F0E0EE0FFF1FE45EFD4F0190F081E02D4F
:10A98000EE56FE4F0190F081E02D8491882341F036
:10A990009091C00095FFFCCF8093C6003196F5CF13
:10A9A000FE01B0968191882339F09091C00095FF07
:10A9B000FCCF8093C600F6CFE5EDF5E484918823C3
:10A9C00041F09091C00095FFFCCF8093C600319676
:10A9D000F5CF8091C00085FFFCCF43C1F201B18269
:10A9E000A0827401FFEFEF1AFF0A78CFC8018659E1
:10A9F0009F4FD2018D939C937601F801E851FE4F51
:10AA00004F01332009F4E5C0D2016D917C916115AD
:10AA1000710519F06C5F7F4F02C060E070E021E0CB
:10AA2000A701C4010E941B322091C011882309F4A0
:10AA30009AC0F40181899289A389B489F801EB56FF
:10AA4000FD4F80839183A283B383E22FF0E0EE0F6A
:10AA5000FF1FE45EFD4F0190F081E02DEC56FE4FAC
:10AA60000190F081E02D8491D801AB56BD4F882331
:10AA700049F09091C00095FFFCCF8093C6003196BD
:10AA80008491F5CFF7018191882339F09091C0002E
:10AA900095FFFCCF8093C600F6CFE091C011F0E0A7
:10AAA000EE0FFF1FE45EFD4F0190F081E02DEA56AE
:10AAB000FE4F0190F081E02D8491882341F0909128
:10AAC000C00095FFFCCF8093C6003196F5CF4D9125
:10AAD0005D916D917C912AE030E08BE295E10E94DE
:10AAE000AEB78091C00085FFFCCF8AE08093C6009E
:10AAF000F801E356FD4F1082118212821382E09119
:10AB0000C011F0E0EE0FFF1FE45EFD4F0190F081F9
:10AB1000E02DE856FE4F0190F081E02D84918823CE
:10AB200041F09091C00095FFFCCF8093C600319614
:10AB3000F5CF8091C00085FFFCCF8AE08093C600EE
:10AB4000A70160E070E0C801FEDCD80151968C914D
:10AB5000882319F0C801419601C0C7010E94899756
:10AB60008CE49CE0B2C0E22FF0E0EE0FFF1FE45E49
:10AB7000FD4F0190F081E02DEE56FE4F0190F081E7
:10AB8000E02D8491882341F09091C00095FFFCCF87
:10AB90008093C6003196F5CFF7018191882339F073
:10ABA0009091C00095FFFCCF8093C600F6CFE3EDF7
:10ABB000F5E48491882341F09091C00095FFFCCF8B
:10ABC0008093C6003196F5CF8091C00085FFFCCF01
:10ABD00048C0F201608171816115710519F06C5FE7
:10ABE0007F4F02C060E070E026E5A701C4010E942B
:10ABF0001B3281113AC0E091C011F0E0EE0FFF1F4F
:10AC0000E45EFD4F0190F081E02DEE56FE4F019085
:10AC1000F081E02D8491882341F09091C00095FF50
:10AC2000FCCF8093C6003196F5CFF7018191882340
:10AC300039F09091C00095FFFCCF8093C600F6CF0D
:10AC4000E1EDF5E48491882341F09091C00095FFF7
:10AC5000FCCF8093C6003196F5CF8091C00085FF70
:10AC6000FCCF8AE08093C60032C081E0D8018C938B
:10AC7000E091C011F0E0EE0FFF1FE45EFD4F019088
:10AC8000F081E02DE656FE4F0190F081E02D849199
:10AC9000882341F09091C00095FFFCCF8093C600BF
:10ACA0003196F5CFF6018191882339F09091C0005B
:10ACB00095FFFCCF8093C600F6CF8091C00085FF42
:10ACC000FCCF8AE08093C600C7010E948997C50126
:10ACD0000E94DF4AAC960FB6F894DEBF0FBECDBF20
:10ACE000DF91CF911F910F91FF90EF90DF90CF9068
:10ACF000BF90AF909F908F907F906F905F904F909C
:10AD00003F902F90089521E0FC01218340E076CC14
:10AD1000CF92DF92EF92FF920F931F93CF93DF9327
:10AD2000CDB7DEB76F970FB6F894DEBF0FBECDBFBD
:10AD30008C016C0128E6C20ED11C86599F4FF6018A
:10AD400091838083E65CFD4F21E030E031832083F6
:10AD50007801FCE5EF1AFDEFFF0AF701118210827E
:10AD600040E050E0BA0104960E94412FF601808134
:10AD700091812BE1FC013496DE01159601900D9234
:10AD80002A95E1F7FC01828193819C838B8383E286
:10AD90009DE09A83898320E030E0AE014F5F5F4FF2
:10ADA00068E07DE0C8010E94744BCE0101960E94CC
:10ADB000DF4AF701808191816F960FB6F894DEBF6C
:10ADC0000FBECDBFDF91CF911F910F91FF90EF90FC
:10ADD000DF90CF900895AF92BF92CF92DF92EF9223
:10ADE000FF920F931F93CF93DF93CDB7DEB76F978B
:10ADF0000FB6F894DEBF0FBECDBF8C017B01CE0134
:10AE000001960E94D54AF801EF58FF4F80816801F2
:10AE1000811104C029E4C20ED11C03C08AE6C80E09
:10AE2000D11C21E0A701B6016C5F7F4FCE010596D2
:10AE30000E941B3281113AC0E2E9F9E4849188232F
:10AE400041F09091C00095FFFCCF8093C6003196F1
:10AE5000F5CFE091C011F0E0EE0FFF1FE45EFD4F73
:10AE60000190F081E02DEE55FE4F0190F081E02D34
:10AE70008491882341F09091C00095FFFCCF80938E
:10AE8000C6003196F5CFF7018191882339F0909172
:10AE9000C00095FFFCCF8093C600F6CF8091C00024
:10AEA00085FFFCCF8AE08093C60036C0F801E154EC
:10AEB000FE4F808191818A30910530F59C012F5F92
:10AEC0003F4F318320832FE1289F7001299FF00C91
:10AED000112429E8E20EF11CE00EF11E5C01B7011D
:10AEE000C7014F960E946D4D81E0A81AB1082FE16D
:10AEF000E21AF1088FEFA816B80689F7B601C80163
:10AF000087579F4F0E946D4DBE016F5F7F4FC801F5
:10AF100086599F4F0E946D4DCE0101960E94DF4AD7
:10AF20006F960FB6F894DEBF0FBECDBFDF91CF9105
:10AF30001F910F91FF90EF90DF90CF90BF90AF9057
:10AF40000895EF92FF920F931F93CF93DF93EC013D
:10AF5000C154DE4F2881398121153105F9F0215086
:10AF60003109398328838C0107571F4FB80186594F
:10AF70009F4F0E946D4DC80100E010E07C012FE161
:10AF8000E20EF11C288139810217130738F40F5F94
:10AF90001F4FB7010E946D4DC701F0CFDF91CF91D8
:10AFA0001F910F91FF90EF900895EF92FF920F93F2
:10AFB0001F93CF93DF93EC010E94D6C08E010D5FEB
:10AFC0001D4FF80180819E0128513E4F7901882351
:10AFD000A1F1C9010E942430F80180818150808351
:10AFE000BE01FDE88F9F600D711D1124685F7D4FCC
:10AFF00021E041E0CE0102DBF8018081FE0124E086
:10B00000829FE00DF11D1124EC5FFD4F40815181C5
:10B0100062817381FE01E356FD4F40835183628359
:10B020007383C7010E94412FCE01DF91CF911F9101
:10B030000F91FF90EF900C94804E0E944CC1C7017D
:10B040000E9424301A8281E895E4DF91CF911F910C
:10B050000F91FF90EF908EC48FEF8EBD0DB407FE61
:10B06000FDCF8EB508958EBD0DB407FEFDCF0895BA
:10B0700061E0FC0180810C9497D6FC012281322F83
:10B08000306A36953CBD20FD06C031E0263009F41B
:10B0900030E0232F01C020E02DBD60E0FC01808165
:10B0A0000C9497D6CF92DF92EF92FF920F931F935B
:10B0B000CF93DF93EC018B017A010E943ED76B01A5
:10B0C000CBDF8B838F3F49F40E943ED76C197D09FB
:10B0D0006D327140A8F381E144C08E3F11F08FE0E2
:10B0E00040C0E114F104D9F0C70101972FEF2EBD44
:10B0F000F8014FEF9F01201B310B2817390738F457
:10B100000DB407FEFDCF2EB521934EBDF3CF0DB488
:10B1100007FEFDCF2EB5F801E80FF91F2083D801F7
:10B12000E00EF11EC12CD12CAE15BF0579F08D912A
:10B13000ED2DFF27E827EE0FFF1FEA59F94B859108
:10B140009491DC2CCC24C826D926EECF85DF082F9D
:10B1500010E0102F002780DF082BC016D10631F039
:10B1600080E28983CE0184DF80E003C0CE0180DFEE
:10B1700081E0DF91CF911F910F91FF90EF90DF90D1
:10B18000CF9008950F931F93CF93DF93EB010E940D
:10B190003ED78B0161DF8F3F49F00E943ED7601B95
:10B1A000710B6C177D07B0F380E001C081E0DF9187
:10B1B000CF911F910F910895CF92DF92FF920F933D
:10B1C0001F93CF93DF9300D01F92CDB7DEB76C01F2
:10B1D000F62E29833A834B835C834FDF6CE271E068
:10B1E000C601D0DF8F2D80643EDF08E110E05C8176
:10B1F0004B813A812981DA01C901002E04C0B6953C
:10B20000A795979587950A94D2F729833A834B831C
:10B210005C8329DF0850110929813A814B815C81C7
:10B22000083F8FEF180739F7FF2029F0E8E0FE16F6
:10B2300021F08FEF03C085E901C087E814DFFCE04F
:10B24000FF1201C009DF10E007DFF601838387FFEB
:10B2500004C01F3F11F01F5FF7CF0F900F900F90AA
:10B260000F90DF91CF911F910F91FF90DF90CF90C2
:10B270000895BF92CF92DF92EF92FF920F931F93A8
:10B28000CF93DF93EC01B62E1C82198248830E9473
:10B290003ED78B0161E088810E945ED6CE01E8DE58
:10B2A00060E082E30E945ED661E083E30E945ED6A6
:10B2B00061E084E30E945ED661E085E30E945ED691
:10B2C00061E085E30E9497D685E08A8382E58CBDA4
:10B2D0001DBC6AE0F62E8FEFC6DEFA94E1F720E09F
:10B2E00030E0A90160E0CE0167DFF82E8B8381E0BA
:10B2F000F81649F00E943ED7601B710B613D774004
:10B3000070F381E046C02AEA31E040E050E068E0B6
:10B31000CE0152DF82FF02C0FC820CC054E0F52E49
:10B320009BDE8B83FA94E1F78A3A11F082E031C018
:10B3300082E08C838C81823031F4C12CD12CE12CC1
:10B3400040E4F42E03C0C12CD12C760120E030E083
:10B35000A90167E3CE0130DFA701960169E2CE01C2
:10B360002BDF8B83882349F00E943ED7601B710B33
:10B37000613D774058F38AE00CC08C818230B1F493
:10B3800020E030E0A9016AE3CE0116DF882329F02E
:10B3900088E08983CE016CDE14C05EDE807C803C58
:10B3A00011F483E08C8358DE57DE56DECE0160DE7A
:10B3B00086E08B1518F488E1898303C0BA8281E0A6
:10B3C00001C080E0DF91CF911F910F91FF90EF902E
:10B3D000DF90CF90BF900895AF92BF92CF92DF924F
:10B3E000EF92FF920F931F93CF93DF93EC016A01CB
:10B3F0007B0189018C81833039F0F9E0CC0CDD1CB4
:10B40000EE1CFF1CFA95D1F773E0B72EE4E0AE2EE8
:10B41000BA94A701960161E1CE01CEDE882311F036
:10B42000A98207C040E052E0B801CE013BDE8111A5
:10B430000EC0CE01BB2049F01BDE20E030E0A901A8
:10B440006CE0CE01B9DE1982E3CF12DE80E0DF913D
:10B45000CF911F910F91FF90EF90DF90CF90BF9011
:10B46000AF900895CF93DF93EC016EBD20E030E004
:10B470000DB407FEFDCFFA01E20FF31F80818EBDF0
:10B480000DB407FEFDCF81818EBD2E5F3F4F21158C
:10B4900082E0380769F70DB407FEFDCF8FEFE3DDDB
:10B4A0008FEFE1DDD9DD8B838F71853031F083E162
:10B4B0008983CE01DDDD80E001C081E0DF91CF91A5
:10B4C00008950F931F93CF93DF93EC0189018C8133
:10B4D000833039F0B9E0440F551F661F771FBA95C6
:10B4E000D1F79A01AB0168E1CE0166DE882311F045
:10B4F00086E01EC0A8016EEFCE01B4DF8823C9F03C
:10B5000068E572E0CE013EDE182F811102C087E1AE
:10B510000FC020E030E0A9016DE0CE014DDE8111C9
:10B5200006C09ADD811103C0CE01A2DD05C086E10F
:10B530008983CE019DDD10E0812FDF91CF911F9196
:10B540000F910895FC0165917591859194910895ED
:10B550002F923F924F925F926F927F928F929F9223
:10B56000AF92BF92CF92DF92EF92FF920F931F9311
:10B57000CF93DF9300D000D0CDB7DEB71C01FC0124
:10B58000ED5AF64B14919C01220F331F220F331FEB
:10B590003E832D8321553E4E4901F90110821182CF
:10B5A000128213822BEB31E147EB51E163EB71E146
:10B5B0008FEA91E10E944BD28D819E818E59964BEC
:10B5C000C1DF6B017C01612F772767FD7095872FA5
:10B5D000972F0E944FDD2B013C012D813E81265883
:10B5E0003E4E590120E030E040EC5FE3C701B60178
:10B5F0000E9482DFA30192010E9482DFF501608335
:10B600007183828393832D813E81215E344F3C83FD
:10B610002B83F90160817181828193816093E10ABA
:10B620007093E20A8093E30A9093E40A20E030E00A
:10B6300040E752E40E94B4DC2BE9C22E21E1D22E75
:10B640007B018C0126E831E142E851E16EE771E1CE
:10B650008AE791E10E9469C80E94D6C0F401108275
:10B660001182128213822BEB31E147EB51E163EB44
:10B6700071E18FEA91E10E944BD22D813E812A5ADD
:10B68000364B3A832983C9015DDF9058A3019201AB
:10B690000E9482DFF501608371838283938320E0BF
:10B6A00030E040E752E46091E10A7091E20A809153
:10B6B000E30A9091E40A0E94B4DC7B018C0126E845
:10B6C00031E142E851E16EE771E18AE791E10E94E0
:10B6D00069C80E94D6C089819A8134DF9B01AC0180
:10B6E0000E94D4DBA30192010E9482DFF5016083F6
:10B6F00071838283938320E030E040E05FE3EB815D
:10B70000FC8160817181828193810E9482DF6093DC
:10B71000E10A7093E20A8093E30A9093E40A20E03E
:10B7200030E040E752E40E94B4DC7B018C0126E863
:10B7300031E142E851E16EE771E18AE791E10E946F
:10B7400069C80E94D6C08D819E818259964BFADECF
:10B750000D811E810D551E4EF801208131814281DF
:10B7600053810E94D4DBF4016083718382839383CD
:10B770008D819E818A57964BE5DE2D813E812D5F1E
:10B78000344F7901F80120813181428153810E9437
:10B79000D4DBF70160837183828393838D819E81E3
:10B7A0008658964BCFDE2D813E812950354F790149
:10B7B000F80120813181428153810E94D4DBF7015D
:10B7C0006083718382839383F40180819181A2815C
:10B7D000B381F50180839183A283B3831092E10A40
:10B7E0001092E20A1092E30A1092E40A0E944FB902
:10B7F000F101E056FE4E81E0808326960FB6F89464
:10B80000DEBF0FBECDBFDF91CF911F910F91FF9093
:10B81000EF90DF90CF90BF90AF909F908F907F90F0
:10B820006F905F904F903F902F900895FC0124916E
:10B83000222341F03091C00035FFFCCF2093C60099
:10B840000196F4CF22E030E08BE295E10C9458B8F9
:10B85000FC012491222341F03091C00035FFFCCF40
:10B860002093C6000196F4CF2AE030E08BE295E108
:10B870000C94AEB72091CF0F3091D00F243031050A
:10B880000CF077C04091D10F5091D20F60E6649FC9
:10B890009001659F300D1124BC01C9018752904F62
:10B8A0000E944DE4E2E9F9E48491882341F090910B
:10B8B000C00095FFFCCF8093C6003196F5CFE09194
:10B8C000C011F0E0EE0FFF1FE45EFD4F0190F0812C
:10B8D000E02DEA5DFE4F0190F081E02D84918823F8
:10B8E00041F09091C00095FFFCCF8093C600319647
:10B8F000F5CF8091D10F9091D20F20E6289FF001D3
:10B90000299FF00D1124E752F04F8191882339F0DF
:10B910009091C00095FFFCCF8093C600F6CFE1E583
:10B92000F9E48491882341F09091C00095FFFCCF09
:10B930008093C6003196F5CF8091C00085FFFCCF83
:10B940008AE08093C6008091D10F9091D20F01962A
:10B9500064E070E00E9478E09093D20F8093D10F62
:10B960008091CF0F9091D00F01969093D00F80933C
:10B97000CF0F08952091CF0F3091D00F2430310593
:10B980000CF077C04091D10F5091D20F60E6649FC8
:10B990009001659F300D1124BC01C9018752904F61
:10B9A0000E94ADE3E2E9F9E48491882341F09091AB
:10B9B000C00095FFFCCF8093C6003196F5CFE09193
:10B9C000C011F0E0EE0FFF1FE45EFD4F0190F0812B
:10B9D000E02DEA5DFE4F0190F081E02D84918823F7
:10B9E00041F09091C00095FFFCCF8093C600319646
:10B9F000F5CF8091D10F9091D20F20E6289FF001D2
:10BA0000299FF00D1124E752F04F8191882339F0DE
:10BA10009091C00095FFFCCF8093C600F6CFEFE475
:10BA2000F9E48491882341F09091C00095FFFCCF08
:10BA30008093C6003196F5CF8091C00085FFFCCF82
:10BA40008AE08093C6008091D10F9091D20F019629
:10BA500064E070E00E9478E09093D20F8093D10F61
:10BA60008091CF0F9091D00F01969093D00F80933B
:10BA7000CF0F08959B9AA3980895FCDF40E052EC05
:10BA800061E070E08BE295E10E9466B6E9E4F9E4DA
:10BA90008491882341F09091C00095FFFCCF809362
:10BAA000C6003196F5CF8091C00085FFFCCF8AE0BB
:10BAB0008093C60022E939E4F9018491882341F09A
:10BAC0009091C00095FFFCCF8093C6003196F5CFD2
:10BAD00084B780FF20C0A091C011B0E0AA0FBB1FA7
:10BAE000A45EBD4FED91FC91E85DFE4F0190F081A9
:10BAF000E02D9491992341F04091C00045FFFCCF87
:10BB00009093C6003196F5CF9091C00095FFFCCF81
:10BB10009AE09093C60081FF20C0A091C011B0E0D0
:10BB2000AA0FBB1FA45EBD4FED91FC91E65DFE4FD9
:10BB30000190F081E02D9491992341F04091C00053
:10BB400045FFFCCF9093C6003196F5CF9091C00091
:10BB500095FFFCCF9AE09093C60082FF20C0A09191
:10BB6000C011B0E0AA0FBB1FA45EBD4FED91FC91C8
:10BB7000E45DFE4F0190F081E02D9491992341F016
:10BB80004091C00045FFFCCF9093C6003196F5CFA1
:10BB90009091C00095FFFCCF9AE09093C60083FF80
:10BBA00020C0A091C011B0E0AA0FBB1FA45EBD4F82
:10BBB000ED91FC91E25DFE4F0190F081E02D9491BA
:10BBC000992341F04091C00045FFFCCF9093C600FF
:10BBD0003196F5CF9091C00095FFFCCF9AE09093FD
:10BBE000C60085FF20C0A091C011B0E0AA0FBB1F06
:10BBF000A45EBD4FED91FC91E05DFE4F0190F081A0
:10BC0000E02D8491882341F09091C00095FFFCCFF6
:10BC10008093C6003196F5CF8091C00085FFFCCFA0
:10BC20008AE08093C60014BEE1E6FCE0849188239C
:10BC300041F09091C00095FFFCCF8093C6003196F3
:10BC4000F5CFE8E6FCE08491882341F09091C000B4
:10BC500095FFFCCF8093C6003196F5CF8091C00050
:10BC600085FFFCCF8AE08093C600F9018491E2E968
:10BC7000F9E4882349F09091C00095FFFCCF8093B0
:10BC8000C60031968491F5CFA091C011B0E0AA0F03
:10BC9000BB1FA45EBD4FED91FC91EC5CFE4F01908B
:10BCA000F081E02D8491882341F09091C00095FFB0
:10BCB000FCCF8093C6003196F5CFE4E3F9E484919C
:10BCC000882341F09091C00095FFFCCF8093C6007F
:10BCD0003196F5CFA091C011B0E0AA0FBB1FA45EB2
:10BCE000BD4FED91FC91EE5CFE4F0190F081E02D97
:10BCF0004491442341F05091C00055FFFCCF409344
:10BD0000C6003196F5CFEDE1F9E48491882341F046
:10BD10009091C00095FFFCCF8093C6003196F5CF7F
:10BD20008091C00085FFFCCF8AE08093C600E2E1ED
:10BD3000F9E48491882341F09091C00095FFFCCFF5
:10BD40008093C6003196F5CFE6E0F9E4849188232C
:10BD500041F09091C00095FFFCCF8093C6003196D2
:10BD6000F5CF8091C00085FFFCCF8AE08093C600AC
:10BD7000F9012491E2E9F9E4222349F08091C0001D
:10BD800085FFFCCF2093C60031962491F5CFE0913A
:10BD9000C011F0E0EE0FFF1FE45EFD4F0190F08157
:10BDA000E02DEA5CFE4F0190F081E02D8491882324
:10BDB00041F09091C00095FFFCCF8093C600319672
:10BDC000F5CF0E944AC44AE050E0BC018BE295E105
:10BDD0000E9482B7E091C011F0E0EE0FFF1FE45E19
:10BDE000FD4F0190F081E02DE85CFE4F0190F08165
:10BDF000E02D8491882341F09091C00095FFFCCF05
:10BE00008093C6003196F5CF4AE050E060ED74E0D3
:10BE10008BE295E10E9482B78091C00085FFFCCF44
:10BE20008AE08093C6001092D50F1092D60F109220
:10BE3000D70F1092D80F0E9489B40E945BB00E9465
:10BE40003A3D0E9419C80E9438C30E942998489917
:10BE500013C0FFEF23ED80E3F15020408040E1F775
:10BE600000C00000489911C06A9A729A0E946497B3
:10BE7000489BFECF729808959FEFE3EDF0E3915059
:10BE8000E040F040E1F700C0000008958091C90F44
:10BE90009091CA0F60E070E001960C9404E18091EB
:10BEA000C90F9091CA0F4AE050E060E070E001963F
:10BEB0000C946CE2682F772767FD70952091D30F63
:10BEC0003091D40F40E6429FC001439F900D112452
:10BED0008752904F0E9439E49093CA0F8093C90F04
:10BEE00021E0892B09F420E0822F08950E943ED79B
:10BEF0006093C50F7093C60F8093C70F9093C80FC0
:10BF000008950E943ED76093C50F7093C60F80932B
:10BF1000C70F9093C80FE091D30FF091D40FEB525D
:10BF2000F04F8081811121C0E091C011F0E0EE0F4F
:10BF3000FF1FE45EFD4F0190F081E02DE65CFE4FB7
:10BF40000190F081E02D8491882341F09091C00010
:10BF500095FFFCCF8093C6003196F5CF8091C0004D
:10BF600085FFFCCF8AE08093C60008958BE295E1BF
:10BF70000E94B8B6E091C011F0E0EE0FFF1FE45E42
:10BF8000FD4F0190F081E02DE659FE4F0190F081C8
:10BF9000E02D8491882341F09091C00095FFFCCF63
:10BFA0008093C6003196F5CF40915E1150915F119C
:10BFB00060916011709161114F5F5F4F6F4F7F4FC4
:10BFC0002AE030E08BE295E10E9457B78091C000F3
:10BFD00085FFFCCF8AE08093C60093CF8F929F921B
:10BFE000AF92BF92CF92DF92EF92FF920F931F9387
:10BFF000CF93DF93B8EEEB2EBCE0FB2E0FEA11E1FE
:10C00000CAE7D1E185ECC82E81E1D82EF7018191F4
:10C010007F0150DF882311F139DF4B015C01F6010C
:10C020008081811103C06091591101C061E070E00D
:10C0300080E090E00E944FDDF80120813181428153
:10C0400053810E9482DF9B01AC01C501B4010E94B3
:10C05000D4DB688379838A839B8309C0F80180815C
:10C060009181A281B38188839983AA83BB830C5F6A
:10C070001F4F2496FFEFCF1ADF0A8CEEE8168CE0F4
:10C08000F80621F686E416DF8823D1F0FFDE6B0187
:10C090007C0160936A1170936B1180936C11909383
:10C0A0006D1120E030E0A9010E94B0DE181644F4C2
:10C0B000C092E10AD092E20AE092E30AF092E40A26
:10C0C000DF91CF911F910F91FF90EF90DF90CF9074
:10C0D000BF90AF909F908F90089580DF89E4EADE53
:10C0E000882351F0D3DE60936E1170936F118093AB
:10C0F00070119093711108C010926E1110926F110F
:10C1000010927011109271118AE4D4DE882351F0DC
:10C11000BDDE6093721170937311809374119093CC
:10C12000751108951092721110927311109274117A
:10C13000109275110895CF92DF92EF92FF92CF93F4
:10C14000DF93EC01C090030BD090040BE090050B43
:10C15000F090060BA7019601688179818A819B8105
:10C160000E94ADDC87FF04C0C882D982EA82FB82CC
:10C17000C090070BD090080BE090090BF0900A0BD1
:10C18000A70196016C817D818E819F810E94ADDC2B
:10C1900087FF04C0CC82DD82EE82FF8220E030E0A7
:10C1A000A90160910B0B70910C0B80910D0B90917C
:10C1B0000E0B0E94D4DB6B017C019B01AC016885F6
:10C1C00079858A859B850E94ADDC87FF04C0C8867F
:10C1D000D986EA86FB86C090F70AD090F80AE090EC
:10C1E000F90AF090FA0AA7019601688179818A819B
:10C1F0009B810E94B0DE181624F4C882D982EA829C
:10C20000FB82C090FB0AD090FC0AE090FD0AF090FF
:10C21000FE0AA70196016C817D818E819F810E941B
:10C22000B0DE181624F4CC82DD82EE82FF82C0904C
:10C23000FF0AD090000BE090010BF090020BA701D9
:10C240009601688579858A859B850E94B0DE1816DF
:10C2500024F4C886D986EA86FB86DF91CF91FF90C9
:10C26000EF90DF90CF900895CF92DF92EF92FF9200
:10C270000F931F938AE791E15EDF0E943ED76093A0
:10C28000C50F7093C60F8093C70F9093C80F20916E
:10C290007A1130917B1140917C1150917D11609108
:10C2A000AF117091B0118091B1119091B2110E94B3
:10C2B000ADDC811179C020917E1130917F114091C8
:10C2C0008011509181116091B3117091B4118091DE
:10C2D000B5119091B6110E94ADDC811165C020E0CE
:10C2E00030E040E752E46091E10A7091E20A809107
:10C2F000E30A9091E40A0E94B4DC2BE9C22E21E10A
:10C30000D22E7B018C0126E831E142E851E16EE753
:10C3100071E18AE791E10E9469C880917A11909158
:10C320007B11A0917C11B0917D118093AF119093FE
:10C33000B011A093B111B093B21180917E11909180
:10C340007F11A0918011B09181118093B3119093CE
:10C35000B411A093B511B093B61180918211909150
:10C360008311A0918411B09185118093B71190939E
:10C37000B811A093B911B093BA1180918611909120
:10C380008711A0918811B09189118093BB1190936E
:10C39000BC11A093BD11B093BE111F910F91FF90DE
:10C3A000EF90DF90CF90089560911D0B70911E0B60
:10C3B000882777FD8095982F0E944FDD2091E10A14
:10C3C0003091E20A4091E30A5091E40A0E9482DF30
:10C3D00020E030E040E752E40E94B4DC20E030E0AE
:10C3E00048EC52E488CFCF92DF92EF92FF92CF9346
:10C3F000C62FE0919B11F0E0882309F4C2C0DF0151
:10C40000A956BE4E8C91811196C18091AF11909129
:10C41000B011A091B111B091B21180937A119093A3
:10C420007B11A0937C11B0937D118091B3119091F9
:10C43000B411A091B511B091B61180937E11909373
:10C440007F11A0938011B09381118091B7119091C9
:10C45000B811A091B911B091BA1180938211909343
:10C460008311A0938411B0938511C090BB11D0901B
:10C47000BC11E090BD11F090BE11C0928611D09217
:10C480008711E0928811F0928911EE0FFF1FEE0FD5
:10C49000FF1FE15FF44F2081318142815381662388
:10C4A00049F06091EF0A7091F00A8091F10A909141
:10C4B000F20A08C06091F30A7091F40A8091F50ABB
:10C4C0009091F60A0E94B4DC9B01AC01C701B60151
:10C4D0000E94D4DB6093BB117093BC118093BD119B
:10C4E0009093BE118BEB91E10E94F0D2C090E10AD3
:10C4F000D090E20AE090E30AF090E40A20E030E015
:10C5000040E752E46091EB0A7091EC0A8091ED0AE9
:10C510009091EE0A0E9482DF6093E10A7093E20A32
:10C520008093E30A9093E40AE0919B11F0E0E956CE
:10C53000FE4E81E0808398DE20919311309194111A
:10C5400040919511509196116091B7117091B81169
:10C550008091B9119091BA110E94D3DB6093B71109
:10C560007093B8118093B9119093BA112BEB31E10C
:10C5700047EB51E163EB71E18FEA91E10E944BD20D
:10C58000D1C0E956FE4E8081882309F4D4C0809141
:10C59000AF119091B011A091B111B091B2118093EF
:10C5A0007A1190937B11A0937C11B0937D118091AF
:10C5B000B3119091B411A091B511B091B6118093BF
:10C5C0007E1190937F11A0938011B093811160919F
:10C5D000B7117091B8118091B9119091BA1160930F
:10C5E0008211709383118093841190938511C09070
:10C5F000BB11D090BC11E090BD11F090BE11C09263
:10C600008611D0928711E0928811F09289112091C1
:10C6100093113091941140919511509196110E946F
:10C62000D4DB6093B7117093B8118093B9119093D4
:10C63000BA112BEB31E147EB51E163EB71E18FEA8A
:10C6400091E10E944BD2F0909B11CC2389F0209174
:10C650008B1130918C1140918D1150918E11609100
:10C66000EF0A7091F00A8091F10A9091F20A10C0DD
:10C6700020918F1130919011409191115091921110
:10C680006091F30A7091F40A8091F50A9091F60A8C
:10C690000E94D4DB24E0F29EF0011124E15FF44F0C
:10C6A00020813181428153810E94B4DC9B01AC0125
:10C6B0006091BB117091BC118091BD119091BE1120
:10C6C0000E94D3DB6093BB117093BC118093BD11AA
:10C6D0009093BE118BEB91E10E94F0D2C090E10AE1
:10C6E000D090E20AE090E30AF090E40A20E030E023
:10C6F00040E752E46091E70A7091E80A8091E90A04
:10C700009091EA0A0E9482DF6093E10A7093E20A44
:10C710008093E30A9093E40AE0919B11F0E0E956DC
:10C72000FE4E1082A1DDC092E10AD092E20AE092B0
:10C73000E30AF092E40ACF91FF90EF90DF90CF9060
:10C740000895AF92BF92CF92DF92EF92FF920F9334
:10C750001F93CF93DF93D82F2091721130917311D3
:10C76000409174115091751160916E1170916F111B
:10C7700080917011909171110E94BDDEC62F172F0C
:10C78000082FF92E60911D0B70911E0B882777FDE5
:10C790008095982F0E944FDD2091E10A3091E20AA6
:10C7A0004091E30A5091E40A0E9482DF20E030E0E9
:10C7B00040E752E40E94B4DC20E030E048EC52E470
:10C7C0000E94B4DC20919B112F93DF93FF920F9373
:10C7D0001F93CF935B016C0142E0E42E01E020E067
:10C7E0004EE651E16AE771E18FEA91E10E94634709
:10C7F00080917A1190917B11A0917C11B0917D1163
:10C800008093AF119093B011A093B111B093B21176
:10C8100080917E1190917F11A0918011B091811132
:10C820008093B3119093B411A093B511B093B61146
:10C830008091821190918311A0918411B091851102
:10C840008093B7119093B811A093B911B093BA1116
:10C850008091861190918711A0918811B0918911D2
:10C860008093BB119093BC11A093BD11B093BE11E6
:10C870000E943ED76093C50F7093C60F8093C70F79
:10C880009093C80F0F900F900F900F900F900F90F4
:10C89000DF91CF911F910F91FF90EF90DF90CF909C
:10C8A000BF90AF900895F8940E94DD3D179A1092C2
:10C8B000A011169A1092A111159A1092A211149A11
:10C8C00060E087E40E945ED6E8E9F9E48491882379
:10C8D00041F09091C00095FFFCCF8093C600319647
:10C8E000F5CFE091C011F0E0EE0FFF1FE45EFD4FC9
:10C8F0000190F081E02DEA59FE4F0190F081E02D8A
:10C900008491882341F09091C00095FFFCCF8093E3
:10C91000C6003196F5CF8091C00085FFFCCF8AE03C
:10C920008093C600E091C011F0E0EE0FFF1FE45EBF
:10C93000FD4F0190F081E02DE653FF4F8081918102
:10C940000E94C6977894C6E0D0E02197209749F0DE
:10C9500068EC70E080E090E00E946DD70E945598EE
:10C96000F4CFF894FFCF2F923F924F925F926F9245
:10C970007F928F929F92AF92BF92CF92DF92EF926F
:10C98000FF920F931F93CF93DF93CDB7DEB76E97D0
:10C990000FB6F894DEBF0FBECDBF30E6D32E44E015
:10C9A000E42EF12C5AE0C52EBB24B3948091AC1533
:10C9B0009091AD152091AE153091AF15821B930B60
:10C9C0008F779927892B09F467C28091CF0F9091B7
:10C9D000D00F04970CF060C28BE295E10E949CB6E8
:10C9E0008093CE0F2091CC0F3091CD0F8A3061F023
:10C9F0008D3051F08A3321F49091CB0F992321F09F
:10CA00002F3531050CF442C12115310509F45CC103
:10CA10008091D10F9091D20FD89E4001D99E900C59
:10CA20001124F401E20FF31FE752F04F108220911E
:10CA3000CB0F211126C11092CB0FFC01EB52F04F0E
:10CA4000108284010752104F6EE470E0C8010E940A
:10CA500039E40097F1F19093CA0F8093C90F801BBE
:10CA6000910B880D991D4AE050E060E070E086521D
:10CA7000904F0E946CE260936211709363118093F7
:10CA800064119093651140905E1150905F11609019
:10CA90006011709061112FEF421A520A620A720AF5
:10CAA0000091D10F1091D20F641575058605970579
:10CAB00009F40DC1D09EC001D19E900D11246DEFDF
:10CAC00078E48752904F0E94E4E3892B09F0FFC07D
:10CAD000A9C16AE270E0C8010E9439E4892B09F417
:10CAE00051C0E8E9F9E48491882341F09091C000B5
:10CAF00095FFFCCF8093C6003196F5CFE091C01131
:10CB0000F0E0EE0FFF1FE45EFD4F0190F081E02D9D
:10CB1000EC5BFE4F0190F081E02D8491882341F081
:10CB20009091C00095FFFCCF8093C6003196F5CF61
:10CB300040915E1150915F1160916011709161118F
:10CB40002AE030E08BE295E10E9457B78091C00067
:10CB500085FFFCCF8AE08093C6001092CD0F109223
:10CB6000CC0F0DC38091621190916311A09164115B
:10CB7000B091651180935E1190935F11A093601145
:10CB8000B09361118091D10F9091D20FD89E800106
:10CB9000D99E100D1124C8018752904F4C0167E4B3
:10CBA00070E00E9439E4009709F447C09093CA0FDF
:10CBB0008093C90F88199909800F911F60E070E078
:10CBC0008652904F0E9404E10E941CDD6430710582
:10CBD000A0F58091B70F882381F1E091C011F0E0BA
:10CBE000EE0FFF1FE45EFD4F0190F081E02DE8594C
:10CBF000FE4F0190F081E02D8491882341F09091C7
:10CC0000C00095FFFCCF8093C6003196F5CF809190
:10CC1000C00085FFFCCFC092C600E091C011F0E0DB
:10CC2000EE0FFF1FE45EFD4F0190F081E02DE45315
:10CC3000FF4F808191810E94B9970091D10F10918F
:10CC4000D20FD09EC001D19E900D11246EE67CE0E3
:10CC50008752904F0E9444E4892B09F424DEC801D6
:10CC60000196B7010E9478E09093D20F8093D10F84
:10CC70008091CF0F9091D00F01969093D00F809319
:10CC8000CF0F1092CD0F1092CC0F90CE8B3311F4AA
:10CC9000B092CB0F9091CB0F911188CE4091D10FD4
:10CCA0005091D20FB9016F5F7F4F7093CD0F60939A
:10CCB000CC0FD49EF001D59EF00D1124E20FF31F8E
:10CCC000E752F04F808372CE1092CB0F58C2D09EA5
:10CCD0004001D19E900C1124C4018752904F3C0119
:10CCE0006AE270E00E9439E4009709F03EC0E8E98A
:10CCF000F9E48491882341F09091C00095FFFCCF26
:10CD00008093C6003196F5CFE091C011F0E0EE0FB0
:10CD1000FF1FE45EFD4F0190F081E02DEE5BFE4FC2
:10CD20000190F081E02D8491882341F09091C00022
:10CD300095FFFCCF8093C6003196F5CF40915E11F0
:10CD400050915F1160916011709161112AE030E0A3
:10CD50008BE295E10E9457B78091C00085FFFCCF20
:10CD60008AE08093C60002D9F8CE20E010E0F401FA
:10CD7000E20FF11DE752F04F30813A3219F02F5F88
:10CD80001327F5CF9093CA0F8093C90F861997097F
:10CD9000880D991D60E070E08652904F0E9404E17A
:10CDA0000E941CDD212F30E02617370709F4DACE68
:10CDB000E8E9F9E48491882341F09091C00095FF5F
:10CDC000FCCF8093C6003196F5CFE091C011F0E022
:10CDD000EE0FFF1FE45EFD4F0190F081E02DE05C5F
:10CDE000FE4F0190F081E02D8491882341F09091D5
:10CDF000C00095FFFCCF8093C6003196F5CF4091DF
:10CE00005E1150915F1160916011709161112AE083
:10CE100030E08BE295E10E9457B78091C00085FF1A
:10CE2000FCCF9ECFE8E9F9E48491882341F090910A
:10CE3000C00095FFFCCF8093C6003196F5CFE091FE
:10CE4000C011F0E0EE0FFF1FE45EFD4F0190F08196
:10CE5000E02DE25CFE4F0190F081E02D849188236B
:10CE600041F09091C00095FFFCCF8093C6003196B1
:10CE7000F5CF40915E1150915F11609160117091FA
:10CE800061112AE030E08BE295E10E9457B7809172
:10CE9000C00085FFFCCF64CF8091D111882309F4B5
:10CEA0006EC18091CC0F9091CD0F892B09F067C195
:10CEB0008091CF0F9091D00F892B11F41092B50F64
:10CEC000F8EE2F2EF3E03F2E412C512CACE3CA2E6E
:10CED000D12CE12CF12C8E010F5F1F4FE0E66E2E5E
:10CEE0007724739440916C1450916D1460916E147A
:10CEF00070916F148091641490916514A0916614E0
:10CF0000B0916714481759076A077B0708F037C1C3
:10CF10008091CF0F9091D00F04970CF030C1809189
:10CF2000B50F81112CC18091BF139091C013A091B6
:10CF3000C113B091C21380936C1490936D14A0939D
:10CF40006E14B0936F1487EB93E10E94782E482FF4
:10CF50008093CE0F8A30B9F04D30A9F0433229F4D6
:10CF60002091CB0F222379F002C04A33C9F32091DC
:10CF7000CC0F3091CD0F2F3531052CF48F3FAFEF13
:10CF80009A0709F0DEC040916C1450916D146091C5
:10CF90006E1470916F148091641490916514A09137
:10CFA0006614B0916714481759076A077B0708F49D
:10CFB0008EC0E091C011F0E0EE0FFF1FE45EFD4F68
:10CFC0000190F081E02DEA5BFE4F0190F081E02DB1
:10CFD0008491882341F09091C00095FFFCCF80930D
:10CFE000C6003196F5CF8091C00085FFFCCFBAE036
:10CFF000B093C6000E943ED76093B90F7093BA0FEA
:10D000008093BB0F9093BC0F8090BD0F9090BE0F8C
:10D01000A090BF0FB090C00F681979098A099B09C9
:10D02000A20191010E948BE049015A01CA01B90194
:10D03000A70196010E948BE0CA01B901A7019601E0
:10D040000E948BE07F936F93C501B40120E13EE025
:10D0500040E050E00E948BE03F932F93A9EEB8E4AC
:10D06000BF93AF931F930F930E9471E4E2E9F9E439
:10D0700084910FB6F894DEBF0FBECDBF882349F070
:10D080009091C00095FFFCCF8093C60031968491AB
:10D09000F5CFF8018191882339F09091C00095FF78
:10D0A000FCCF8093C600F6CF8091C00085FFFCCFF7
:10D0B0003AE03093C600C8010E9489978FEC91E155
:10D0C0000E94D55761E08FEC91E10E9498518091C8
:10D0D000CE0F833211F47092B50F2091CC0F3091A6
:10D0E000CD0F2115310509F4EFCD8091D10F90912D
:10D0F000D20F689EF001699EF00D1124E20FF31F1C
:10D10000E752F04F1082FC01EB52F04F70822091F9
:10D11000CF0F3091D00F2F5F3F4F3093D00F209320
:10D12000CF0F019664E070E00E9478E09093D20FF8
:10D130008093D10F1092CB0F1092CD0F1092CC0F85
:10D14000D1CE4B3311F47092CB0F4091CB0F4111E4
:10D15000C5CE4091D10F5091D20FB9016F5F7F4F73
:10D160007093CD0F6093CC0F649EF001659EF00D1F
:10D170001124E20FF31FE752F04F8083B3CE6E9677
:10D180000FB6F894DEBF0FBECDBFDF91CF911F91D8
:10D190000F91FF90EF90DF90CF90BF90AF909F9056
:10D1A0008F907F906F905F904F903F902F90089559
:10D1B000CF92DF92EF92FF920F931F93CF93C82FDE
:10D1C0008091CF0F9091D00F03970CF4CCDB0E948D
:10D1D0003ED70091C10F1091C20F2091C30F309123
:10D1E000C40FC090C50FD090C60FE090C70FF0904D
:10D1F000C80F6C197D098E099F09061717072807A4
:10D20000390728F4012B022B032B09F04CDB40914A
:10D21000DD0A5091DE0A6091DF0A7091E00A452B29
:10D22000462B472B19F10E943ED70091C50F109154
:10D23000C60F2091C70F3091C80F601B710B820B76
:10D24000930B0091DD0A1091DE0A2091DF0A3091E4
:10D25000E00A061717072807390740F49091FD15D3
:10D260008091FC15981302C0CC2349F0CF911F91F7
:10D270000F91FF90EF90DF90CF900C944DC8179ACC
:10D280001092A011169A1092A111159A1092A21143
:10D29000149AECCF0E94DD3D8091B70F811151C0EF
:10D2A00081E08093B70F80915E1190915F11A09102
:10D2B0006011B091611180935A1190935B11A0930A
:10D2C0005C11B0935D11E8E9F9E48491882341F0A1
:10D2D0009091C00095FFFCCF8093C6003196F5CFAA
:10D2E000E091C011F0E0EE0FFF1FE45EFD4F0190F2
:10D2F000F081E02DE859FE4F0190F081E02D8491FE
:10D30000882341F09091C00095FFFCCF8093C60028
:10D310003196F5CF8091C00085FFFCCF8AE08093E5
:10D32000C600E091C011F0E0EE0FFF1FE45EFD4F7C
:10D330000190F081E02DE453FF4F808191810C94A6
:10D34000B99708958091B70F0895CF93DF93EC01BB
:10D3500080919B118093B80F84E50E945A5F8111E0
:10D3600002C080E0B8C00E94465F0E9421DD609349
:10D37000B80F6623B1F3E2E9F9E48491882341F020
:10D380009091C00095FFFCCF8093C6003196F5CFF9
:10D39000CD36D10509F454C0BCF4C836D10561F1CD
:10D3A000C936D10509F087C0E091C011F0E0EE0F59
:10D3B000FF1FE45EFD4F0190F081E02DE25BFE4F28
:10D3C0000190F081E02D38C0CA3DD10509F451C06B
:10D3D000CD3DD10509F06FC0E091C011F0E0EE0F36
:10D3E000FF1FE45EFD4F0190F081E02DEC5AFE4FEF
:10D3F0000190F081E02D5CC0E091C011F0E0EE0FF3
:10D40000FF1FE45EFD4F0190F081E02DE45BFE4FD5
:10D410000190F081E02D8191882309F44CC0909116
:10D42000C00095FFFCCF8093C600F5CF9091C0005F
:10D4300095FFFCCF8093C60081918111F7CF3BC04F
:10D44000E091C011F0E0EE0FFF1FE45EFD4F019090
:10D45000F081E02DE85AFE4F0190F081E02D81919E
:10D46000882349F19091C00095FFFCCF8093C600BE
:10D47000F6CFE091C011F0E0EE0FFF1FE45EFD4F2C
:10D480000190F081E02DEE5AFE4F0190F081E02DE9
:10D490008191882381F09091C00095FFFCCF80930B
:10D4A000C600F6CF9091C00095FFFCCF8093C600D8
:10D4B00081918111F7CF40E050E06091B80F8BE28D
:10D4C00095E10E94B9B78091C00085FFFCCF8AE04A
:10D4D0008093C60081E0DF91CF910895CF92DF92D3
:10D4E000EF92FF922091BF112223F1F020E030E073
:10D4F00040E05FE30E9482DF6B017C0120E030E0CE
:10D50000A9010E94ADDC882379F0A7019601C7012B
:10D51000B6010E9482DF2BED3FE049E450E40E9417
:10D5200082DF9B01AC0104C020E030E040E85FE313
:10D5300060E070E080E89FE30E94B4DCFF90EF9031
:10D54000DF90CF9008956091130B7091140B809130
:10D55000150B9091160BC2DF60930F0B7093100B9D
:10D560008093110B9093120B08953F924F925F920C
:10D570006F927F928F929F92AF92BF92CF92DF92E3
:10D58000EF92FF920F931F93CF93DF93CDB7DEB748
:10D59000E9970FB6F894DEBF0FBECDBF81E40E94BD
:10D5A0005A5F882309F44CC082E70E945A5F88239F
:10D5B000A9F0E3E7FCE08191882339F09091C00065
:10D5C00095FFFCCF8093C600F6CF8091C00085FF09
:10D5D000FCCF8AE08093C6000C94778386E70E9494
:10D5E0005A5F8823A9F0E9E7FCE08191882339F0AC
:10D5F0009091C00095FFFCCF8093C600F6CF80913C
:10D60000C00085FFFCCF8AE08093C6000C9477832E
:10D6100087E60E945A5F882321F00E9464970C9449
:10D6200077838AE70E945A5F882311F40C947783EA
:10D6300060E070E089EF9FE00E941C940C94778377
:10D6400087E40E945A5F882309F46EC20E94465FF5
:10D650000E941CDD6A30710509F4BBC09CF4623085
:10D66000710509F44CC024F477FF25C00C9477832E
:10D670006330710509F44EC06430710509F455C07A
:10D680000C9477836A35710509F4FAC154F46B3050
:10D69000710509F4A4C06C31710509F4A6C00C949D
:10D6A00077836B35710509F4EFC16C35710509F4A9
:10D6B000F0C10C9477838091B70F81110C9477831C
:10D6C0000E94EE5F809198118823A9F088E50E945E
:10D6D0005A5F811110C089E50E945A5F81110BC009
:10D6E0008AE50E945A5F811106C085E40E945A5F54
:10D6F00081110C947A830E9434610C947783809119
:10D70000B70F81110C9477830E946D6081E019D866
:10D710000C9477838091B70F81110C9477830E94CA
:10D720006D6080E00ED80C947783E091C011F0E03A
:10D73000EE0FFF1FE45EFD4F0190F081E02DE054FD
:10D74000FF4F808191810E94B99780E50E945A5FC6
:10D75000882339F00E94465F0E9421DD4B015C0165
:10D7600003C0812C912C540183E50E945A5F8823C9
:10D7700061F00E94465F20E030E04AE754E40E94F6
:10D7800082DF0E9421DD4B015C010E94D6C00E9415
:10D790003ED76B017C01C80CD91CEA1CFB1C0E9403
:10D7A0003ED76093C50F7093C60F8093C70F9093B9
:10D7B000C80F0E943ED76C157D058E059F0510F0A1
:10D7C0000C9477830E940A3B80E0F2DC0E9455981B
:10D7D000F0CF60E081E00E94F3610C94778360E019
:10D7E00080E00E94F3610C9477838091E10A90912C
:10D7F000E20AA091E30AB091E40A80936611909343
:10D800006711A0936811B093691180911D0B9091DD
:10D810001E0B9093C4118093C31184E690E0909303
:10D820001E0B80931D0B0E943ED76093C50F709313
:10D83000C60F8093C70F9093C80F81E00E9456B91E
:10D840008091AF119091B011A091B111B091B2112E
:10D8500080937A1190937B11A0937C11B0937D11EA
:10D860008091B3119091B411A091B511B091B611FE
:10D8700080937E1190937F11A0938011B0938111BA
:10D880008091B7119091B811A091B911B091BA11CE
:10D890008093821190938311A0938411B09385118A
:10D8A0008091BB119091BC11A091BD11B091BE119E
:10D8B0008093861190938711A0938811B09389115A
:10D8C0001092E10A1092E20A1092E30A1092E40A1E
:10D8D00088E50E945A5F882311F090E00AC089E52C
:10D8E0000E945A5F8111F9CF8AE50E945A5F91E048
:10D8F00098279093E50A91110C94A98388E50E94DA
:10D900005A5F81110C94A9838091E50A81110C94CE
:10D91000AF8389E50E945A5F81110C94AF8388E53B
:10D920000E945A5F8823D1F00E944F5F672B682BBB
:10D93000692BA1F00E94465F2091A3113091A411A0
:10D940004091A5115091A6110E94D4DB6093AF11B4
:10D950007093B0118093B1119093B21189E50E9438
:10D960005A5F8823D1F00E944F5F672B682B692B89
:10D97000A1F00E94465F2091A7113091A81140911B
:10D98000A9115091AA110E94D4DB6093B311709336
:10D99000B4118093B5119093B6118091E50A81116D
:10D9A0000C94B5838AE50E945A5F81110C94B5836B
:10D9B0008AE50E945A5F8823D1F00E944F5F672B4F
:10D9C000682B692BA1F00E94465F2091AB1130912A
:10D9D000AC114091AD115091AE110E94D4DB609317
:10D9E000B7117093B8118093B9119093BA112BEBC2
:10D9F00031E147EB51E163EB71E18FEA91E10E9484
:10DA00004BD280E00E9456B98091661190916711C7
:10DA1000A0916811B09169118093E10A9093E20A94
:10DA2000A093E30AB093E40A8091C3119091C411CA
:10DA300090931E0B80931D0B0E943ED76093C50FE1
:10DA40007093C60F8093C70F9093C80F0E944FB971
:10DA50008091D111882311F40C9477836DEC71E1DE
:10DA600089EF9FE00E942D948091CD119091CE116D
:10DA7000892B11F40C9477830E94C9AA0C947783A4
:10DA8000109259110C94778381E0809359110C9472
:10DA9000778385E40E945A5F811102C00E94D6C03C
:10DAA00098EEC92E9CE0D92E23EAE22E21E1F22E37
:10DAB0000FEA11E1B12CF60181916F010E945A5FCA
:10DAC000882339F1F3E0BF120CC00E94465FF801D1
:10DAD00060837183828393838BEB91E10E94F0D208
:10DAE00018C00E94465FF701208131814281538135
:10DAF0000E94D4DBF80160837183828393832BEBD4
:10DB000031E147EB51E163EB71E18FEA91E10E9472
:10DB10004BD2B394F4E0EF0EF11C0C5F1F4F24E0E6
:10DB2000B212C9CF0C9477838DE40E945A5F882388
:10DB300011F40C947E820E94465F0E941CDD6537C2
:10DB4000710511F40C949B760CF0D0C06032710515
:10DB500009F44EC30CF071C06731710509F4A3C21A
:10DB60000CF044C06231710511F40C94BF751CF5C2
:10DB700077FF02C00C947783623071050CF498C172
:10DB80006131710511F00C947783E091C011F0E0E0
:10DB9000EE0FFF1FE45EFD4F0190F081E02DE85392
:10DBA000FF4F808191810E94B99717981698159818
:10DBB00014980C9477836531710509F468C20CF0F0
:10DBC0006CC26431710511F00C947783E091C0113F
:10DBD000F0E0EE0FFF1FE45EFD4F0190F081E02DBD
:10DBE000E85BFE4F0190F081E02D20C26B317105A2
:10DBF00009F485C2B4F46931710509F46CC20CF002
:10DC000070C28FEC91E10E94804E0E943ED76093DB
:10DC1000BD0F7093BE0F8093BF0F9093C00F0C94F5
:10DC200077836E31710509F4A5C20CF07DC36C31A8
:10DC3000710509F46AC20C9477836C35710509F497
:10DC4000ECC7ECF46235710509F490C764F46035F3
:10DC5000710509F443C70CF058C76A32710509F41D
:10DC6000C1C30C9477836435710509F488C70CF43B
:10DC700081C76535710509F4B5C70C9477836B3698
:10DC8000710509F425C764F46936710509F422C4E5
:10DC90000CF0EEC66836710509F4EBC30C9477837B
:10DCA0006037710509F403C434F46D36710509F465
:10DCB0001EC50C9477836237710511F40C94AF760E
:10DCC0006337710511F00C947783E091C011F0E097
:10DCD000EE0FFF1FE45EFD4F0190F081E02DEE5945
:10DCE000FE4F0190F081E02D0C949676623E710516
:10DCF00011F40C94FD7B0CF05FC06B3C710511F4CA
:10DD00000C943C7AACF56C38710509F4D2C304F577
:10DD10006837710511F40C949C776937710511F41B
:10DD20000C94A1776737710511F00C947783E0911B
:10DD3000C011F0E0EE0FFF1FE45EFD4F0190F08197
:10DD4000E02DE258FE4F0190F081E02D0C94AD776C
:10DD5000683C710511F40C949979693C710511F4D2
:10DD60000C941B7A6E3B710511F00C94778355C5AA
:10DD70006F3C710511F40C94F97A54F46D3C710503
:10DD800011F40C947B7A14F40C94597A0C94DB7A89
:10DD9000613D710511F40C94587B14F40C94307BA4
:10DDA0006C3D710511F40C94C87B6D3D710511F447
:10DDB0000C94D77B0C947783653F31E0730711F4A3
:10DDC0000C94AA7D54F56F3291E0790711F40C940C
:10DDD0006F7D84F46D32F1E07F0711F40C948E7C3A
:10DDE00014F00C94617D6C32714011F40C94587CE9
:10DDF0000C9477836F3581E0780711F40C942282BC
:10DE0000603991E0790711F40C94A77D6E3571406B
:10DE100011F00C9477830C94EB816835F2E07F0766
:10DE200011F40C94F27EA4F4673F31E0730711F40F
:10DE30000C94B27D14F40C94AF7D6D3F714011F0E1
:10DE40000C9477830E946497E2E9F9E40C94BC7D1A
:10DE50006B38E3E07E0711F40C94C5813CF4633524
:10DE6000734011F40C94CD7D0C947783603A33E0C9
:10DE7000730709F426C2673E734011F00C94778350
:10DE80001092B70F0E94CC9780915A1190915B111C
:10DE9000A0915C11B0915D1180935E1190935F1120
:10DEA000A0936011B09361110E94B65F0C947783C8
:10DEB0000091C90F1091CA0F0E5F1F4F80E50E949D
:10DEC0005A5F882379F00E94465F0E9421DD6B0132
:10DED0007C01BB24B394611571058105910531F472
:10DEE000B12C04C0B12CC12CD12C760183E50E9449
:10DEF0005A5F882399F00E94465F20E030E04AE7AD
:10DF000054E40E9482DF0E9421DD6B017C01AA247F
:10DF1000A394611571058105910509F4A12C6AE2AC
:10DF200070E0C8010E9439E4009711F0FC011082F2
:10DF3000F801CF0121912032E1F3B11007C0A11007
:10DF400005C0222319F00E94899710C0E091C011EA
:10DF5000F0E0EE0FFF1FE45EFD4F0190F081E02D39
:10DF6000EE53FF4F808191810E94B99781E00E941A
:10DF700069970E94D6C00E943ED76093C50F7093E8
:10DF8000C60F8093C70F9093C80FC114D104E1044A
:10DF9000F104A9F00E943ED74B015C018C0C9D1C42
:10DFA000AE1CBF1C0E943ED7681579058A059B05EB
:10DFB000B8F40E943D99811113C00C94BB830E9458
:10DFC0003B99882311F40C9477830E943D99811129
:10DFD0000AC00E940A3B80E0EBD80E945598F5CF1A
:10DFE00080E00E9469978091D111E091C011F0E02A
:10DFF000EE0FFF1FE45EFD4F0190F081E02D8823BE
:10E0000041F0EC53FF4F808191810E94B9970C94AD
:10E010007783808191810E94B9970C947783909146
:10E02000C00095FFFCCF8093C6003196849181118A
:10E03000F6CF8091C00085FFFCCF8AE08093C600B8
:10E040008FEC91E10E94284DE091C011F0E0EE0FBD
:10E05000FF1FE45EFD4F0190F081E02DE65BFE4F77
:10E060000190F081E02D8491882341F09091C000CF
:10E0700095FFFCCF8093C6003196F5CF8091C0000C
:10E0800085FFFCCF8AE08093C6000C9477838FECE9
:10E0900091E10E947D4D0C9477838FEC91E10E9479
:10E0A0007C4E0C9477830091C90F1091CA0F0C5FBE
:10E0B0001F4F6AE270E0C8010E9439E4009711F036
:10E0C000FC01108221E041E0B8018FEC91E10E9457
:10E0D000FE520C9477838FEC91E10E94874E0C9452
:10E0E00077838091D211882311F40C94778383E590
:10E0F0000E945A5F81110C94C4830C9477838FEC37
:10E1000091E10E942B500C9477838091C90F9091DC
:10E11000CA0F6AE270E004960E9439E48C0100970D
:10E12000D9F02091D30F3091D40F40E6429FC00127
:10E13000439F900D11246EE470E08752904F0E942F
:10E1400039E460E270E00E9439E401969093CA0FCE
:10E150008093C90FF80110826091C90F7091CA0FA6
:10E160006C5F7F4F21E040E08FEC91E10E94FE5216
:10E170000C9477838091D211882311F40C947783C7
:10E1800060E08FEC91E10E948E528091C90F9091D6
:10E19000CA0F6AE270E004960E9439E48C0100978D
:10E1A000D9F02091D30F3091D40F40E6429FC001A7
:10E1B000439F900D11246EE470E08752904F0E94AF
:10E1C00039E460E270E00E9439E401969093CA0F4E
:10E1D0008093C90FF80110826091C90F7091CA0F26
:10E1E0006C5F7F4F8FEC91E10E94EB4E0C94778334
:10E1F0008091D11181110E94D6C00091C90F109158
:10E20000CA0F0C5F1F4F6AE270E0C8010E9439E438
:10E210007C0161E270E0C8010E9439E4009719F0C6
:10E220008C010F5F1F4FE114F10411F0F701108210
:10E2300080E50E945A5FF82E2091C90F3091CA0FD5
:10E240000217130708F4F12C8091D211882311F4DE
:10E250000C94778321E02F2541E0B8018FEC91E108
:10E260000E94FE5283E50E945A5F8823B9F02091F4
:10E27000C90F3091CA0F2017310780F40E944F5FF9
:10E28000AB01BC0140936C1450936D1460936E14F9
:10E2900070936F1487EB93E10E94412F8FEC91E113
:10E2A0000E94804EF1100C9477830E943ED76093B9
:10E2B000BD0F7093BE0F8093BF0F9093C00F0C944F
:10E2C00077838091C90F9091CA0F6AE270E005963A
:10E2D0000E9439E48C010097D9F02091D30F30913E
:10E2E000D40F40E6429FC001439F900D11246EE47D
:10E2F00070E08752904F0E9439E460E270E00E9423
:10E3000039E401969093CA0F8093C90FF8011082E7
:10E310006091C90F7091CA0F6B5F7F4F8FEC91E1D5
:10E320000E9483560C9477830E943ED76093B90F66
:10E330007093BA0F8093BB0F9093BC0F0091BD0FE9
:10E340001091BE0F2091BF0F3091C00F601B710B59
:10E35000820B930B28EE33E040E050E00E948BE00C
:10E36000CA01B9012CE330E040E050E00E948BE0AC
:10E370007F936F933F932F938AED98E49F938F93AE
:10E38000CE0101969F938F930E9471E4E2E9F9E434
:10E3900084910FB6F894DEBF0FBECDBF882349F03D
:10E3A0009091C00095FFFCCF8093C6003196849178
:10E3B000F5CFFE0131968191882339F09091C0000C
:10E3C00095FFFCCF8093C600F6CF8091C00085FFFB
:10E3D000FCCF8AE08093C600CE0101960E94899707
:10E3E0000C94778383E50E945A5F882311F40C9480
:10E3F00077830E94465F0E941CDDF62EE72E862F53
:10E400009E2D8C0180E50E945A5F882331F00F3FDA
:10E41000110509F010F40C94D5830DE010E0E0EB49
:10E42000FCE0819191918017910711F40C9477830E
:10E430003CE0E83EF307A9F70630110539F48F2DCB
:10E440009E2D90939A118093991104C017FF02C0DA
:10E450000C94778361E0802F0E945ED66F2D802F11
:10E460000E9497D66F2D7E2D802F0E9454D50C943C
:10E47000778388E690E00E94A56981110C947783E8
:10E4800083E50E945A5F882371F00091B80F0E94C3
:10E49000465F10E0000F111F0256104F0E941CDD56
:10E4A000F801718360830E94DC3D0C9477830E94A5
:10E4B000536483E50E945A5F882311F40C94778398
:10E4C0000E94465F0E941CDD70939D0F60939C0F1D
:10E4D0000C94778389E690E00E94A56981110C94E1
:10E4E0007783E4EDF8E48491882341F09091C000B3
:10E4F00095FFFCCF8093C6003196F5CFE091B80F21
:10E5000024E0E29FF0011124EA56F04F408151814E
:10E510006281738121E030E08BE295E10E9458B87E
:10E52000E1EDF8E48491882341F09091C00095FFDB
:10E53000FCCF8093C6003196F5CFE091B80FF0E0A4
:10E54000EE0FFF1FE256F04F60817181882777FD43
:10E550008095982F0E944FDDAB01BC0121E030E097
:10E560008BE295E10E9458B8EDECF8E484918823A1
:10E5700041F09091C00095FFFCCF8093C60031968A
:10E58000F5CF4091900F5091910F6091920F709143
:10E59000930F21E030E08BE295E10E9458B8EAEC5D
:10E5A000F8E48491882341F09091C00095FFFCCF5E
:10E5B0008093C6003196F5CF60919C0F70919D0FAE
:10E5C000882777FD8095982F0E944FDDAB01BC0115
:10E5D00021E030E08BE295E10E9458B8E7ECF8E4E6
:10E5E0008491882341F09091C00095FFFCCF8093E7
:10E5F000C6003196F5CF4AE050E060E070E08BE273
:10E6000095E10E9482B7E5ECF8E48491882341F01B
:10E610009091C00095FFFCCF8093C6003196F5CF56
:10E620004091960F5091970F6091980F7091990FAC
:10E6300021E030E08BE295E10E9458B8E2ECF8E48A
:10E640008491882341F09091C00095FFFCCF809386
:10E65000C6003196F5CF60919E0F70919F0F88276D
:10E6600077FD8095982F0E944FDDAB01BC0121E022
:10E6700030E08BE295E10E9458B8EEEBF8E484912B
:10E68000882341F09091C00095FFFCCF8093C60095
:10E690003196F5CF8091B80F90E00E94D43A4AE0CD
:10E6A00050E0BC018BE295E10E9482B7E9EBF8E40F
:10E6B0008491882341F09091C00095FFFCCF809316
:10E6C000C6003196F5CF8FEF9FEF0E94D43A4AE013
:10E6D00050E0BC018BE295E10E9482B78091C000BE
:10E6E00085FFFCCF8AE08093C6000C9445858DE6BB
:10E6F00090E00E94A56981110C947783E091C0118C
:10E70000F0E0EE0FFF1FE45EFD4F0190F081E02D81
:10E71000E65AFE4F808191810E94B99783E50E945D
:10E720005A5F882391F00091B80F0E94465F10E075
:10E73000000F111F0256104F0E941CDDF80171835B
:10E74000608381E08093DC0A15C082E50E945A5FF5
:10E75000882381F00091B80F0E94465F10E0000FFF
:10E76000111F0256104F0E941CDDF8017183608357
:10E770001092DC0A0E94DC3D0E943ED74B015C01F6
:10E780000091B80F10E0F801EE0FFF1FE256F04FB6
:10E7900060817181882777FD8095982F0E944FDDD9
:10E7A000F801EE0FFF1FEE0FFF1FEA56F04F11E0CA
:10E7B00020813181428153810E94B0DE18160CF015
:10E7C00010E01093B60F10928A11CC24CA94DC2C5E
:10E7D0007601F8EE4F2EF3E05F2E612C712CAAE04B
:10E7E0003A2E80918A1181110C94F084FFEFCF169C
:10E7F000DF06EF06FF0611F40C94DC83F7FE02C07F
:10E800000C94F0840E943ED76C197D09683B7B40D4
:10E8100010F40C94DC830C94F084E091C011F0E0CF
:10E82000EE0FFF1FE45EFD4F0190F081E02DE25AF4
:10E83000FE4F808191810E94B99783E50E945A5FC3
:10E84000882361F00E94465F0E941CDD70939D0F3B
:10E8500060939C0F81E08093DC0A0FC082E50E94E8
:10E860005A5F882351F00E94465F0E941CDD70931E
:10E870009D0F60939C0F1092DC0A0E943ED74B01C3
:10E880005C0110928A1160919C0F70919D0F8827F6
:10E8900077FD8095982F0E944FDD11E02091900F19
:10E8A0003091910F4091920F5091930F0E94B0DEE2
:10E8B00018160CF010E01093B60F0BEA18E487EA74
:10E8C000E82E88E4F82E93EAC92E98E4D92E2AE09F
:10E8D000722E8091B60F60919C0F70919D0F8823CE
:10E8E00009F48BC080918A11811187C0882777FD38
:10E8F0008095982F0E944FDD2091900F3091910FBD
:10E900004091920F5091930F0E94B0DE18160CF0B8
:10E910008BC00E943ED7681979098A099B09693E14
:10E9200073408105910508F460C0E0919B1184E07B
:10E93000E89FF0011124EA56F04F40815181628135
:10E940007381F8018491EBEAF8E4882349F090910F
:10E95000C00095FFFCCF8093C60031968491F5CF1F
:10E9600022E030E08BE295E10E9458B8F7018491F3
:10E97000E7EAF8E4882349F09091C00095FFFCCFC6
:10E980008093C60031968491F5CF60919B1170E021
:10E990004AE050E08BE295E10E9482B7F601849153
:10E9A000E3EAF8E4882349F09091C00095FFFCCF9A
:10E9B0008093C60031968491F5CF4091900F50918D
:10E9C000910F6091920F7091930F21E030E08BE2F4
:10E9D00095E10E9458B88091C00085FFFCCF7092ED
:10E9E000C6000E943ED74B015C010E940A3B80E0BA
:10E9F0000E94D8680E9455986CCF882777FD809533
:10EA0000982F0E944FDD2091900F3091910F4091EF
:10EA1000920F5091930F0E94ADDC87FF05C080914B
:10EA2000DC0A882309F475CFE091C011F0E0EE0F05
:10EA3000FF1FE45EFD4F0190F081E02DE05AFE4F94
:10EA4000808191810E94B9978091D111882321F012
:10EA50008CE49CE00E9489970E943ED76093C50F8A
:10EA60007093C60F8093C70F9093C80F0C94778351
:10EA700083E50E945A5F882319F10E94465F20E0D7
:10EA800030E0A9010E94ADDC87FD0FC00E94465F07
:10EA900020E030E04FE753E40E94B0DE181644F067
:10EAA0000E94465F0E941CDD05C060E070E002C06D
:10EAB0006FEF70E070939A11609399110C947783C3
:10EAC0008FEF90E090939A11809399110C94778333
:10EAD00010929A11109299110C9477839B9AA39893
:10EAE00081E08093E60AE091C011F0E0EE0FFF1F95
:10EAF000E45EFD4F0190F081E02D808191810E94C4
:10EB0000B9970E9455980C9477830E94DD3D0E942E
:10EB1000D6C0149A0E9440C110929A111092991175
:10EB200068EE73E080E090E00E946DD79B9AA39A14
:10EB30001092E60AE091C011F0E0EE0FFF1FE45ED4
:10EB4000FD4F0190F081E02DE459FF4F408151814C
:10EB500021EA38E46FE978E485E99CE00E941447F3
:10EB60000E94B9970E9455980C9477831092C8110F
:10EB70000C94778381E08093C8110C94778383E5AC
:10EB80000E945A5F8823A1F00E94465F20E030E097
:10EB90004AE754E40E9482DF0E9421DD6093DD0A8F
:10EBA0007093DE0A8093DF0A9093E00A0C947783D7
:10EBB00088E50E945A5F81110C941D8589E50E94A9
:10EBC0005A5F81110C941D858AE50E945A5F81115C
:10EBD0000C941D8585E40E945A5F81110C941D855B
:10EBE0000C943F8583E50E945A5F882311F40C94AE
:10EBF00077830E94465F20E030E04AE754E40E94B9
:10EC000082DF0E9421DD6093C10F7093C20F809359
:10EC1000C30F9093C40F0C94778328EE3CE039AF78
:10EC200028AF01E31BE1E1E48E2EEBE19E2EF5EF30
:10EC3000AF2EFAE1BF2E312CE8ADF9AD8191F9AFDD
:10EC4000E8AF0E945A5F882309F45BC0F3E03F12EB
:10EC500051C00E94465F6B017C0120E030E040EA39
:10EC600051E40E94ADDC87FF3FC0A7019601F80187
:10EC700060817181828193810E94B4DC2B013C010F
:10EC80009B01AC016091091B70910A1B80910B1BC9
:10EC900090910C1B0E9482DF6093091B70930A1BEA
:10ECA00080930B1B90930C1BA3019201F4016081D4
:10ECB0007181828193810E9482DFF401608371837C
:10ECC00082839383F50160817181828193810E94A7
:10ECD0004DDDA30192010E9482DF0E9421DDF5013A
:10ECE0006083718382839383F801C082D182E28240
:10ECF000F38207C00E94465FF801608371838283BC
:10ED0000938333940C5F1F4FF4E08F0E911C24E02B
:10ED1000A20EB11C34E033128FCF0C947783909104
:10ED2000C00095FFFCCF8093C6003196849181117D
:10ED3000F6CF0C9477830091C90F1091CA0F0B5F27
:10ED40001F4F6AE270E0C8010E9439E4009711F099
:10ED5000FC011082C8010E9489970C947783ECE92A
:10ED6000F8E48491882341F09091C00095FFFCCF96
:10ED70008093C6003196F5CF4091AF115091B011FC
:10ED80006091B1117091B21122E030E08BE295E117
:10ED90000E9458B8E8E9F8E48491882341F0909102
:10EDA000C00095FFFCCF8093C6003196F5CF40910F
:10EDB000B3115091B4116091B5117091B61122E068
:10EDC00030E08BE295E10E9458B8E4E9F8E48491E0
:10EDD000882341F09091C00095FFFCCF8093C6003E
:10EDE0003196F5CF4091B7115091B8116091B9119A
:10EDF0007091BA1122E030E08BE295E10E9458B8A0
:10EE0000E0E9F8E48491882341F09091C00095FFF7
:10EE1000FCCF8093C6003196F5CF4091BB11509145
:10EE2000BC116091BD117091BE1122E030E08BE207
:10EE300095E10E9458B8E091C011F0E0EE0FFF1F7D
:10EE4000E45EFD4F0190F081E02DEC59FE4F019002
:10EE5000F081E02D8491882341F09091C00095FFCE
:10EE6000FCCF8093C6003196F5CF0E9432C10E943C
:10EE70004FDD2091311B3091321B4091331B50915B
:10EE8000341B0E94B4DCAB01BC0122E030E08BE219
:10EE900095E10E9458B8ECE8F8E48491882341F0A9
:10EEA0009091C00095FFFCCF8093C6003196F5CFBE
:10EEB00081E00E9432C10E944FDD2091351B3091CC
:10EEC000361B4091371B5091381B0E94B4DCAB01BC
:10EED000BC0122E030E08BE295E10E9458B8E8E8FE
:10EEE000F8E48491882341F09091C00095FFFCCF15
:10EEF0008093C6003196F5CF82E00E9432C10E9415
:10EF00004FDD2091391B30913A1B40913B1B5091B2
:10EF10003C1B0E94B4DCAB01BC0122E030E08BE280
:10EF200095E10E9458B88091C00085FFFCCF8AE02F
:10EF30008093C6000C94778380E00E9456B90C94AD
:10EF4000778381E00E9456B90C9477839091C0003A
:10EF500095FFFCCF8093C600319684918111F6CF46
:10EF60008091C00085FFFCCF8AE08093C600E091CD
:10EF7000C011F0E0EE0FFF1FE45EFD4F0190F08145
:10EF8000E02DEE58FE4F0190F081E02D8491882312
:10EF900041F09091C00095FFFCCF8093C600319660
:10EFA000F5CFE091C011F0E0EE0FFF1FE45EFD4FE2
:10EFB0001E9B13C00190F081E02DE058FE4F0190A0
:10EFC000F081E02D84918823D9F09091C00095FFC5
:10EFD000FCCF8093C6003196F5CF0190F081E02DF3
:10EFE000EE57FE4F0190F081E02D8491882341F08F
:10EFF0009091C00095FFFCCF8093C6003196F5CF6D
:10F000008091C00085FFFCCF8AE08093C600E0912C
:10F01000C011F0E0EE0FFF1FE45EFD4F0190F081A4
:10F02000E02DEC58FE4F0190F081E02D8491882373
:10F0300041F09091C00095FFFCCF8093C6003196BF
:10F04000F5CFE091C011F0E0EE0FFF1FE45EFD4F41
:10F05000029913C00190F081E02DE058FE4F01901D
:10F06000F081E02D84918823D9F09091C00095FF24
:10F07000FCCF8093C6003196F5CF0190F081E02D52
:10F08000EE57FE4F0190F081E02D8491882341F0EE
:10F090009091C00095FFFCCF8093C6003196F5CFCC
:10F0A0008091C00085FFFCCF8AE08093C600E0918C
:10F0B000C011F0E0EE0FFF1FE45EFD4F0190F08104
:10F0C000E02DEA58FE4F0190F081E02D84918823D5
:10F0D00041F09091C00095FFFCCF8093C60031961F
:10F0E000F5CFE091C011F0E0EE0FFF1FE45EFD4FA1
:10F0F0001D9B13C00190F081E02DE058FE4F019060
:10F10000F081E02D84918823D9F09091C00095FF83
:10F11000FCCF8093C6003196F5CF0190F081E02DB1
:10F12000EE57FE4F0190F081E02D8491882341F04D
:10F130009091C00095FFFCCF8093C6003196F5CF2B
:10F140008091C00085FFFCCF8AE08093C600E091EB
:10F15000C011F0E0EE0FFF1FE45EFD4F0190F08163
:10F16000E02DE858FE4F0190F081E02D8491882336
:10F1700041F09091C00095FFFCCF8093C60031967E
:10F18000F5CFE091C011F0E0EE0FFF1FE45EFD4F00
:10F19000019913C00190F081E02DE058FE4F0190DD
:10F1A000F081E02D84918823D9F09091C00095FFE3
:10F1B000FCCF8093C6003196F5CF0190F081E02D11
:10F1C000EE57FE4F0190F081E02D8491882341F0AD
:10F1D0009091C00095FFFCCF8093C6003196F5CF8B
:10F1E0008091C00085FFFCCF8AE08093C600E0914B
:10F1F000C011F0E0EE0FFF1FE45EFD4F0190F081C3
:10F20000E02DE658FE4F0190F081E02D8491882397
:10F2100041F09091C00095FFFCCF8093C6003196DD
:10F22000F5CFE091C011F0E0EE0FFF1FE45EFD4F5F
:10F230001C9B13C00190F081E02DE058FE4F01901F
:10F24000F081E02D84918823D9F09091C00095FF42
:10F25000FCCF8093C6003196F5CF0190F081E02D70
:10F26000EE57FE4F0190F081E02D8491882341F00C
:10F270009091C00095FFFCCF8093C6003196F5CFEA
:10F280008091C00085FFFCCF8AE08093C600E091AA
:10F29000C011F0E0EE0FFF1FE45EFD4F0190F08122
:10F2A000E02DE458FE4F0190F081E02D84918823F9
:10F2B00041F09091C00095FFFCCF8093C60031963D
:10F2C000F5CFE091C011F0E0EE0FFF1FE45EFD4FBF
:10F2D000379913C00190F081E02DE058FE4F019066
:10F2E000F081E02D84918823D9F09091C00095FFA2
:10F2F000FCCF8093C6003196F5CF0190F081E02DD0
:10F30000EE57FE4F0190F081E02D8491882341F06B
:10F310009091C00095FFFCCF8093C6003196F5CF49
:10F320008091C00085FFFCCF8AE08093C6000C94DA
:10F33000778380919B118093B80F84E50E945A5F78
:10F34000882381F10E94465F0E9421DD6093B80FFF
:10F35000662341F1E2E9F9E48491882341F0909138
:10F36000C00095FFFCCF8093C6003196F5CFE091A9
:10F37000C011F0E0EE0FFF1FE45EFD4F0190F08141
:10F38000E02DE05BFE4F0190F081E02D819188231C
:10F3900011F40C9477839091C00095FFFCCF80937B
:10F3A000C600F4CF84E40E945A5F882311F40C94C1
:10F3B00077830E94465F20E030E0A9010E94ADDC27
:10F3C000811103C01092BF1132C00091B80F10E03C
:10F3D0000E94465FF801EE0FFF1FEE0FFF1FED5E6C
:10F3E000F44F6083718382839383E090130BF090DA
:10F3F000140B0091150B1091160B20E030E0A901C1
:10F40000B701C8010E94ADDC811104C0E12CF12CD0
:10F4100000E410E4C701D8018093130B9093140B00
:10F42000A093150BB093160B81E08093BF110E943F
:10F43000A36A0C94778308EE1CE021E2E22E2BE114
:10F44000F22EF80181918F010E945A5F882349F0C2
:10F450000E94465F0E9421DDF701608371838283F1
:10F460009383F4E0EF0EF11C2CE00C3E120749F7F9
:10F470000E941DD30C94778308EE1CE091E4E92EE2
:10F480009BE1F92EF80181918F010E945A5F882338
:10F4900039F00E94465FF701608371838283938312
:10F4A000F4E0EF0EF11C2CE00C3E120759F70C941F
:10F4B000778383E50E945A5F882351F00E94465F5C
:10F4C0006093191B70931A1B80931B1B90931C1B3A
:10F4D00084E50E945A5F882311F40C9477830E947C
:10F4E000465F6093151B7093161B8093171B9093B8
:10F4F000181B0C94778383E50E945A5F882351F090
:10F500000E94465F60931D1B70931E1B80931F1B00
:10F510009093201B84E50E945A5F882351F00E943B
:10F52000465F6093051B7093061B8093071B9093A7
:10F53000081B82E40E945A5F882361F00E94465FA4
:10F540000E9421DD6093511B7093521B8093531BCB
:10F550009093541B88E50E945A5F882351F00E94C3
:10F56000465F6093111B7093121B8093131B909343
:10F57000141B8AE50E945A5F882351F00E94465F5F
:10F5800060930D1B70930E1B80930F1B9093101BA9
:10F5900085E40E945A5F882311F40C9477830E94BB
:10F5A000465F6093091B70930A1B80930B1B90931B
:10F5B0000C1B0C94778308EE1CE083EAE82E81E1B3
:10F5C000F82EF80181918F010E945A5F882339F04B
:10F5D0000E94465FF7016083718382839383F4E026
:10F5E000EF0EF11C2CE00B3E120711F40C94778304
:10F5F000E8CF83E50E945A5F882351F00E94465F5E
:10F600006093F30A7093F40A8093F50A9093F60AD4
:10F6100086E40E945A5F882381F00E94465F20E0C2
:10F6200030E040E752E40E94B4DC6093EB0A709350
:10F63000EC0A8093ED0A9093EE0A8AE50E945A5FE5
:10F64000882311F40C9477830E94465F6093931192
:10F650007093941180939511909396110C947783E5
:10F6600083E50E945A5F882351F00E94465F6093B1
:10F670008F1170939011809391119093921186E461
:10F680000E945A5F882311F40C9477830E94465F8E
:10F6900020E030E040E752E40E94B4DC6093E70AE7
:10F6A0007093E80A8093E90A9093EA0A0C947783AE
:10F6B00083E50E945A5F882311F40C9477830E949B
:10F6C000465F0E941CDD6115710551F061307105C6
:10F6D00069F481E080939811109297110C947783CC
:10F6E00010929811109297110C947783E2E9F9E443
:10F6F0008491882341F09091C00095FFFCCF8093C6
:10F70000C6003196F5CFE091C011F0E0EE0FFF1F7B
:10F71000E45EFD4F0190F081E02DE459FE4F019031
:10F72000F081E02D8491882341F09091C00095FFF5
:10F73000FCCF8093C6003196F5CF8091D30F909186
:10F74000D40F20E6289FF001299FF00D1124E752E5
:10F75000F04F8191882339F09091C00095FFFCCF44
:10F760008093C600F6CFE6E8F8E48491882341F060
:10F770009091C00095FFFCCF8093C6003196F5CFE5
:10F780008091C00085FFFCCF8AE08093C600AFC7A0
:10F7900083E50E945A5F882309F4A9C70E94465F47
:10F7A0000E941CDD70931E0B60931D0BA0C783E5A8
:10F7B0000E945A5F882309F49AC70E94465F0E94FC
:10F7C0001CDD6B017C0184E50E945A5F882381F077
:10F7D0008DED90E00E94A569811189C7E091B80F75
:10F7E000F0E0EE0FFF1FE75EF44FD182C0827FC7CB
:10F7F000D0921C0BC0921B0B7AC780E50E945A5F07
:10F80000882309F474C70E94465F0E941CDDD62E2F
:10F81000062F172F83E50E945A5F882331F00E943C
:10F82000465F0E941CDD7B0103C0EE24EA94FE2C9F
:10F83000C7010196039708F05AC7E0EBFCE08191FD
:10F8400091918017910709F452C73CE0E83EF30715
:10F85000B1F717FD4CC70E94D6C0CD2C60E08D2DAE
:10F860000E945ED68FEFE816F80631F0EA94EF2892
:10F8700071F000E010E00DC08D2D0E94CCD631E07B
:10F8800020E0892B09F030E0032F122F02C001E0A5
:10F8900010E08C2D0E94CCD68017910709F427C761
:10F8A0000E940A3B80E00E94D8680E945598F1CFE0
:10F8B00083E50E945A5F882331F00E94465F0E94D0
:10F8C0001CDD8B0102C00EE610E080E50E945A5F4D
:10F8D000882331F00E94465F0E941CDDCB0102C0EC
:10F8E00088EE93E06C01EE24D7FCE094FE2C101619
:10F8F00011067CF420E030E0A901B8018EE40E94FA
:10F900000AD8C701B6010E946DD78EE40E941BDBA6
:10F91000EEC6C701B6010E946DD7E9C680E50E9418
:10F920005A5F882351F00E94465F609318027093DB
:10F93000190280931A0290931B0289E40E945A5F75
:10F94000882361F00E94465F0E944F446093140236
:10F9500070931502809316029093170284E40E941C
:10F960005A5F882361F00E94465F0E945B44609367
:10F97000100270931102809312029093130283E499
:10F980000E945A5F882351F00E94465F60930C02E8
:10F9900070930D0280930E0290930F020E94BD3A65
:10F9A000E091C011F0E0EE0FFF1FE45EFD4F01900B
:10F9B000F081E02DE65CFE4F0190F081E02D819119
:10F9C000882339F09091C00095FFFCCF8093C6004A
:10F9D000F6CFEEE9FCE08191882339F09091C000E8
:10F9E00095FFFCCF8093C600F6CF4091180250914E
:10F9F000190260911A0270911B0222E030E08BE242
:10FA000095E10E9458B8E2EAFCE08191882339F040
:10FA10009091C00095FFFCCF8093C600F6CF609117
:10FA200014027091150280911602909117020E94A3
:10FA30005544AB01BC0122E030E08BE295E10E942D
:10FA400058B8E6EAFCE08191882339F09091C00033
:10FA500095FFFCCF8093C600F6CF609110027091A5
:10FA6000110280911202909113020E946144AB0135
:10FA7000BC0122E030E08BE295E10E9458B8EAEA4E
:10FA8000FCE08191882339F09091C00095FFFCCF74
:10FA90008093C600F6CF40910C0250910D02609108
:10FAA0000E0270910F0222E030E08BE295E10E949D
:10FAB00058B88091C00085FFFCCF8AE08093C600D3
:10FAC00016C683E50E945A5F882319F00E94465F9C
:10FAD00003C060E070E0CB010E9414D308C685E447
:10FAE0000E945A5F882341F00E94465F0E941CDDFD
:10FAF0008B0177FF03C009C000E010E0C12CD12CBE
:10FB0000F6E1EF2EF3E4FF2E06C0C12CD12CECE879
:10FB1000EE2EE2E4FE2E83E50E945A5F882321F058
:10FB20000E94465F6B017C0183E40E945A5F882338
:10FB300031F00E94465F0E941CDD9B0102C025E05F
:10FB400030E0A801C701B6010E94F03DD0C50E9477
:10FB5000D6C0CDC50E9489B40E945BB0C8C50E94C2
:10FB600089B4C5C50E945BB0C2C59091C00095FF25
:10FB7000FCCF8093C600319684918111F6CFE6E7E1
:10FB8000F8E48491882309F4B2C59091C00095FFF0
:10FB9000FCCF8093C6003196F4CF8AE50E945A5F6D
:10FBA000882309F4D6C00E94465F6B017C0120E0E7
:10FBB00030E040E751EC0E94B0DE87FD57C020E006
:10FBC00030E040EA50ECC701B6010E94ADDC1816E7
:10FBD0000CF44CC0F7FAF094F7F8F094C0929C1132
:10FBE000D0929D11E0929E11F0929F11E2E9F9E40A
:10FBF0008491882341F09091C00095FFFCCF8093C1
:10FC0000C6003196F5CFE091C011F0E0EE0FFF1F76
:10FC1000E45EFD4F80819181FC01E65CFE4F4081F6
:10FC20005181E255F10925E738E465E07DE0808106
:10FC300091810E941447FC012491222341F03091CC
:10FC4000C00035FFFCCF2093C6000196F4CF809111
:10FC5000C00085FFFCCF8AE08093C6008091C00081
:10FC600085FFFCCF8AE08093C60041C5E2E9F9E454
:10FC70008491882341F09091C00095FFFCCF809340
:10FC8000C6003196F5CFE091C011F0E0EE0FFF1FF6
:10FC9000E45EFD4F0190F081E02DE851FF4F0190AF
:10FCA000F081E02D8491882341F09091C00095FF70
:10FCB000FCCF8093C6003196F5CFE091C011F0E003
:10FCC000EE0FFF1FE45EFD4F0190F081E02DE6583E
:10FCD000FE4F0190F081E02D8491882341F09091B6
:10FCE000C00095FFFCCF8093C6003196F5CF4AE067
:10FCF00050E061EF7FEF8BE295E10E9482B7E091E7
:10FD0000C011F0E0EE0FFF1FE45EFD4F0190F081A7
:10FD1000E02DE458FE4F0190F081E02D849188237E
:10FD200041F09091C00095FFFCCF8093C6003196C2
:10FD3000F5CF4AE050E06BEF7FEF8BE295E10E9458
:10FD400082B78091C00085FFFCCF8AE08093C60017
:10FD5000CEC4E2E9F9E48491882341F09091C00097
:10FD600095FFFCCF8093C6003196F5CFE091C0118E
:10FD7000F0E0EE0FFF1FE45EFD4F0190F081E02DFB
:10FD8000E851FF4F61E778E4808191810E94F3465A
:10FD9000FC012491222341F03091C00035FFFCCFBB
:10FDA0002093C6000196F4CF8091C00085FFFCCF60
:10FDB0008AE08093C60040919C1150919D11609102
:10FDC0009E1170919F11705822E030E08BE295E116
:10FDD0000E9458B88091C00085FFFCCF8AE08093D4
:10FDE000C60085C480911D0B90911E0B9093180B3B
:10FDF0008093170BC090AF11D090B011E090B1116B
:10FE0000F090B211CF8ED8A2E9A2FAA20091B3115C
:10FE10001091B4112091B5113091B6110BA31CA310
:10FE20002DA33EA34091B7115091B8116091B91123
:10FE30007091BA114FA358A769A77AA78091BB11F7
:10FE40009091BC11A091BD11B091BE118BA79CA740
:10FE5000ADA7BEA7C982DA82EB82FC820D831E8326
:10FE60002F83388749875A876B877C878D879E8742
:10FE7000AF87B88B85E40E945A5F882359F00E94AF
:10FE8000465F9B01AC016BA57CA58DA59EA50E943C
:10FE9000D4DB0AC020E030E040E050E46BA57CA554
:10FEA0008DA59EA50E94D3DB6BA77CA78DA79EA7DF
:10FEB0009BE9C92E91E1D92EE12CF12C08EC13E439
:10FEC0009E01255D3F4FAE01495D5F4FBE016D5DF7
:10FED0007F4FCE014F960E9469C88AE50E945A5F03
:10FEE000882349F00E94465F9B01AC016FA178A571
:10FEF00089A59AA51EC020E030E040E050E46FA143
:10FF000078A589A59AA50E94D4DB6B017C016FA31B
:10FF100078A789A79AA720E030E040E251E40E9448
:10FF2000ADDC87FF0CC020E030E040E251E4C701C7
:10FF3000B6010E94D4DB6FA378A789A79AA7BBE973
:10FF4000CB2EB1E1DB2EE12CF12C06E913E49E016E
:10FF5000255D3F4FAE01495D5F4FBE016D5D7F4F37
:10FF6000CE014F960E9469C888E50E945A5F882397
:10FF700079F00E94465F9B01AC016F8D78A189A149
:10FF80009AA10E94D4DB6F8F78A389A39AA308C09B
:10FF900080E090E0A3E5B3E48F8F98A3A9A3BAA370
:10FFA00089E50E945A5F882339F00E94465F6BA35F
:10FFB0007CA38DA39EA304C01BA21CA21DA21EA2F3
:10FFC000FBE9CF2EF1E1DF2EE12CF12C0CE812E45D
:10FFD0009E01255D3F4FAE01495D5F4FBE016D5DE6
:10FFE0007F4FCE014F960E9469C88CE40E945A5FF1
:10FFF000882359F00E94465F9B01AC016BA57CA54C
:020000021000EC
:100000008DA59EA50E94D4DB0AC020E030E040EA26
:1000100052E46BA57CA58DA59EA50E94D3DB6BA7A2
:100020007CA78DA79EA77BE9C72E71E1D72EE12C77
:10003000F12C08EC13E49E01255D3F4FAE01495DB4
:100040005F4FBE016D5D7F4FCE014F960E9469C824
:100050000E94D6C0149A64E670E080E090E00E94AE
:100060006DD70E94E1A300E010E0F12C0E943D99C1
:1000700081111BC0F3940E940A3B81E00E94D86862
:10008000F110F4CF043FF1E01F0711F400E010E09D
:100090006A9A0115110511F4729A04C00431110510
:1000A00009F472980F5F1F4FE1CF729820E030E0A3
:1000B0004CE852E46BA57CA58DA59EA50E94D4DBDF
:1000C0006BA77CA78DA79EA74BE9C42E41E1D42E38
:1000D000E12CF12C00EA11E49E01255D3F4FAE01B9
:1000E000495D5F4FBE016D5D7F4FCE014F960E940F
:1000F00069C820E030E048E452E46BA57CA58DA5FA
:100100009EA50E94D4DB6BA77CA78DA79EA7E12CA0
:10011000F12C00E010E49E01255D3F4FAE01495DEA
:100120005F4FBE016D5D7F4FCE014F960E9469C843
:100130001092C2111092C1110E9477A48091C11136
:100140009091C211019709F47CC01092C2111092D3
:10015000C1110E94CAA48091C1119091C211823034
:10016000910549F1039709F069C020E030E048E4C7
:1001700052E46BA57CA58DA59EA50E94D4DB6BA740
:100180007CA78DA79EA7BBE9CB2EB1E1DB2EE12C8E
:10019000F12C00E010E49E01255D3F4FAE01495D6A
:1001A0005F4FBE016D5D7F4FCE014F960E9469C8C3
:1001B0000E9424A4C3CF20E030E04CE852E46BA5B9
:1001C0007CA58DA59EA50E94D4DB6BA77CA78DA7DF
:1001D0009EA79BE9C92E91E1D92EE12CF12C00EAD2
:1001E00011E49E01255D3F4FAE01495D5F4FBE01A9
:1001F0006D5D7F4FCE014F960E9469C820E030E0D0
:1002000048E452E46BA57CA58DA59EA50E94D4DB95
:100210006BA77CA78DA79EA7E12CF12C00E010E432
:100220009E01255D3F4FAE01495D5F4FBE016D5D93
:100230007F4FCE014F960E9469C87ECF0E940DA4C9
:100240007DCF20E030E040EA50E46BA57CA58DA591
:100250009EA50E94D4DB6BA77CA78DA79EA75BE918
:10026000C52E51E1D52EE12CF12C00E010E49E01C9
:10027000255D3F4FAE01495D5F4FBE016D5D7F4F14
:10028000CE014F960E9469C8A80197016BA57CA575
:100290008DA59EA50E94D3DB6BA77CA78DA79EA7EB
:1002A000E12CF12C08EC13E49E01255D3F4FAE01DB
:1002B000495D5F4FBE016D5D7F4FCE014F960E943D
:1002C00069C8E12CF12C0CE812E49E01255D3F4F3A
:1002D000AE01495D5F4FBE016B5F7F4FCE0101965E
:1002E0000E9469C8E12CF12C06E913E49E01255D0A
:1002F0003F4FAE01475F5F4FBE016B5F7F4FCE0147
:1003000001960E9469C820E030E040E050E46BA50F
:100310007CA58DA59EA50E94D4DB6BA77CA78DA78D
:100320009EA7E12CF12C08EC13E49E01255D3F4FC4
:10033000AE01475F5F4FBE016B5F7F4FCE010196FD
:100340000E9469C8CE010D960E94F0D28091170BD1
:100350009091180B80931D0B90931E0B9F938F937E
:1003600088E698E49F938F938E01015D1F4F1F9342
:100370000F930E9471E4C8010E943A5C0F900F90A5
:100380000F900F900F900F90B2C188E50E945A5FB6
:10039000882339F00E94465F0E941CDD80E00E94A5
:1003A00000C28AE50E945A5F882339F00E94465FA6
:1003B0000E941CDD81E00E9400C285E40E945A5F19
:1003C000882309F494C10E94465F0E941CDD82E0EC
:1003D0000E9400C28CC183E50E945A5F811104C053
:1003E00008EE1CE0F12C10C010E00E94465F0E9455
:1003F00021DD812F0E94D6C21F5F1530B1F7F0CFEB
:10040000F394F4E0FF1679F0F80181918F010E94D6
:100410005A5F8823A9F30E94465F0E9421DD8F2D39
:100420000E94D6C2EDCF82E40E945A5F882339F041
:100430000E94465F0E9421DD84E00E94D6C20E9495
:100440009CC355C183E50E945A5F882309F453C0B9
:100450000E94465F0E941CDD6130710541F06230F0
:10046000710509F048C008EE1CE0F12C25C008EE2B
:100470001CE0F12CF80181918F010E945A5F8823C2
:1004800041F00E94465F0E941CDD4FEF8F2D0E94BD
:1004900098C2F394F4E0FF12EDCF82E40E945A5F19
:1004A000882349F10E94465F0E941CDD4FEF20C067
:1004B000F394F4E0FF1689F0F80181918F010E9416
:1004C0005A5F8823A9F30E94465F0E941CDD462FD5
:1004D0006FEF8F2D0E9498C2EBCF82E40E945A5F8B
:1004E000882349F00E94465F0E941CDD462F6FEF73
:1004F00084E00E9498C20E949CC3F9C084E50E94D7
:100500005A5F882309F4A2C00E94465F0E9421DD41
:100510006093B80F662309F442C0E2E9F9E48491DC
:10052000882341F09091C00095FFFCCF8093C600D6
:100530003196F5CFEEEAFCE08191882339F0909175
:10054000C00095FFFCCF8093C600F6CF40E050E09E
:100550006091B80F8BE295E10E94B9B7E091C011AC
:10056000F0E0EE0FFF1FE45EFD4F0190F081E02D03
:10057000E059FE4F0190F081E02D8191882339F000
:100580009091C00095FFFCCF8093C600F6CF80917C
:10059000C00085FFFCCF8AE08093C600A8C086E437
:1005A0000E945A5F8823D9F00E94465F6B017C014C
:1005B00060936A1170936B1180936C1190936D111D
:1005C00020E030E0A9010E94B0DE181644F4C09289
:1005D000E10AD092E20AE092E30AF092E40AE2E948
:1005E000F9E48491882341F09091C00095FFFCCFFD
:1005F0008093C6003196F5CFE091C011F0E0EE0F88
:10060000FF1FE45EFD4F0190F081E02DE259FE4FA7
:100610000190F081E02D8191882339F09091C00004
:1006200095FFFCCF8093C600F6CF60919B1170E0E0
:100630004AE050E08BE295E10E9482B78091C000D1
:1006400085FFFCCF8AE08093C60051C0E2E9F9E45F
:100650008491882341F09091C00095FFFCCF809356
:10066000C6003196F5CFE091C011F0E0EE0FFF1F0C
:10067000E45EFD4F0190F081E02DE459FE4F0190C2
:10068000F081E02D8491882341F09091C00095FF86
:10069000FCCF8093C6003196F5CF8091D30F909117
:1006A000D40F20E6289FF001299FF00D1124E75276
:1006B000F04F8191882339F09091C00095FFFCCFD5
:1006C0008093C600F6CFE6E6F8E48491882341F0F3
:1006D0009091C00095FFFCCF8093C6003196F5CF76
:1006E0008091C00085FFFCCF8AE08093C6000E9405
:1006F000815FCBC1C0908611D0908711E0908811A6
:10070000F09089112091BB113091BC114091BD1125
:100710005091BE11C701B6010E94D3DB2DEC3CEC19
:100720004CEC5DE30E94B0DE181614F00C947B6B69
:10073000C092BB11D092BC11E092BD11F092BE11DB
:100740008BEB91E10E94F0D260E080E00E94F361C7
:100750009CC180E090E00E94A85A0C94846C81E0D7
:1007600090E00E94A85A0C948F6C82E090E00E9466
:10077000A85A0C94D86C0E940A3B80E00E94D8686A
:100780000E9455980C94D26F0E944F5FAB01BC0140
:1007900040936C1450936D1460936E1470936F14A7
:1007A00087EB93E10E94412FA2CF0E94465F0E94F7
:1007B0001CDD8B010C940F720E943ED768197909D9
:1007C0008A099B09693E73408105910508F479C047
:1007D000E6EBF8E48491882341F09091C00095FF06
:1007E000FCCF8093C6003196F5CFE091B80F24E09E
:1007F000E29FF0011124EA56F04F4081518162815D
:10080000738121E030E08BE295E10E9458B8E2EB81
:10081000F8E48491882341F09091C00095FFFCCFCB
:100820008093C6003196F5CF6091B80F70E04AE032
:1008300050E08BE295E10E9482B7EEEAF8E4849101
:10084000882341F09091C00095FFFCCF8093C600B3
:100850003196F5CFF7FE03C0E3E9FCE025C00E9426
:100860003ED78B019C01C701B6016854744F8F4F6E
:100870009F4F601B710B820B930BA30192010E948F
:100880008BE0BA01A9012AE030E08BE295E10E94F9
:10089000AEB78091C00085FFFCCF0DC09091C00025
:1008A00095FFFCCF8093C60081918111F7CF809195
:1008B000C00085FFFCCF3092C6000E943ED74B019E
:1008C0005C010E940A3B80E00E94D8680E94559813
:1008D000FFEFCF16DF06EF06FF0609F046C0809156
:1008E000B60FE091B80FF0E08F01000F111F000F5D
:1008F000111F0A56104FEE0FFF1FE256F04F608196
:1009000071818823C9F0882777FD8095982F0E94F0
:100910004FDD20E030E040E85FE30E94D3DB9B0145
:10092000AC01F80160817181828193810E94B0DE07
:1009300087FF50C00C94F173882777FD8095982F1E
:100940000E944FDD20E030E040E85FE30E94D4DB0E
:100950009B01AC01F80160817181828193810E94C9
:10096000ADDC1816BCF50C94F173F7FE02C00C94C4
:10097000F173E091B80FF0E08F01000F111F000F2D
:10098000111F0A56104FEE0FFF1FE256F04F608105
:100990007181882777FD8095982F0E944FDD9B01FC
:1009A000AC01F80160817181828193810E94D3DB67
:1009B0000E941CDD97FF07C090958095709561950A
:1009C0007F4F8F4F9F4F663071058105910514F45D
:1009D0000C94F1730E943ED76B017C010C94F1736F
:1009E000E091C011F0E0EE0FFF1FE45EFD4F0190BB
:1009F000F081E02DE45AFE4F808191810E94B997E9
:100A00008091D111882321F08CE49CE00E94899789
:100A10000E943ED76093BD0F7093BE0F8093BF0FAF
:100A20009093C00F0E943ED76093C50F7093C60F7E
:100A30008093C70F9093C80F5ACE0E94D6C088E506
:100A40000E945A5F882319F0179A1092A01189E525
:100A50000E945A5F882319F0169A1092A1118AE514
:100A60000E945A5F882319F0159A1092A21185E40A
:100A70000E945A5F882309F43ACE149A38CE0E9415
:100A8000D6C0149A0E9440C132CEE9960FB6F894AF
:100A9000DEBF0FBECDBFDF91CF911F910F91FF90B1
:100AA000EF90DF90CF90BF90AF909F908F907F900E
:100AB0006F905F904F903F900895CF93DF93809118
:100AC000CF0F9091D00F039714F40E94B36460E0AD
:100AD0008FEC91E10E9498518091CF0F9091D00FAF
:100AE000892B09F47EC08091CF118823E1F0809199
:100AF000D30F9091D40F20E6289FE001299FD00DBD
:100B00001124C752D04F62E079E4CE010E94E4E3A1
:100B1000892B59F5BE018FEC91E10E941A51809109
:100B2000D011882319F00E94B56A45C0E091C01128
:100B3000F0E0EE0FFF1FE45EFD4F0190F081E02D2D
:100B4000E65CFE4F0190F081E02D8491882341F016
:100B50009091C00095FFFCCF8093C6003196F5CFF1
:100B60008091C00085FFFCCF23C060E08FEC91E155
:100B70000E948E52E091C011F0E0EE0FFF1FE45E84
:100B8000FD4F0190F081E02DE45CFE4F0190F0817B
:100B9000E02D8491882341F09091C00095FFFCCF17
:100BA0008093C6003196F5CF8091C00085FFFCCFC1
:100BB0008AE08093C6008091CF0F9091D00F01976B
:100BC0009093D00F8093CF0F8091D30F9091D40F3B
:100BD000019664E070E00E9478E09093D40F8093D7
:100BE000D30F0E940A3B80E00E94D8680E9477B829
:100BF000DF91CF910C9455988F929F92AF92BF92B4
:100C0000CF92DF92EF92FF920F931F93CF93DF93D8
:100C10008C018C519E4F0E94DF4A680189E8C80E02
:100C2000D11C21F1780181E4E81A8EEFF80AE7017E
:100C300057018FE1A81AB10863E2862E6DE0962E67
:100C4000CC15DD0599F0FE01EE19FF09EA0DFB1D3B
:100C500091828082FE0178978081811102C06F9716
:100C6000EFCFCE014B970E942430F9CFC8018659AF
:100C70009F4F0E94DF4AC801875B9F4FDF91CF9152
:100C80001F910F91FF90EF90DF90CF90BF90AF90AA
:100C90009F908F900C94DF4A8FEC91E10C94EB4A7B
:100CA0008FEC91E1A9CFFB016091300B7091310B7A
:100CB00070939F1460939E146091A8147091A9146E
:100CC00070939D1460939C1462E060932F0B65E811
:100CD00071EA7093310B6093300B90939B14809367
:100CE0009A14F0939914E0939814662757FD609531
:100CF000762F4093941450939514609396147093A8
:100D00009714C901AA2797FDA095BA2F841B950BAC
:100D1000A60BB70B8093901490939114A093921408
:100D2000B093931480819181AA2797FDA095BA2F43
:100D3000841B950BA60BB70B8093A8149093A91452
:100D4000A093AA14B093AB140895CF93DF93CDB7BB
:100D5000DEB7C054D1090FB6F894DEBF0FBECDBFC9
:100D600088E0E7E6FBE0DE01D99601900D928A95D6
:100D7000E1F788E0EFE6FBE0DE01D19601900D920D
:100D80008A95E1F788E0E7E7FBE0DE0199960190BC
:100D90000D928A95E1F788E0EFE7FBE0DE0191969E
:100DA00001900D928A95E1F788E0E7E8FBE0DE012B
:100DB000599601900D928A95E1F788E0EFE8FBE003
:100DC000DE01519601900D928A95E1F788E0E7E9FE
:100DD000FBE0DE01199601900D928A95E1F788E01B
:100DE000EFE9FBE0DE01119601900D928A95E1F7A3
:100DF000AE01475C5F4F60E083EB94E10E94B44634
:100E0000AE014F5C5F4F61E083EB94E10E94B4461A
:100E1000AE01475D5F4F62E083EB94E10E94B44610
:100E2000AE014F5D5F4F63E083EB94E10E94B446F7
:100E3000AE01475E5F4F64E083EB94E10E94B446ED
:100E4000AE014F5E5F4F65E083EB94E10E94B446D4
:100E5000AE01475F5F4F66E083EB94E10E94B446CA
:100E6000AE014F5F5F4F67E083EB94E10E94B446B1
:100E7000C05CDF4F0FB6F894DEBF0FBECDBFDF9171
:100E8000CF9108950F931F93CF93DF93EB01142F0E
:100E9000022F482F60E083EB94E10E941645612FFA
:100EA00083EB94E10E94CCDB11E1FE0164916623A7
:100EB00011F0111117C0112339F060E283EB94E1B6
:100EC0000E94CCDB1150F7CF602F83EB94E10E949E
:100ED000CCDB60E283EB94E1DF91CF911F910F9126
:100EE0000C94CCDB83EB94E10E94CCDB2196115077
:100EF000DCCFEF92FF920F931F93CF93DF93EB0121
:100F0000E42E8901F90101900020E9F7F22EFE1A82
:100F100092E1F90E482F60E083EB94E10E941645C0
:100F20006E2D83EB94E10E94CCDBFE01649166237D
:100F300011F0F11019C06AE383EB94E10E94CCDB5D
:100F4000FF2039F060E283EB94E10E94CCDBFA945D
:100F5000F7CFB80183EB94E1DF91CF911F910F910F
:100F6000FF90EF900C94CBDB83EB94E10E94CCDB01
:100F70002196FA94DACF8093C01191E09093320BCE
:100F8000682F88EF9FE00E9495E68091871481305A
:100F900019F482E0809387140895109222158FEC43
:100FA00091E10E94A1571092B11408958FEC91E144
:100FB0000C94804E8FEC91E10C94874ECF9382E09D
:100FC00080932F0B0E943ED76C507E4F8F4F9F4FC8
:100FD0006093AD147093AE148093AF149093B014DB
:100FE0006A9ACAE0729A84E690E00E9491D7729859
:100FF00084E690E00E9491D7C150A1F7CF91089567
:10100000E091300BF091310BE817F90771F09093F4
:10101000310B8093300B4093A8145093A914609324
:10102000AA147093AB142111C9CF089521E040E0B8
:1010300050E0BA01E5CF21E040E050E0BA01E0CF56
:10104000CF92DF92EF92FF920F931F93CF93DF9394
:101050008091A8149091A914A091AA14B091AB14F6
:1010600081309048A105B10540F01092A81410926B
:10107000A9141092AA141092AB148091A814909104
:10108000A914A091AA14B091AB14B695A795979501
:1010900087954091B11450E060E070E084179507A7
:1010A000A607B70710F48093B114D091B114109132
:1010B000B21412FB112710F9C0E0B1E1CB2ED12CF4
:1010C000E12CF12C01E04091A8145091A9146091F9
:1010D000AA147091AB14D11138C080912F0B8823C2
:1010E000C1F0E091C011F0E0EE0FFF1FE45EFD4F94
:1010F0000190F081E02D8681978123E042305105F7
:101100006105710510F443E001C040E2BC018C2F81
:10111000B9DE112309F49CC18091A8149091A914FF
:10112000A091AA14B091AB140297A105B10508F0E3
:101130008FC144DF8AE096EADF91CF911F910F9132
:10114000FF90EF90DF90CF9071CFD13051F580912B
:101150002F0B882389F0769567955795479523E05F
:10116000413051056105710511F443E001C040E2D1
:1011700060EA7AE48C2F86DE112309F469C180913C
:10118000A8149091A914A091AA14B091AB14B6958B
:10119000A795979587950197A105B10509F058C1C5
:1011A000C8CFD230B9F580912F0B8823F1F0E091B0
:1011B000C011F0E0EE0FFF1FE45EFD4F0190F081E3
:1011C000E02DE854FE4F8081918176956795579583
:1011D000479523E0423051056105710511F443E064
:1011E00001C040E2BC018C2F4DDE112309F430C157
:1011F0008091A8149091A914A091AA14B091AB1455
:10120000B695A795979587950297A105B10509F021
:101210001FC18FCFD330B9F580912F0B8823F1F008
:10122000E091C011F0E0EE0FFF1FE45EFD4F019072
:10123000F081E02DE654FE4F80819181769567958F
:101240005795479523E0433051056105710511F429
:1012500043E001C040E2BC018C2F14DE112309F4ED
:10126000F7C08091A8149091A914A091AA14B091EC
:10127000AB14B695A795979587950397A105B105EA
:1012800009F0E6C056CFD430B9F580912F0B8823F2
:10129000F1F0E091C011F0E0EE0FFF1FE45EFD4FB2
:1012A0000190F081E02DE454FE4F8081918176958C
:1012B00067955795479523E04430510561057105C1
:1012C00011F443E001C040E2BC018C2FDBDD1123AF
:1012D00009F4BEC08091A8149091A914A091AA14F9
:1012E000B091AB14B695A795979587950497A105EE
:1012F000B10509F0ADC01DCFD53051F580912F0B50
:10130000882389F0769567955795479523E0453072
:1013100051056105710511F443E001C040E263E944
:101320007AE48C2FAFDD112309F492C08091A814C8
:101330009091A914A091AA14B091AB14B695A79559
:10134000979587950597A105B10509F081C0F1CE64
:10135000D63051F580912F0B882389F076956795CB
:101360005795479523E0463051056105710511F405
:1013700043E001C040E26CE87AE48C2F83DD112366
:1013800009F466C08091A8149091A914A091AA14A0
:10139000B091AB14B695A795979587950697A1053B
:1013A000B10509F055C0C5CED73041F580912F0B5E
:1013B000882389F0769567955795479523E04730C0
:1013C00051056105710511F443E001C040E263E895
:1013D0007AE48C2F57DD1123D9F18091A8149091D4
:1013E000A914A091AA14B091AB14B695A79597959E
:1013F00087950797A105B10559F59BCED83041F5E2
:1014000080912F0B882389F076956795579547959E
:1014100023E0483051056105710511F443E001C036
:1014200040E269E77AE48C2F2DDD112389F0809169
:10143000A8149091A914A091AA14B091AB14B695D8
:10144000A795979587950897A105B10509F471CEE1
:101450008091A8149091A914A091AA14B091AB14F2
:101460004297A105B10540F0C092A814D092A914EA
:10147000E092AA14F092AB144091A8145091A914D0
:101480006091AA147091AB1476956795579547951E
:101490008091B11490E00396242F30E082179307D7
:1014A0004CF48DEF840F8093B11400932F0BDCEF7D
:1014B000D40FCFEFCF5FDF5FC43008F404CEDF91ED
:1014C000CF911F910F91FF90EF90DF90CF900895F3
:1014D0007F928F929F92AF92BF92CF92DF92EF92C4
:1014E000FF920F931F93CF93DF938091A814909155
:1014F000A914A091AA14B091AB1481309048A10511
:10150000B10540F01092A8141092A9141092AA14D8
:101510001092AB148091A8149091A914A091AA14D0
:10152000B091AB14B695A795979587954091B11456
:1015300050E060E070E084179507A607B70710F445
:101540008093B114E090B114D090B214D2FADD249B
:10155000D0F8F12CCC24C3948091871481113BC026
:10156000EE2019F07724739437C080912F0B8823D5
:1015700001F1E091C011F0E0EE0FFF1FE45EFD4FBE
:101580000190F081E02DEA50FF4F608171818091E0
:10159000A8149091A914A091AA14B091AB1423E0BF
:1015A0000297A105B10510F443E001C040E28F2D80
:1015B00069DCDD20B9F28091A8149091A914A09162
:1015C000AA14B091AB140297A105B10558F6F6DC48
:1015D00087EB94E951C0712C80918714823009F017
:1015E0005AC07E1057C080912F0B882359F1E0918B
:1015F000C011F0E0EE0FFF1FE45EFD4F0190F0819F
:10160000E02DE055FF4F0190F081E02D8091A8146E
:101610009091A914A091AA14B091AB14B695A79576
:1016200097958795472D50E060E070E023E08417A0
:101630009507A607B70711F443E001C040E2BF01D8
:101640008F2D20DCDD2031F18091A8149091A91418
:10165000A091AA14B091AB14B695A79597958795CC
:10166000472D50E060E070E084179507A607B707A4
:1016700089F4A4DC8EE19DEADF91CF911F910F9157
:10168000FF90EF90DF90CF90BF90AF909F908F90A2
:101690007F90CCCC73940CE112E0C0E0D0E08E2CB3
:1016A000912CA12CB12C7E104AC080912F0B882345
:1016B00019F1D801ED91FC91EC54FE4F60817181DC
:1016C0008091A8149091A914A091AA14B091AB1480
:1016D000B695A79597958795272D30E040E050E087
:1016E00082179307A407B50719F420E24EE302C05E
:1016F00020E240E28F2DC6DBDD2009F18091A814A5
:101700009091A914A091AA14B091AB14B695A79585
:101710009795879588159905AA05BB0581F44EDC38
:101720008C2FDF91CF911F910F91FF90EF90DF9061
:10173000CF90BF90AF909F908F907F901CCC739470
:1017400021960E5F1F4FC530D10509F0ACCF4091F7
:10175000A8145091A9146091AA147091AB147695B5
:10176000679557954795872D90E0A0E0B0E0481722
:1017700059076A077B0788F0872D90E0880F991F2B
:101780000197AA2797FDA095BA2F8093A81490934C
:10179000A914A093AA14B093AB144091A81450912B
:1017A000A9146091AA147091AB147695679557951A
:1017B00047958091B11490E00396242F30E0821772
:1017C00093075CF48DEF840F8093B114C0922F0BBC
:1017D000DCEFED2EE40EFF24FA94F394E394B3E0EF
:1017E000BF1508F0B9CEDF91CF911F910F91FF90F7
:1017F000EF90DF90CF90BF90AF909F908F907F90B1
:1018000008950F931F93CF93DF938091A814909125
:10181000A914A091AA14B091AB1481309048A105ED
:10182000B10540F01092A8141092A9141092AA14B5
:101830001092AB148091A8149091A914A091AA14AD
:10184000B091AB14B695A795979587954091B11433
:1018500050E060E070E084179507A607B70710F422
:101860008093B114D091B1141091B21412FB1127CE
:1018700010F9C0E001E08091A8149091A914A09102
:10188000AA14B091AB14D11134C020912F0B222394
:10189000C1F0E091C011F0E0EE0FFF1FE45EFD4FDC
:1018A0000190F081E02DEA50FF4F6081718123E0CB
:1018B0000297A105B10510F443E001C040E28C2F6E
:1018C000E1DA112309F482C08091A8149091A9143F
:1018D000A091AA14B091AB140297A105B10508F02C
:1018E00075C06CDB87EB94E9DF91CF911F910F916D
:1018F0009DCBD130A9F520912F0B2223D1F0E0917F
:10190000C011F0E0EE0FFF1FE45EFD4F0190F0818B
:10191000E02D62AD73ADB695A795979587952EE7A7
:101920000197A105B10511F44EE301C040E28C2FEF
:10193000A9DA112309F44AC08091A8149091A9143E
:10194000A091AA14B091AB14B695A79597958795D9
:101950000197A105B105D1F531DB81ED92EABFC058
:10196000D230A1F520912F0B2223D1F0E091C011AC
:10197000F0E0EE0FFF1FE45EFD4F0190F081E02DDF
:1019800064AD75ADB695A795979587952EE70297A7
:10199000A105B10511F44EE301C040E28C2F72DACB
:1019A0001123A1F08091A8149091A914A091AA14D8
:1019B000B091AB14B695A795979587950297A10519
:1019C000B10521F4FBDA88ED92EA89C020E030E02D
:1019D00040E251E4609183147091841480918514E5
:1019E000909186140E94ADDC87FF7EC08091A81480
:1019F0009091A914A091AA14B091AB14D330B1F571
:101A000020912F0B2223D1F0E091C011F0E0EE0FD6
:101A1000FF1FE45EFD4F0190F081E02D66AD77ADD4
:101A2000B695A795979587952EE70397A105B105DC
:101A300011F44EE301C040E28C2F24DA111102C0F0
:101A400025E053C08091A8149091A914A091AA14E4
:101A5000B091AB14B695A795979587950397A10577
:101A6000B10571F7ABDA8FED92EA39C0D43041F7A6
:101A700020912F0B2223E1F0E091C011F0E0EE0F56
:101A8000FF1FE45EFD4F0190F081E02DE05CFF4F11
:101A900060817181B695A795979587952EE70497F4
:101AA000A105B10511F44EE301C040E28C2FEAD943
:101AB000112331F24091A8145091A9146091AA14F5
:101AC0007091AB14769567955795479544305105BD
:101AD0006105710509F0B4CF71DA8BE091EADF910D
:101AE000CF911F910F91A7CA23E04091A814509164
:101AF000A9146091AA147091AB14769567955795C7
:101B00004795822F90E0A0E0B0E0481759076A0798
:101B10007B0788F0822F90E0880F991F0197AA27F2
:101B200097FDA095BA2F8093A8149093A914A09321
:101B3000AA14B093AB144091A8145091A9146091C9
:101B4000AA147091AB147695679557954795809137
:101B5000B11490E00396242F30E0821793074CF4E1
:101B60008DEF840F8093B11400932F0BDCEFD40F13
:101B7000CFEFCF5FDF5FC43008F47DCEDF91CF9130
:101B80001F910F91089580E090E0A0E8BFE380935B
:101B9000831490938414A0938514B093861431CE4B
:101BA00020E044E064E183EB94E10E944945CDD814
:101BB00083EB94E10C940A45F3DF20E040E050E031
:101BC000BA018EE19DEA1CCA10929F0F10929E0FDF
:101BD00010929D0F10929C0F10929A1110929911D1
:101BE000EBCF83EB94E10C940A4580911F15909103
:101BF000201590939F0F80939E0F80911D159091BB
:101C00001E1590939D0F80939C0F10929A11109225
